:020000040800F2
:100000000002002029050008C5040008810400083A
:10001000D5040008E5040008F5040008000000000D
:10002000000000000000000000000000450400087F
:100030000505000800000000290400081505000857
:100040008901000889010008890100088901000868
:10005000890100088901000899160008991600080E
:1000600099160008991600089916000889010008D9
:100070008901000889010008890100088901000838
:100080008901000889010008890100088901000828
:1000900089010008890100088901000899160008F3
:1000A0008901000889010008890100088901000808
:1000B0003118000889010008890100088901000839
:1000C00089010008890100088901000889010008E8
:1000D0008901000889010008491200084F12000830
:1000E00099160008890100088901000889010008A3
:1000F00089010008890100088901000889010008B8
:1001000089010008890100083718000889010008E2
:100110008901000889010008890100088901000897
:100120008901000889010008890100088901000887
:100130008901000889010008890100088901000877
:100140008901000889010008890100088901000867
:100150008901000889010008890100088901000857
:100160008901000889010008890100088901000847
:1001700089010008890100088901000800000000C9
:10018000000000008901000800F0C4B900F004BBC1
:100190007047000070B50C46064600F061F9094B47
:1001A000094A1D682919914202D8084A914204D28D
:1001B0000C2333604FF0FF3500E0196000F058F970
:1001C000284670BD0002002000000220FC510020E3
:1001D0001946104600F0ECBA1946104600F0F0BA85
:1001E000132303604FF0FF307047132303604FF079
:1001F000FF307047132303604FF0FF307047022930
:100200004FF0000303608CBF002001207047000006
:10021000114B70B500241C60104B114D18682E68EE
:1002200000F09CF80F4B53F820301B68A3F1080234
:1002300096420FD026B13179092904BF0A213171C4
:10024000092103F8041C33F9021C074B2A601980AA
:10025000012070BD204670BD00030020D4030020A3
:10026000080300201003002004030020082930B5F3
:10027000037919D9082B32D842791A4B53F82250F6
:1002800000F108042DB12D68856053F822502C60D0
:1002900000E0846043F82240134C4279012303FAC2
:1002A00002F22368134319E0082B18D945790D4B46
:1002B00053F825203AB11468A2420BBF00222468EB
:1002C00043F825201460427953F822303BB9064C9C
:1002D000012303FA02F2236823EA02032360017177
:1002E00030BD00BF10030020D403002008B50A4B26
:1002F0001B681A79082A02D95B7983420AD900F06F
:10030000BAF818B1054B01221A6008BDBDE80840D3
:1003100000F082B808BD00BF0803002000030020E1
:1003200008B500F09DF8094B094A1B88094D1BB21E
:10033000002442F82340084A286813682146013BFC
:100340001360FFF793FF2C6000F062F804030020B5
:1003500050030020080300200C0300200023C207E4
:1003600002D440080133FAE718467047134423F0DB
:10037000030310B54FF077321C1F43F8042C6207BB
:1003800042BF4FF0883243F8082CA3F108044FF025
:10039000807304E909000F4B44F80C3C002344F837
:1003A000103C032344F8143C2246022344F8183C32
:1003B000012344F81C3C42F8201D0B2342F8043D65
:1003C000013B032BFAD120466FF0020340F8443D75
:1003D00010BD00BF21030008064B0749074A1868F3
:1003E000884203D1934201D20433F8E70348C01A8C
:1003F000704700BF00000020FEE7FEE7000200207B
:10040000EFF30880704700000048704700000020AC
:1004100000F02AF801DFFEE7024A536843F08053F8
:100420005360704700ED00E0EFF3098020E9F00F22
:1004300040F804ED02490968086000F003F8000084
:1004400008030020FFF7E4FE04480068016801C9C2
:10045000B1E8F00F81F3098800470000080300208D
:10046000EFF3108072B6704762B6EFF310807047FA
:1004700080F310887047EFF30580C0B2704700002A
:100480000D490E4A0E4B6846904203D8984201D956
:10049000002102E009468D460121042072460242F5
:1004A00002D1EFF3088001E0EFF309802DE9F00FAE
:1004B0006B4600F06FF800BF000200200000022031
:1004C0006005002008B50249042000F08DFB00BF44
:1004D0008C07010808B50249062000F085FB00BF23
:1004E0009807010808B50249072000F07DFB00BF0E
:1004F000AB07010808B50249082000F075FB00BFF2
:10050000BD07010808B50249092000F06DFB00BFD6
:10051000D107010808B502490A2000F065FB00BFB9
:10052000E30701087047704708B5FFF7FBFF6A460D
:10053000114B1249934202D243F8041BFAE7104AC6
:10054000104B11498B4204D252F8040F43F8040BAC
:10055000F8E70E4B0E4A0021934202D243F8041BE7
:10056000FAE7FFF7E0FF00F01FFB0EF0F9F9BDE836
:10057000084000F073BB00BF00000020FEE7FEE76C
:10058000D8420108000200200003002000030020E0
:10059000FC5100202DE9F04F9A46494B8FB093460D
:1005A0009A6B03925A6B04929F6ADA6A05921A6BED
:1005B000DB6B0793434B06921A68434B9A420446FF
:1005C000884602D041480EF0B5FCB8F1000F05D0C6
:1005D0003F4800250EF0AEFC2E4626E094E80E00C3
:1005E000E068D4F81C9008902069099060690A902E
:1005F00019F4007F3748A6690D930CBF04F120055C
:1006000004F124050C920B910EF094FC089B0093CE
:100610000BA90EC930480EF003FCCDF8009033460C
:100620000A9A09992D480EF0FBFB2D480EF082FC2A
:1006300039462C480EF0F4FB05992B480EF0F0FBE0
:1006400006992A480EF0ECFB079929480EF0E8FBC2
:100650003A0403D5039927480EF0E2FB3B0603D585
:10066000049925480EF0DCFB24480EF063FC594643
:1006700023480EF0D5FBB8F1000F1BD121480EF036
:1006800059FC314620480EF0CBFB69461F4BC91A76
:1006900003D549421E480EF0C3FB20468268C3685A
:1006A00001698C4641698E46AD46514691E8F00F8E
:1006B0004168006801BE1749052000F095FA00BFA7
:1006C00000ED00E000000020FEE7FEE7F107010872
:1006D0000708010836080108510801088E080108BA
:1006E000CC080108D5080108E5080108F50801084B
:1006F000050901081509010825090108350901083E
:100700003A0901084C0901087D0901085801002037
:10071000A5090108D209010810B568B1012815D151
:10072000174A136823F003031360136843F400733C
:1007300043F0010313601BE0114B1A6842F00E02F4
:100740001A605A6842F480725A6011E00D4A1369C7
:1007500023F0040313610024FFF782FEBFF34F8FE1
:1007600030BFFFF785FE54B1BDE8104000F010BC6B
:10077000044A136943F0040313610124ECE710BD3C
:100780000070004000ED00E008B5FFF769FE0020B2
:10079000BDE80840FFF7C0BF034B044A4FF4E13106
:1007A000002000F0C7BC00BF04020020270E000894
:1007B0000A460146014800F041BB00BF0402002088
:1007C00010B50A460C460146002000F019FD2046EF
:1007D00010BD002000F0D6BF034B1968024611B9C6
:1007E000084600F0AFBF70471C04002010B5094A4E
:1007F00013685BB19C6881688C4202D21A461B6800
:10080000F7E703D15C6841688C42F7D90360106058
:1008100010BD00BF28040020F0B51F4E1F4D3368E7
:100820001F4C013333601F4B00201A6818602B687F
:10083000226019460746B64641B1DEF800C08E6810
:10084000664503D80F4601200968F5E700B1296025
:1008500007B9F0BD00213960E2B133B15168586881
:10086000814294BF1146194600E0114608461268BD
:100870001B680AB903600BE00BB9026008E0556819
:100880005E68B54294BF15461D4605602846EEE7F2
:100890002160F0BD2360F0BD20040020280400206A
:1008A00024040020180400202DE9F0412E4F2F4C85
:1008B00001233B6023683BB9FFF7AEFFFFF789FFD9
:1008C0000130FBD0002502E0FFF783FF05464FF023
:1008D0000008236823B9FFF77CFF854214D91AE08A
:1008E0005E68FFF776FF854208D923685E68FFF7E8
:1008F00070FFA8422CD3B042F7D329E08642F4D946
:10090000361A132EE7D8F0E7236843B9FFF761FFE3
:10091000854206460BD9FFF77FFF0025D9E75E68C1
:10092000FFF757FF063E14308642D2D309E010F19C
:10093000140F04D3FFF74DFF8642FBD9EBE74FF0CE
:10094000FF3600233B603046BDE8F041FFF744BF6F
:1009500023681A682260C3F80480C3F80880DA6844
:1009600018699047B5E700BF1C040020240400204C
:10097000144B1A6882420AD112681A6012B1506888
:10098000063801E04FF0FF30FFF726BF13461A6824
:1009900022B19042FAD102681A6070470A4A13687D
:1009A0001BB1984203D01A46F9E7084A05E00368EC
:1009B000136070479842FAD01A461368002BF9D199
:1009C000704700BF240400201804002028040020E1
:1009D00008B500231846054A054900F0E5FE4FF02A
:1009E000FF30BDE80840FFF7F7BE00BFA9080008C8
:1009F00040420F0070B5084EFFF7EBFE3468054625
:100A0000FFF7E7FE8542F7D800222346141843F18A
:100A100000052046294670BD20040020F8B5044694
:100A20000D46FFF7D6FE002385420646236010D30D
:100A3000A5F10A0383420CD20A35FFF7CAFE8542AC
:100A4000FBD3FFF7C6FE8542FBD8E36820699847D1
:100A50003EE0FFF705FD63680746002B34D1A3682D
:100A6000002B31D11B4B65601A681B68B54238BF3B
:100A70000132A260A2689A4203D92046FFF7B6FE6F
:100A80001EE0B54202D9144B19460EE0134A136812
:100A900023B159688D4201D31A46F8E723601460E8
:100AA0000EE05068854203D313461A68002AF8D135
:100AB00022601C600B689C4202D1A81FFFF78CFECD
:100AC0003846FFF7D5FC03E02046FFF751FFC9E7A2
:100AD0000020F8BD20040020240400201804002079
:100AE00038B50446FFF7BCFC6368054633B9A36814
:100AF00023B92846BDE83840FFF7BABC2046FFF7C7
:100B000037FFF6E7C36870B504460D46C3B1FFF77B
:100B1000E7FF092D0CD8FFF75CFE0646FFF759FEEC
:100B2000801B8542FAD8E3682069BDE87040184709
:100B3000FFF74FFE29182046BDE87040FFF76EBF53
:100B400070BD00002DE9F04704460E4690461AB9E4
:100B5000BDE8F047FFF7D6BFFFF782FC63680746A2
:100B6000E3B9A368D3B9DFF83CA0FFF732FEDAF8A7
:100B700000508146FFF72DFE8145F6D8304408EB42
:100B80000502864288BF01326060A2602046FFF7FE
:100B90002DFE3846BDE8F047FFF76ABC2046FFF758
:100BA000E7FEE0E72004002008B50121094800F035
:100BB0009BFC0121084800F097FC0121074800F048
:100BC00093FC0121064800F08FFCBDE8084000F0CE
:100BD00021B900BF0D0C02400C0C02400E0C02406B
:100BE0000F0C02407047000008B50F4B1A680C4606
:100BF0009AB9012203281A6003D171460B480EF0FE
:100C00000FF921460A480EF00BF900F04FF9094898
:100C10000EF006F908480EF003F9FFF721FCFFF784
:100C2000E1FFFFF7B1FD00BF2C040020F709010828
:100C3000FB090108230A0108170A010808B500F09A
:100C4000EBFF03480EF0ECF800F020FE002008BD9A
:100C5000250A010808B500F00BF9FCE71FB5FFF7FE
:100C6000FFFB0E4B0E481B68029300240D4B0093B4
:100C70000F220C234FF48071019400F055F80A4BB9
:100C80000A481B6802930A4B009307220C234FF477
:100C9000C061019400F048F8FFF7BAFB1802002089
:100CA00030040020550C00081C02002030050020F4
:100CB0003D0C000808B5FFF7D3FB094B1B681A79F8
:100CC000082A07D95A79074B53F8221011B109683D
:100CD00043F82210FFF7CCFBBDE80840FFF79CBBB0
:100CE000080300201003002038B50B79082B03D926
:100CF00008490320FFF778FF4C7901F108020368E7
:100D00002BB113F8035CAC4201D31846F7E78B60B4
:100D1000026038BDE5090108031F53F8042F9A4209
:100D2000FBD0181A704700000F2A2DE9F74F05462F
:100D30008B4691469A462AD810F003031BBFC3F195
:100D40000403ED180B46CB1A303B23F003031AF0D3
:100D5000080F05EB030405D02A46A24203D2126015
:100D60000432FAE72D600193FFF77AFB2749019BD4
:100D70008046012251F8227016B25FB10132212A59
:100D8000F8D14046FFF774FB6FF08A003BE06FF04C
:100D9000150038E01D490C9841F822402A46E680AB
:100DA0000D99FFF7E3FA0E9B194AA3624FF0FF3348
:100DB000E3611368206001331AF0010F6562C4F823
:100DC0002CB084F805902771A760E7602761676100
:100DD000A7612762136004D001212046FFF746FA7D
:100DE0000DE00A212046FFF741FA1AF0040F06D160
:100DF0004046FFF73DFB4846FFF778FA02E04046E1
:100E0000FFF736FB304603B0BDE8F08F50030020FB
:100E10000C03002008B501F071F900F0B9F8BDE845
:100E2000084000F01CB838B50446043000F01BFD43
:100E30000546204600F062FF284638BDF8B5044656
:100E40000E461746051D3A463146284600F0F6FC88
:100E500020B90121204600F021FFF4E7F8BD08B5D4
:100E6000002000F01BFA0120BDE8084000F016BA8F
:100E7000F8B50D4B1E68C6F307221D4622B9F4B221
:100E8000003418BF012400E00224FFF7E9FA2B68C0
:100E90009E42074602D12046FFF73EFC3846BDE899
:100EA000F840FFF7E5BA00BF200200202DE9F04F1F
:100EB0002C4B2D4A1B882D492D482E4EDFF8CCB0E7
:100EC0008BB00DF1280906F1800A29F8043D0DF0D8
:100ED000A7FFFFF781FA0546FFF796FA0446FFF7EA
:100EE0008FFA2A46009023464FF4007122480DF0F5
:100EF00097FF25EAE5754FF4007856F8044B14B3D4
:100F00002779E26A5BF82730606A0793904406927B
:100F1000FFF702FF069AB4F90610079B101A226821
:100F20000592626A04920390E26A029262790192E7
:100F3000082FD4BF4F4609F1010700970544A26A64
:100F40000E480DF06DFFB245D7D10D4B02958DE8DF
:100F500008010C4A0C4819460DF062FF0BB0BDE8C1
:100F6000F08F00BF7D0A0108AC0A0108B20A01082F
:100F7000B70A010854030020FF0A0108490B0108C1
:100F8000850B0108870B01088B0B0108800A0108FB
:100F900038B5FFF765FA1B4C0023E360054600F007
:100FA00037F84FF41443A360A268164B12F00C0FED
:100FB000FAD1154A40F20571116081221A601A684F
:100FC00042F480321A601A6812F4003F0D4AFAD0D7
:100FD0000E4B5360136843F0807313601168094B24
:100FE0008901FBD59A6842F002029A609A6802F081
:100FF0000C02082AFAD100F017F82846BDE838405C
:10100000FFF736BA00380240003C0240042A40078D
:10101000044B1A6842F001021A601A689207FCD564
:10102000704700BF00380240044B9A6812F00C0F62
:101030001EBF1A6822F001021A6070470038024091
:10104000034B044A00280CBF10461846704700BFE7
:1010500000BD010580DE800204281CD8DFE800F016
:1010600003080D1217000D4B1A6C1143196412E09E
:101070000A4A536C194351640DE0084A136B194333
:10108000116308E0054A536B1943516303E0034AB7
:10109000936B19439163BFF34F8F70470038024041
:1010A000042821D8DFE800F003090F151B000F4AC0
:1010B000136C23EA0101116470470C4A536C23EA54
:1010C000010151647047094A136B23EA010111635E
:1010D0007047064A536B23EA010151637047034A84
:1010E000936B23EA01019163704700BF003802400F
:1010F00038B514230C4A4343D4582568AA0608D5AA
:101100000A4B616803EBC002C9B253F83030506833
:1011100098472B0748BF6368054B1B681BB1BDE8A8
:101120003840FFF7C7BD38BD040C0108300B002064
:101130000003002001282DE9F04780460D461746A0
:1011400003D92B490320FFF74FFDDFF8B090294A60
:10115000142404FB009442F83070E66802EBC002ED
:1011600001215360304600F0BFF9304600F080FAAC
:101170003046617C00F054FA4E464FB1D4F80890E6
:101180000021484600F0B0F9217C484600F048FABA
:10119000142303FB08F806EB080999F812A0D9F804
:1011A00004105046FFF758FF56F808400023E3604C
:1011B000504623616361FFF743FFB0FBF5F080B257
:1011C000A06077B199F8133001215AB203F01F03E0
:1011D00001FA03F35209084941F8223042F22C0384
:1011E00001E042F20803E3600020BDE8F08700BFA1
:1011F000E5090108300B002000E100E0040C0108C3
:10120000012838B505D80E4C14230A4403FB0043CB
:1012100009E00C490320FFF7E7FC25682D06FCD503
:1012200011F8015B65608A4201D01C68F5E7142360
:101230005843034B1A5813685B06FCD538BD00BFF2
:10124000040C0108E50901080020FFF751BF012047
:10125000FFF74EBFF8B5104C04EB4014012167684E
:10126000384600F041F9A6680021304600F03CF90C
:10127000E5680121284600F037F9247D38462146EB
:1012800000F0CEF92146304600F0CAF92146284642
:10129000BDE8F84000F0C4B9380C010801282DE978
:1012A000F041044603D910490320FFF79DFC0F4B82
:1012B000DFF83C80002543F820506401FFF7CAFFA7
:1012C00008EB04031E7F9F6930463946FFF7C4FED2
:1012D00058F8043039461D603046DD615D60BDE878
:1012E000F041FFF7DDBE00BFE5090108400B00201B
:1012F000380C0108012870B50C4621D84A1C22D0B0
:1013000021F0FF0313F5807F11D114F0FF041AD1EF
:101310000E4B03EB40152E69731C14D0012130468F
:1013200000F0E2F8297D304600F07AF906E001216C
:10133000204600F0D9F8204600F09AF9002070BD50
:101340004FF0FF3070BD6FF0010070BD380C010828
:10135000042B2DE9F84304460E461546984603D95A
:1013600017490320FFF740FC1648DFF8609067013B
:10137000012100EB840000F091FC09EB07031C7FC6
:1013800099692046FFF768FE0F4B59F8071004EBE8
:1013900084041C4416F5807F14F8082045EAC20531
:1013A00045F004050D6015BF0B684B6843F44073AE
:1013B00043F0040314BF0B604B600020BDE8F883CA
:1013C000E5090108400B00202C0C0108380C01082D
:1013D0000B4A430110B50446D018D3588169007FE9
:1013E00000221A605A6822F004025A60FFF758FE81
:1013F000044800EB8400BDE8104000F07FBC00BF53
:10140000380C0108400B00202DE9F843089E099F85
:10141000884691461D4623B91EB931490320FFF77E
:10142000E3FB304B400118F5807F1C58236843F0E4
:101430004003236005D0B8F1FF3F02D0404600F0E2
:1014400020F9A6B92F44AF4206D0A3689E07FCD569
:1014500015F8013B2373F6E7A3689807FCD5A3684A
:101460001906FCD4A368DA0720D5E368FAE70DB1C2
:10147000002319E030463744B84217D0A3689B07D1
:10148000FCD52573A368DE07FCD5237B00F8013B60
:10149000F2E7A2689007FCD5EA5C2273A268D10744
:1014A000FCD5227BF2540133BB42F2D1A3689A07E8
:1014B000FCD5A3681B06FCD4B9F1000F0ED1B8F11E
:1014C000FF3F0BD0236818F5807F23F04003236093
:1014D00004D04046BDE8F84300F0CAB8BDE8F88340
:1014E000E5090108380C0108F8B50D460126C0F3DE
:1014F000832120F00F0400F00F0706FA01F102200B
:10150000FFF7AAFD07FA06F00323216883406FEA7C
:10151000030C01EA0C012160216805F0030E0EFAAC
:1015200000FE4EEA01012160E2680CEA0202E2607C
:10153000E168C5F3810282400A43E2606268BE400E
:1015400022EA060666606268C5F30015BD401543D1
:101550006560A2681343A3600020F8BD2DE9F04147
:1015600000F00F0415462B4A42F8343002EBC40257
:10157000069B536006468846C0F383274FF480419C
:101580000120FFF769FD41463046FFF7ADFF042C0F
:10159000214B03DCA11D01228A4003E0092C03DC5E
:1015A0004FF400021A6002E04FF480725A601B4B45
:1015B0000120996800FA04F2D243114099609968B9
:1015C00005EA000E0EFA04FE4EEA01019960D968A0
:1015D0000A40DA60C540DA68A54004F00C0404F162
:1015E000804404F59C341543DD6006F00302A568D1
:1015F00092000F21914025EA0101A160A168974066
:10160000B0400F43A76058611A681043186000206B
:10161000BDE8F081480B002000E100E0003C014003
:1016200020F00F0300F00F02F0B51E6857000325ED
:10163000BD4026EA05051D601D680224072A04FA3C
:1016400007F444EA050494BF002201221C6003EB66
:10165000820300F007001C6A80000F22824024EA07
:1016600002021A621A6A814041EA02001862F0BD61
:1016700020F00F02012300F00F0003FA00F0906148
:10168000704720F00F0200F00F001030012303FA22
:1016900000F0906170470000104B2DE9F0415E6949
:1016A0001A680F4F164000244FF001081D4608FA33
:1016B00004F31E4206D06B6107EBC40357F83420D5
:1016C000586890470134102CF1D1064B1B681BB1B0
:1016D000BDE8F041FFF7EEBABDE8F081003C014003
:1016E000480B0020000300202DE9F843124ADFF8E0
:1016F000508003010746D5582E69EB6800241E4030
:1017000008EBC0090223A3401E4209D0EA68D9F8B9
:10171000040022EA0303EB60214658F8373098476B
:101720000134042CEED1054B1B681BB1BDE8F84316
:10173000FFF7C0BABDE8F883780C01080003002069
:10174000C80B0020032910B516D80D4B00011C183A
:101750001B586068024001F10C0003EB80004260FE
:101760001869022202FA01F120EA01021A61DA681C
:101770001143D960002010BD4FF0FF3010BD00BFF5
:10178000780C01080001024B1B58586A704700BFD3
:10179000780C0108034B00011A58136843F0010349
:1017A00013607047780C010801282DE9F8430546BD
:1017B000884630D81A4E1B490401371941F83020A9
:1017C00097F80C9001EBC00148464B60B968FFF7F1
:1017D00043FC36597B680024346048467460F362E9
:1017E000FFF72EFC104B7A7B13F809305843B0FBFF
:1017F000F8F3013BB36251B2012302F01F0273619F
:1018000049099340094A284642F82130FFF7C2FFB0
:101810002046BDE8F8834FF0FF30BDE8F88300BFF5
:10182000780C0108C80B0020980C010800E100E0CA
:101830000020FFF759BF0120FFF756BF70B51346D0
:101840007BB18568C468A5420BD084680668651CB6
:1018500085604568013D2C40013B345D01F8014B3A
:10186000EEE7D01A70BDC368426830B584681B1BB0
:10187000934208D0C3680468013A5D1C1340C560F8
:10188000E154002030BD4FF0FF3030BD2DE9F04174
:101890000821AEB0534800F01DFC53480DF04AFB40
:1018A000102200210AA80DF0B3F9102200210EA881
:1018B0000DF0AEF907A803F01FFCBA238DF828300D
:1018C000AD238DF82930A5238DF82A3055238DF8C6
:1018D0002B3008230093002208AB0221BDF91C0025
:1018E00003F0F6F90028A4BF9DF820308DF83630BB
:1018F0004FF08002A4BF9DF821308DF837300AA93F
:101900000EA80DF087F8002340220AA9BDF91C009B
:1019100001F08EFD9DF83640172C58D19DF83730D8
:10192000022B03D18DF8464036232FE0322B28D1ED
:101930003623002610258DF847304FF0FF372B4B0C
:10194000BDF91C10019304972B460396029500964F
:101950000EAA27488DF8464000F03AFD02238DF884
:101960004730BDF91C10234B8DF846400497039671
:101970000295019300962B460EAA1D4800F028FD03
:1019800028E0362B23D18DF8464002231A4F8DF8DC
:101990004730002610254FF0FF38BDF91C10CDF858
:1019A00010802B46039602958DE8C0000EAA1048C1
:1019B00000F00EFD32238DF846408DF84730BDF91A
:1019C0001C10CDF81080039602950197D2E70B48C2
:1019D0000DF0B0FA0A480DF0ADFA80220EA90948C0
:1019E00007F082FFD80B0020B40C0108440200204D
:1019F000A81000202402002034020020DB0C010883
:101A0000E50C01089C0C01082DE9F04F012889B074
:101A100006460D4602DC0968664882E06649686849
:101A20000DF082FB0446002871D1042E02DC2968E7
:101A3000624876E0052E0AD068690CF041FD062E5A
:101A4000814606D0A8690CF03BFD074602E04FF046
:101A500001095B4FAB68019301992B69EE68029312
:101A600004A807F0EFFD08B9564898E030460CF09E
:101A700027FD1FFA80F88246B8F1000F01D000263A
:101A80000DE051488BE01FFA8AF3019A03994F4801
:101A90000DF0C6F9002138460AF096FE01364E4593
:101AA00000F0848002980DF00BFD0023024602999D
:101AB000184603F069FD054608B945486FE0C3685C
:101AC00003934246414607F0F5FA834608B9414878
:101AD00018E004AA002101F00BFB054638B93E4886
:101AE0000DF028FA2946584603F040FE5EE0034612
:101AF00040F202223949042003F096F88346002878
:101B0000C1D137480DF016FA59462846ECE7354959
:101B100068680DF009FB002844D1022E05D1296820
:101B200031480DF07DF9012440E03049A8680DF0FE
:101B3000FBFA0446F8B9032E02D129682C48F0E7D5
:101B40002C4EB6F90C3013B171682B4810E0E868E0
:101B50000CF0B6FC85B20DB9284820E0284B756022
:101B60001B88B3813146042003F012FB2548294627
:101B70000DF056F91AE02449A8680DF0D5FA04468C
:101B800080B91C4DB5F90C301BB920480DF048F94F
:101B90000CE00420294603F01DFB1D48AC810DF02C
:101BA000C9F903E01B480DF0C5F90024204609B02F
:101BB000BDE8F08F320D0108CC0B01084B0D010878
:101BC00040420F00880D0108B30D0108750E010891
:101BD000DB0D0108070E01082C0E01080000FFFFB5
:101BE000520E0108880F01089A0E0108B90E01086B
:101BF000BF0E010854020020DD0E0108080F010885
:101C0000B8310020260F01084F0F0108540F0108BA
:101C1000730F01088F0F010808B5002007F00AFEB6
:101C2000FEF7D6FE03F094FC03F076FE05F000FB11
:101C300001F034F807F050FA00F006F801F07EFDEC
:101C4000BDE8084003F086BE13B50E4C0E490F48A0
:101C50000AF026FE0D49204603F08EF9002806DA28
:101C60000B48002102B0BDE810400DF0D9B8009437
:101C7000084B094802224FF4806103F013FA02B0C6
:101C800010BD00BF70100020A80F01081810002020
:101C9000C00F0108FA0F0108180C002070B50546A6
:101CA0000C46FEF7DDFB2B6806462BB94FF0FF33E1
:101CB0002B60FEF7DDFB18E0CCB10F4B1C68022156
:101CC0002046FEF7D3FA2B68013305D104F108034F
:101CD0002B600023A36003E021462846FFF704F8A9
:101CE0003046FEF7C5FBFEF797FB012070BDFEF7FF
:101CF000BFFB204670BD00BF0803002070B504463E
:101D0000FEF7AEFB256806461DB16B1C05D100230E
:101D10002360BDE87040FEF7ABBB28460A2150F8AF
:101D200008392360FEF7A2FA236813B94FF0FF3396
:101D3000236015F8034C3046FEF79AFB2046BDE8B9
:101D40007040FEF7D3BA0000F8B505460E46FEF720
:101D500087FB364B364A1B881BB2074652F82320B6
:101D6000D2F820E0BEF1000F1AD054699369A34263
:101D700016D9631C5361D3691C4046B9136933B942
:101D8000631C04D13846FEF773FB2046F8BD002CD7
:101D90000ADB0EEBC40393E8030085E8030004E0CC
:101DA0004FF0FF34002EE9D0D560166976B3336862
:101DB0001361002C0CDB95695169D369691A8B4258
:101DC000A9BF691C4FF0FF351D4091610EEBC505A1
:101DD000736893E8030085E8030016F8043C052BBC
:101DE00009D0002373600A21A6F10800FEF73EFA2D
:101DF00016F8034C00E00F243846FEF739FB0E2C92
:101E000002D82046FEF772FA0120F8BD002C09DA4C
:101E100010460321FEF72AFA3846FEF729FBFEF7A3
:101E2000FBFAF1E73846FEF723FBEDE70403002059
:101E30005003002010B583694469C2691C1BA2428B
:101E400001DA002010BD5C1C13408461F9D4026AE1
:101E500003C902EBC30383E80300012010BD0000A7
:101E60002DE9F8431E46264B53F82150254B1B887D
:101E70000380074691462DB93046FEF7F9FA4FF038
:101E8000FF3439E02B79032B28D01F4B014628461D
:101E9000D3F80080FFF7CEFF044638B13046FEF796
:101EA000E7FA98F80430052B25D122E0B9F1000FAC
:101EB00003D13046FEF7DCFA1EE098F80430C8F88B
:101EC0000C70052B0CBF052104214046FEF7CEF90E
:101ED000414605F11000FEF707FF07E003C8EB6875
:101EE00083E803000A212846FEF7C0F93046FEF7D2
:101EF000BFFAFEF791FA01242046BDE8F88300BF3F
:101F000050030020040300200803002038B50446D5
:101F1000FEF7A6FA074B1B882380074B2146054690
:101F20001868FFF787FF04462846FEF7A1FA204607
:101F300038BD00BF040300200803002008B50F4B84
:101F400053F82130B3B1212202801A79032A0BD130
:101F500003C8DA6882E8030018460A21FEF786F90A
:101F6000074B0120186008BD01461846BDE808402F
:101F7000FFF760BF4FF0FF3008BD00BF50030020E7
:101F80000003002070B504460D46FEF774FA28B130
:101F900029462046BDE87040FFF7D0BF094B1B889B
:101FA0001BB29D4204D12046BDE87040FFF7AEBF92
:101FB000FEF756FA2946034601222046BDE8704046
:101FC000FFF74EBF0403002070B504460D46FEF730
:101FD00052FA064628B129462046BDE87040FFF770
:101FE000ADBF0A4B1B881BB29D4204D12046BDE801
:101FF0007040FFF78BBFFEF733FA3246034629469F
:102000002046BDE87040FFF72BBF00BF040300204F
:102010002DE9F041124F3B881BB2934206460C4615
:10202000154603D10F490320FEF7DEFDFEF718FA2F
:102030003A880D4B12B2804653F82270052138467B
:10204000FEF714F996E80300FC60434684E80300B9
:10205000012229462046BDE8F041FFF701BF00BF3D
:1020600004030020E50901085003002070B5044670
:102070000D46FEF7F5F9B4F90020114B53F8224054
:1020800006461CB90F490320FEF7AEFD2379052B48
:1020900004D0FEF7EDF94FF0FF3070BD95E8030076
:1020A000E36883E803000A212046FEF7DFF864793D
:1020B0003046FEF7DDF92046FEF718F9012070BD25
:1020C00050030020E50901080021FFF73DBE012172
:1020D000FFF73ABE08B5074B4A1E1B68114018624D
:1020E00003D005490320FEF77FFD59619961DA614C
:1020F00008BD00BF08030020E50901080F4BD3F815
:10210000882042F47002C3F888200D4A9A60102299
:1021100083F822200021DA7701F1604000F5614068
:102120000131522980F80023F6D11A6942F01002D9
:102130001A615A6942F400725A61704700ED00E07A
:10214000000000080121FFF7A9BD10B50446406951
:1021500008B10AF071FAE06908B10AF06DFA0020DE
:102160000022002360612061E061A0612080C4E959
:10217000022310BDFEF73EBC2DE9F04F89B08A4620
:1021800015469B460446FFF7F5FFCDE90401EB0039
:102190000393079355445346AB4205D013F8012BE4
:1021A000002AF9D0002300E00123002702936FF0FA
:1021B00075030193B846B9463E46A268974270D26D
:1021C00022687D0102EB050EDEE90201002908BF4D
:1021D000B0F1FF3F23D0DDE90423994208BF9042CC
:1021E0001DD200220023CEE9022322682A44166170
:1021F00022682A4496612268565322682A4450690C
:1022000020B10AF019FA22682A44566122682A4449
:10221000D06920B10AF010FA22682A44D661039BE3
:1022200098453CD222682A445069002837D007AA32
:1022300051460AF037FA38B923681D44129BCBF88F
:1022400000500120186034E0029B13B102282DD108
:10225000F2E7012814D122681544296911F07F4F53
:102260001BD0079AB2EB116F17D3B8F1000F01D052
:10227000904512D20023CBF80050904601930AE01B
:1022800002280AD1B8F1000F07D12268CDF80480E6
:102290001544CBF800504FF00109039B0793013719
:1022A0008BE7129B0198C3F8009002E00128F4D15B
:1022B000D1E709B0BDE8F08F38B505460C46FFF709
:1022C00059FF4FF47A736B43C01841F10001C4E920
:1022D000000138BD2DE9F04788B0972990461BBF13
:1022E000109A0792424605AA8A461CBFCDF8148070
:1022F0008DF81830ADF806100292DF0000F11205DB
:1023000000F1200600F11C046FF0010935F9023FCD
:10231000DBB1BAF1970F03D000976A46414607E058
:10232000D8F8183019684B78DB0000936A46023100
:1023300030680AF0B7F9023007D0B5F9002003A9D8
:1023400001A8FFF765FE4FF00009A54206F104065B
:10235000DCD1484608B0BDE8F087000030B587B052
:1023600006AA102302AD294642F8143D0AF07CF972
:10237000A842014620D1019B102B08D128220F48EA
:1023800007F0AAF801460E480CF04AFD14E00024BC
:10239000019BA34204D3295D0A480CF041FD02E0F1
:1023A00009480CF03DFD0134102CF1D107240748F9
:1023B0000CF036FD013CFAD107B030BD8010002092
:1023C000041001080A100108D01E0108D11E0108DE
:1023D0002DE9F04F00F10C0787B0044638469A46C5
:1023E0008B469046149EFFF7ADFE01230493B8F18F
:1023F000000F01D0119B2BB93846FFF77FFC6FF01F
:102400000D006AE004AB0093524605AB41462046FE
:10241000FFF7B2FE012802D04FF000091CE012992C
:102420001198059C0AF0A6F8054610B96FF00B0448
:102430004FE0E0690AF000F9139BE561721CA361AB
:1024400002D004F1080139E04FF0FF320023C4E963
:1024500002233DE009F10109A2689145E6D2226814
:102460004FEA49152A44D2E9020150EA0103F1D1A9
:102470005146404603920AF07DF8039A5061226863
:102480002A44516971B1109B136122681299119805
:102490002A4403920AF06EF8039A139BD0612268D3
:1024A0002A44936122682A44D1690029D2D0A2F833
:1024B00000B0731C216805D0294408313046FFF76D
:1024C000FBFE05E00D444FF0FF320023C5E9022377
:1024D00000243846FFF712FC204607B0BDE8F08F15
:1024E0002DE9F04300F10C0585B0044628461F464F
:1024F000884691460E9EFFF725FE01230293B8F110
:10250000000F00D02FB92846FFF7F8FB6FF00D0041
:102510002CE002AB00934A4603AB41462046FFF74E
:102520002BFE012802D06FF00B041BE038460C99FB
:10253000039C0AF01FF807460028F4D0E0690AF06F
:102540007BF80D9BA361731CE76105D004F10801C2
:102550003046FFF7B1FE04E04FF0FF320023C4E93C
:10256000022300242846FFF7C9FB204605B0BDE83A
:10257000F083F0B500F10C0485B0054620460E4608
:102580001746FFF7DFFD0123029302AB00933A46A3
:1025900003AB31462846FFF7EFFD012802D103982F
:1025A000FFF7D3FD2046FFF7A9FB05B0F0BDF8B556
:1025B00000F10C06054630460F46FFF7C3FD002428
:1025C000AB689C420AD22868630117B1C25EBA4266
:1025D00002D11844FFF7B9FD0134F1E73046BDE8F8
:1025E000F840FFF78BBB2DE9F04F00F10C0485B0EC
:1025F000054620469B46894692460F9EFFF7A2FD60
:1026000001230293B9F1000F04D0BBF1000F01D0F8
:102610000E9B2BB92046FFF771FB6FF0150049E0C8
:1026200016B1BAF1000F05D12046FFF767FB6FF036
:102630000D003FE002AF009703AB109A31462846E9
:10264000FFF79AFD0128804615D9119B0093324669
:10265000109B99212846FFF73DFE48B901230293BC
:10266000009703AB109A31462846FFF785FD804658
:10267000B8F1010F0CD8039B5A465146D86909F0AE
:10268000F3FF58B92046FFF739FB6FF0680011E0FF
:102690002046FFF733FB6FF075000BE0039BB3F9A7
:1026A0000020A9F800200E9A9B6913602046FFF7CE
:1026B00025FB002005B0BDE8F08FF8B506460025E3
:1026C00046F80C5F04463046FFF73CFD04F1120269
:1026D00004F11C0304F1300122F8025F43F8045FA7
:1026E0008B424FF00007F7D123792761022BA268B4
:1026F0000BD123685201394618680CF089FA236817
:102700009A685868D200394602E02068520139467A
:102710000CF07EFA0AF028F83046BDE8F840FFF7E2
:10272000EDBA00002DE9F04F044600F10C0585B02C
:102730002846FFF707FDFFF71DFD2379012B804693
:1027400089466AD1674A684B684969488DE80C0038
:10275000684B0CF065FB4FF0000BA3689B456BD2F8
:1027600021684FEA4B1A5144D1E90223134351D057
:102770004869FFF7F3FD23685F48534419690CF07B
:102780004FFB23685344196911F07F4F04D0090EA1
:102790005A480CF045FB02E059480CF041FB236815
:1027A0005344D869FFF7DAFD2368534853449969C5
:1027B0000CF036FB23685344D3E90267002F08BFAF
:1027C000B6F1FF3F1CD0B6EB080667EB0907002EF9
:1027D00077F1000301DA4B4913E0304639464A4AA3
:1027E00000230BF0E1FC002303923046464A3946B1
:1027F0000BF0DAFC039A014644480CF011FB03E0AD
:10280000434944480CF00CFB2368434833F90A1051
:102810000CF006FB0BF1010B9FE7022B0CD1324BA6
:1028200000933E4A3E4B3F493F480CF0F9FA4FF0C7
:10283000000BA3689B4505D3284605B0BDE8F04FC3
:10284000FFF75CBA236819684FEA4B1A5144D1E983
:102850000223134343D08B691868FFF77FFD236879
:102860001B6853445B691868FFF778FD23682F489D
:102870001B68534419690CF0D3FA23681B6853444E
:10288000D3E90267002F08BFB6F1FF3F1CD0B6EBBB
:10289000080667EB0907002E77F1000301DA1949F2
:1028A00013E030463946184A00230BF07DFC002324
:1028B00003923046144A39460BF076FC039A0146DF
:1028C00012480CF0ADFA03E0114912480CF0A8FAD6
:1028D000236811481B6833F90A100CF0A1FA0BF1B8
:1028E000010BA6E74C11010807110108621101084C
:1028F000DE100108D51001080F1101081911010897
:10290000221101082A11010840420F003911010863
:1029100043110108321101082E100108521101085B
:10292000491101085F1101086E1101089011010899
:10293000034600201BB1DA685B681044FAE7704771
:1029400010B50822094904460CF032F848B1237842
:10295000FF2B08D1607800F00F00831E58425841C9
:1029600010BD012010BD002010BD00BF5E13010886
:10297000002102F0FBBE38B5CBB20021144602465E
:10298000084602F0CFFB054618B92046FFF7F0FFD6
:102990000FE094F9103001330AD1A36882681B79E3
:1029A00003F03F0321462046137102F09FFC0446CA
:1029B0006C60284638BD00002DE9F0478C6807465A
:1029C000104688461546FFF7B3FFA37940BAFF2BA0
:1029D000A0800AD12B7C023BDBB2022B03D8214A18
:1029E000D35CFF2B00D13B23A371E37943B90FB92B
:1029F000402304E0384600F0FDFC90F8CA31E37152
:102A000004F108061022184930460BF0D1FF824627
:102A1000D0B904F118091549102248460BF0C8FF37
:102A2000014630B9102230460CF0F2F80123E3756C
:102A30000AE049465246384600F0B6FD014618B154
:102A4000102230460BF0E6FF4146284602F008FC13
:102A5000002804DA831C08BF0020BDE8F0870020AE
:102A6000BDE8F0879F110108AE130108BE130108ED
:102A70008B6870B558800C46054600F0BBFC0146DB
:102A800018B919490320FEF7AFF866683046FFF71A
:102A90004FFFB1F8C831984204D92046BDE87040D4
:102AA000FFF766BFD1F81C320133C1F81C32304643
:102AB000FFF73EFFD1F824321844B1F8C631C1F80F
:102AC0002402DB0708D5234640F2022207490120F1
:102AD00002F0AAF830B9E0E72146284602F0DDF816
:102AE0000028DADD70BD00BFE50901080000FFFF26
:102AF0002DE9F04F85B090F91030013300AF044656
:102B000089460AD18368B3F9026002F03DFE0028CD
:102B10006AD043680446984601E080460026404655
:102B200002F032FE054600285ED04445836818BF97
:102B300060601A461B7ED0F8048008BF0446FF2B55
:102B40002BD186B907F1080002F0D6FA00284BD045
:102B5000002122460846B7F90860FFF70CFF04463B
:102B6000002800F09380B9F1000F06D042462946B4
:102B70003046FFF721FF002836DBA268137943F0C7
:102B800040031371304600F08DFE4368013343600B
:102B900021463046FFF76CFF78E0134618331022C9
:102BA0003C4918469B460BF003FF40B15946002EA6
:102BB00039D1381D00F09CFC0646002838D0B9F108
:102BC000000F06D0424629463046FFF7F5FE0028A2
:102BD0000ADB2846FFF7ACFE002102460223084626
:102BE00002F0D2FC064608B9204619E083689846F0
:102BF000EA68A96840460BF00DFFEB686D68424635
:102C00001A449046002DF3D12046FFF7B1FE224B27
:102C10003146B3F9000002F04DF8002836DC3046AA
:102C2000FFF7A6FE32E0304600F03AFC0028C6D19D
:102C300007F11001082301F80D3D32465B4607F10C
:102C4000080005F09DFDEA46064640B1B9F1000FC7
:102C500009D042462946FFF7AFFE002803DA204696
:102C6000FFF786FE11E02246F97807F10800FFF72A
:102C700082FE044648B1304600F014FE036801337A
:102C8000036021463046FFF7F3FED5461437BD46B4
:102C9000BDE8F08FBE130108DC1000201FB50F4CFB
:102CA000B4F9003063B90E4A01930E4B02920093BF
:102CB000042208234FF480610B48FEF735F820808A
:102CC0000A480B4B03600123037114238360FFF751
:102CD000F4FCB4F9000004B010BD00BFDC1000200B
:102CE0009A110108952F0008DE100020A81000207E
:102CF000E0140020292B2DE9F84381460F461446A5
:102D00001D4606D03A2B06D0112B0CBF04230023FE
:102D100002E0022300E00323292D3B7401D03A2D69
:102D200003D1A74259D1012605E0A74202D063682A
:102D30009F4252D100267B6893F91000022805D0EB
:102D400016B30121204602F0FFFC1DE0294602F0E7
:102D50006BFA18B986F0010836B101E04FF00008AF
:102D60000121204602F0F0FC234640F201221E49D8
:102D700097F9100001F058FF10B92046FFF7F8FD51
:102D8000B8F1000FDCD00AE0234640F201222946C8
:102D9000022001F049FF10B92046FFF7E9FD06B314
:102DA000292D07D03A2D18D121464846BDE8F843D1
:102DB0000AF03ABD00232374616839B191F91030EB
:102DC000022B03D1204602F091FAF5E70223237487
:102DD0002046BDE8F84300F00BB804490320FDF796
:102DE00003FFBDE8F88300BF0000FFFFE50901080D
:102DF0002DE9F047044618B964490320FDF7F4FEB5
:102E00004FF0FF3102F03DFA0546A0B18368B3F9F7
:102E10000260002EF0D0304600F044FD43690133DB
:102E2000014643612046FFF783FDEA688B699B1AE0
:102E30001844886100E006462746254695F910307B
:102E4000022B08D1EB68282B05D1AB681B7803F067
:102E5000F003602B08D0D5F804802F46B8F1000F9E
:102E60006ED04546EAE73C46D5F80880E368B8F8F6
:102E7000041049BA89B2994203D2204602F00CFCF0
:102E80000FE022460023D068034492F91000022884
:102E900003D1283B994204D95DE05268002AF2D15F
:102EA000F7E708F118091022394948460BF080FD70
:102EB000002855D04846FFF743FD494600B136B9D2
:102EC000002000F015FB002E08BF064602E0304649
:102ED00000F0E6FAB0FA80F04009002840D008F18E
:102EE0000800FFF72DFDB0BB4846FFF729FD90BB5A
:102EF00098F80730013BDBB288F807305BB328460F
:102F000002F042FC38B34FF0FF31204602F0B9F92D
:102F1000014610B1204602F0E9F921460025084695
:102F200002F032FC18B92846FFF722FD13E0416891
:102F3000456005460029F2D1BDE8F047FFF7D8BD4E
:102F4000A3681B7803F0F003602B04D1204602F045
:102F50001BFC074668B92046BDE8F047FFF708BDEF
:102F600098F80630224639463046BDE8F047FFF76C
:102F7000C1BE0222282102F021FB87F810800546FD
:102F800000287FF470AF3846E6E700BFE509010886
:102F9000BE13010810B5102298B00DEB02000021FD
:102FA0000BF036FE504B0593504B08211B88ADF8B3
:102FB0001C3008A8FFF78EF804A9022002F0E8F8F8
:102FC00040F20523ADF80A3000246846FFF77FF889
:102FD000BDF802306FF400721344222BF5D801A221
:102FE00052F823F07130000879300008833000086F
:102FF00083300008CB2F0008CB2F0008CB2F000810
:10300000CB2F0008CB2F0008CB2F0008CB2F0008B8
:10301000CB2F0008CB2F0008CB2F0008CB2F0008A8
:1030200093300008CB2F00089F300008CB2F0008FA
:10303000CB2F0008D7300008CB2F0008A73000089E
:10304000CB2F0008CB2F0008CB2F0008CB2F000878
:10305000CB2F0008CB2F0008CB2F0008CB2F000868
:10306000AF300008B7300008BF300008CF3000088C
:103070000198FFF7BDFEA8E701210198FFF738FD91
:10308000A3E76FF0850302A968460393FEF7EEFFFE
:103090009BE7019A537E23F00803537695E7019846
:1030A00000F072FF91E7019800F0FCFF8DE70198B6
:1030B00005F0E0FA89E7019805F032FB85E7019B0E
:1030C000587C00F00F0004F01FF904747DE70198AC
:1030D00005F08CFD79E7019A00231946B2F91A0030
:1030E00001F040FB71E700BF0000FFFF0403002078
:1030F000F8B50F46164602232822002102F044FAB2
:10310000054600B38468102204F10800394617B15F
:103110000BF080FC01E00BF07BFD04F118001022A5
:10312000314616B10BF076FC04E00BF071FD012383
:1031300084F82730602200232270FF226370A3707E
:10314000E370A271E3712846F8BD0121FEF7A6BD28
:103150002DE9F84300F5E075074628468846FFF755
:10316000F4FF00244FF0380909FB0476414630464D
:1031700006F04BF938B11022002130460BF048FD23
:103180000023337402E00134082CEDD12846BDE859
:10319000F843FEF7B3BD000008B5102203490BF059
:1031A00007FCB0FA80F0400908BD00BFAE1301086B
:1031B00010B50822094904460BF0FAFB48B1237800
:1031C000FF2B08D1607800F00F00831E5842584151
:1031D00010BD012010BD002010BD00BF5E1301080E
:1031E0002DE9FF4700260546884692469946344613
:1031F000AF194146384606F008F900287FD1384615
:10320000FFF7CAFF10B1002C08BF3C463836B6F5B0
:10321000E07FEDD12746002C71D010224146204698
:103220000BF0F8FB237884F811A0FF2B84F81090A2
:1032300016D0B5F8C631DA0712D501F0E1F88146AB
:1032400070B105F5E0763046FEF758FDB5F9C401DA
:103250004B464A46214601F083F93046FFF775FF99
:1032600098F80030FF2B04D1237C43F00103237432
:1032700041E04046FFF79CFF8146C8B9B5F8C6213A
:1032800002F00602062A17D105F5E0763046FEF771
:1032900035FDB5F8C631DB0706D54B464A464946EB
:1032A000B5F9C40101F05EFA3046FFF74EFF03E0C6
:1032B000237C63F07F032374B5F8C63103F0030366
:1032C000012B18D040F2FF220023CDE900234FF05C
:1032D00080730293FF238DF80C3098F80D308DF831
:1032E0000D30B8F80E30ADF80E308022002369465C
:1032F0002846FFF775FF40F2112363866463384662
:1033000004B0BDE8F08703885BBA23F03F031B04D9
:103310001B0C4FF6C062934209D00378FF2B08D1F3
:10332000407800F00F00052818BF0E2070470520D8
:1033300070470E2070472DE9F047002580469146E2
:103340001F460C462E464FF0010A3FB13A780AFA62
:1033500005F31A421AD0237CDB0717D42046FFF767
:103360001BFF98B94946204606F064F837B999F82A
:103370000030FF2B02D0637C834207D8B04205D9CE
:10338000B8F1000F01D0C8F8004006460135082DFD
:1033900004F13804D9D13046BDE8F08770B5134C3C
:1033A000B4F9C451A84206461ED0EDB904F5E07048
:1033B000FFF7CBFE4FF4A063A4F8C831402384F894
:1033C000CA31A4F8C4612B46A4F8C651802208492A
:1033D0002046FFF705FF04F5E070FEF78FFC20465E
:1033E000BDE8704000F06CBE70BD00BF60170020EB
:1033F0007E130108034BB3F9C42182420CBF184667
:103400000020704760170020B0F8C631DA0707D5F2
:1034100011B143F0020301E023F00203A0F8C6312A
:103420007047B0F8C631DB0701D505F09FBB704788
:103430002DE9F0410D4617469846FFF7DBFF04469D
:1034400010B90020BDE8F0810029FAD00846FFF746
:10345000A3FE0028F5D1802FF3DC04F5E07630469A
:10346000FFF773FE43463A4629462046FFF7B8FE6B
:1034700004463046FEF742FC2046BDE8F0810000DD
:1034800010B520B90548B0F9C43133B101E0FFF7F8
:10349000B1FFBDE81040FFF75BBE10BD6017002014
:1034A0002DE9F8438946FFF7A5FF0446E8B100F58A
:1034B000E0763046FFF749FE002504EB0508494653
:1034C000404605F0A2FF074628B13046FEF716FC3D
:1034D0004046BDE8F8833835B5F5E07FEDD130469C
:1034E000FEF70CFC3846BDE8F883BDE8F883000021
:1034F00038B5084C0546B4F9C4011DB9FFF7D0FF33
:1035000020B938BDFFF7CCFF286008B1B4F9C40179
:1035100038BD00BF601700202DE9F34102AD002641
:103520000E4C45F8046D8846074604F5E070FFF739
:103530000CFE3346424621462846FFF7FCFE20B1EA
:10354000019B3B60B4F9C44100E004460448FEF727
:10355000D5FB204602B0BDE8F08100BF6017002017
:10356000201900202DE9F34102AC0027884644F8D9
:10357000047DFFF73FFF00F5E07506462846FFF79C
:10358000E4FD20463B4642463146FFF7D4FE044662
:1035900028461CB1FEF7B2FB019802E0FEF7AEFB35
:1035A000204602B0BDE8F0812DE9F04F87B00F460C
:1035B0001546FFF71FFF00F5E0738046184601939C
:1035C000FFF7C3FD0122002102A80BF021FB4646B4
:1035D000C3464FF0FF3A00244FF001099BF800204A
:1035E000FF2A12D05846FFF7D7FD70B945B99DF8AC
:1035F000081009FA04F20A438DF80820A24604E0F4
:103600005846FFF7D5FD0028F1D10134082C0BF105
:10361000380BE3D1BAF1FF3F00F0878004AD2246BA
:10362000002128460BF0F4FA3B78FF2B04D197F8E1
:10363000019009F00F0309E03846FFF7B9FD20B902
:103640003846FFF760FE009001E0022300934FF040
:1036500000094C469DF80810012303FA04F21142B8
:1036600032D039463046B34605F0CFFE002855D15A
:103670003046FFF79DFD18B93046FFF744FE00E0E5
:103680000220009B834208D12A5D0432D2B22A551F
:103690004A4588BF4FF004090AE009D92A5D023281
:1036A000D2B24A4513462A5538BF4B465FFA83F9D2
:1036B000B2694AB12A5D0132D2B24A4513462A554F
:1036C00038BF4B465FFA83F90134082C06F13806FF
:1036D000C0D10122002102A80BF09AFA00209DF827
:1036E0000820014601246E5C4E4504BF04FA01F037
:1036F000024301F1010104BFD2B201200829F2D135
:1037000008B18DF8082006A8002340F80C3D3A4681
:1037100002AB4146FFF70FFEDDF80CB0BBF1000F26
:1037200005D1382202FB0A8B01E04FF0000B019813
:10373000FEF7E4FA584607B0BDE8F08F2DE9F04FE8
:103740008DB005A801F0D8FC0026544F03900DF170
:103750001205B146039B9E4200F09D8035F9020F91
:10376000FFF748FE0446002800F0918000F5E07A5B
:103770005046FFF7EAFC0123B5F900000093002250
:103780000DF1130317218DF8139001F0A1FA863083
:103790002CD09DF91330012B28D108230DF13008CE
:1037A000ADF818304FF6FF7328F8103DB7F8C63162
:1037B000B5F9000043F003034FF0020BA7F8C63140
:1037C000002206AB0521CDF800B001F0A7FAB5F94B
:1037D0000000CDF800B011214346002201F078FA34
:1037E000BDF82010B5F9000005F04CFB4FF00808BB
:1037F000B5F90000CDF8008006AB0022414601F08B
:1038000067FA00280FDB424606A90AA80BF002F966
:103810004246234908A80BF0FDF80023402208A9DE
:103820002046FFF7DDFC0223B5F9000000930022DB
:103830000DF11603112101F04BFA002806DBBDF84B
:103840001630B3F5A06F28BFA4F8C83100231A467C
:103850002421B5F90000CDF8009001F039FAB4F850
:10386000C6310028CCBF43F0800323F08003A4F8C6
:10387000C6315046FEF742FA01212046FFF7C4FD4B
:10388000B4F8C631DB0702D5204604F0BBFE013692
:1038900007F50C775EE70DB0BDE8F08F60170020EC
:1038A0005E13010808B5FFF7A5FD00F5057008BD1A
:1038B0002DE9F3410746884616461C460AF04CF9A6
:1038C000054640B9032300933246A3B24146384629
:1038D0000AF0D4F820E0437E03F00703012B01D166
:1038E00003210DE0027EA3B29A4200F110070CD032
:1038F00031462C76224638460BF08CF803212846B8
:1039000002B0BDE8F04100F08FBE22463946304695
:103910000BF04EF80028EBD102B0BDE8F0810000BA
:103920002DE9F04F1D46D37991B0FF2B80460691CB
:1039300016461A9F40F0B4806B78002B40F0B080A0
:10394000172F40F2AD802B7AFF2B00F0A98002F1F7
:1039500008095549102248460BF02AF870B105F1C4
:1039600008014046FFF79CFD0590002800F0988074
:103970000023183F1C4619469A461BE00D224B496E
:1039800006F118000BF014F8002800F08980E6E733
:103990000AF1180205EB020BAA5C012A0DD0212ABC
:1039A00008BF5C469BF801200AEBC20A1FFA8AFA9C
:1039B000A7EBC207002FEBDC0BE008AB2A780698D8
:1039C000009331465B4601F00DF8031E68DB594653
:1039D000E8E7404607930691FFF70CFD0699079B21
:1039E00018B933490320FDF7FFF808AA002942D08F
:1039F000002C40D0B0F8C61101F0030103293AD1E0
:103A00002978029301924B460A460094314640467B
:103A100004F0A6FF002304F108020F21074604F07A
:103A200085FF054617B91022494620E0237A83F026
:103A300002038DF82830637A8DF82930A37A8DF847
:103A40002A30E37A8DF82B30237B8DF82C30637B82
:103A50008DF82D30A37B8DF82E300822E37B8DF876
:103A60002F300AA90EA80AF0D5FF124908220CA887
:103A70000AF0D0FF09E049464046FFF719FF10223F
:103A800049460CA80AF0C6FF0025337E0095A3F135
:103A9000FF025342534105990CAA404600F0D4FC62
:103AA00011B0BDE8F08F00BFAE1301089E130108EE
:103AB000E50901085E1301082DE9F04F89B003F113
:103AC00008099246059149461D468046129E0AF015
:103AD00043F89AF80730FF2B40F0B5806C78002C43
:103AE00040F0B180172E40F2AE802B7AFF2B00F011
:103AF000AA80002800F0A780183E2746002E27DD68
:103B000007F1180305EB030BEB5C022B0DD0212B07
:103B100016D10023029301932A78CDF800B04B46CA
:103B20005146404604F01CFF0AE006AB00932A7899
:103B300005985B46514600F09CFF041EC0F283804E
:103B40009BF8013007EBC307BFB2A6EBC306D5E76E
:103B50004FF0FF31059801F094FB08B1876800E051
:103B600007464946404609F0F7FF064600286AD056
:103B7000437E03F00703022B12D127B13B7813B128
:103B80007B78002B31D106A9A6F81A80347622461C
:103B900006F110000AF03EFF2B79590616D512E007
:103BA0001FB13B780BB17B7813BB002C49D1377E1A
:103BB000003718BF01272B799A062AD44FB3A4BB2C
:103BC0002B795B0601D5072101E01FB103213046A7
:103BD00000F02AFD95F90430002B737EB4BF43F04A
:103BE000080323F0080373762DE0002CCBD12AE0E4
:103BF0002CB3337E9C4209D0224606A906F1100060
:103C00000AF0D6FEB0FA80F0400900E00020074636
:103C1000D1E7002CD4D0A6F81A803476224606A923
:103C200006F110000AF0F6FECAE7737E03F0070300
:103C3000072B08D10321304600F0F6FC03E02746AD
:103C4000B9E70027B7E709B0BDE8F08F2DE9F04FDD
:103C500087B01546984681460291109FFFF7CAFB30
:103C6000B0F8C6319A07064669D5EB79FF2B66D1C5
:103C700098F80140002C62D1072F60D905F10803A4
:103C8000083F0DF1100A0393002F1FDD04F1080314
:103C900008EB030B18F80330012B0FD198F8002024
:103CA0000298CDF800A05B46294600F09BFE031E5B
:103CB00045DB524603994846FFF7FAFD9BF8013071
:103CC00004EBC304A4B2A7EBC307DDE7B6F8C63123
:103CD00013F0040F05F1080528D013F0010F194B5C
:103CE000194C18BF1C4605F0ABFD06F5FC77804665
:103CF0003846FCF7F5FEB6F8C631DB0716D529467F
:103D0000484609F029FF88B1B8FBF4F140F21523C9
:103D1000A6F80E320D4BC6F81002B3F9003006F5C6
:103D2000037204FB1181384608F078FD29464846A5
:103D300009F012FF18B1437E23F00803437607B061
:103D4000BDE8F08F80841E0020A10700DC10002059
:103D50002DE9F04F89B09246059181461E46FFF746
:103D600049FB0AF1080B05460822844958460AF027
:103D70001FFE002840F0FF809AF80830FF2B00F06B
:103D8000FA809AF80730FF2B40F0F5807378002B0B
:103D900040F0F180129B0F2B40F2ED8059464846CF
:103DA00009F0DAFE074650B90B230093024603469A
:103DB0005946484609F062FE074668B9DBE0437E93
:103DC000190706D5F28852BA92B212B923F0080345
:103DD00001E043F008037B76F3889CB264B15CBADF
:103DE000674B68491B88A4B21BB207F130026143DC
:103DF00007F11C0008F012FD33790BB185F8CA31C8
:103E0000B5F8C631C3F30D02A5F8C62173791B02BC
:103E100003F440431343A5F8C631B068A8B1D5F800
:103E2000D03190FA80F898450FD005F009FD0A22AC
:103E3000B0FBF2F303FB1200053008FB00F0C5F8FD
:103E4000D081B0FBF2F0C5F8D401F36813B11BBA0E
:103E5000C5F8D83105F5E070FDF750FF129B103B17
:103E60000393002302930493039B002B58DD029BD2
:103E7000103306EB0308F35C052B1CD004D8012B90
:103E80000DD0032B1ED03FE0222B2AD0232B3BD179
:103E90004346129A3146484604F0E0FE34E006AB51
:103EA0000093327805984346514600F09BFD031E6F
:103EB000049329DA5FE042463178484600F013FE69
:103EC00010BB58E042463178484600F029FE0028F1
:103ED00051D0D8F804301BBAB3B19C4228BF1C465D
:103EE00012E04146307804F00DFE002843D0B8F8C7
:103EF00006305BBA9BB23BB13C22B4FBF2F2934278
:103F000002D23C2202FB03F498F80130029A02EB41
:103F1000C30292B20292039AA2EBC3030393A3E7F4
:103F2000049B06AA59464846FFF7C2FC05F5EE7009
:103F3000FCF7D6FDB5F8C631DA071CD504EB44040E
:103F4000042C88BFA1084FF0000498BF0121384617
:103F500085F8CB4104F0BEFC3B463A462146B7F912
:103F60001A0000F0FDFAB5F8C6319B0703D5012110
:103F70002846FFF756FA09B0BDE8F08F5E13010836
:103F80000403002040420F002DE9F041437E03F07E
:103F90000703022B86B0044601D0052B7BD194F891
:103FA0009420B4F91A50012A71D9022B11D14FF083
:103FB00080730493FF238DF81430637B8DF81530E4
:103FC00040F2FF200021E389ADF81630CDE902016F
:103FD0000BE094E8030002AB83E8030004F108035C
:103FE00093E8030006AB03E90300013A84F8942048
:103FF0001DBB01AE304601F07FF80746BD4208D038
:1040000036F9150002AB2246002100F0A9FA01356D
:10401000F4E7224B04F13805B3F900602846FCF7B9
:104020005FFD40F21223A4F84E3004F14C023346F7
:104030001B49284608F0F2FB2DE02846FFF7DAF985
:104040000646224602AB06F5E075B4F91A000021D7
:1040500000F086FA01212846FDF720FE0F4BD6F826
:10406000D871B3F9008004F138063046FCF738FD0A
:1040700040F21223A4F84E303046434604F14C027D
:10408000394608F0CBFB2846FDF738FE03E0214611
:10409000284609F089FD06B0BDE8F081DC1000205B
:1040A00040420F00437E03F00703042B03D0072B8D
:1040B00004D1032100E0052100F0B6BA70470000EA
:1040C00038B500F5E075044601212846FDF7E6FD08
:1040D00005F0B6FB0A210A4BB0FBF1F202FB11001E
:1040E0000530C4F8D0314343B3FBF1F3C4F8D43105
:1040F000044BC4F8D8312846BDE83840FDF7FEBD72
:1041000080C3C90140420F0010B504460846237819
:10411000FF2B14D000221823872109F0EFFB002287
:1041200070B183681A715A719A71DA712168626884
:10413000DA609960A168E2685A61196110BD0020D7
:1041400010BD38B50B78FF2B05460C46104616D02F
:1041500000221823882109F0D1FB002280B1836856
:1041600025F01F051D71DA719A715A712168626814
:10417000DA609960A168E2685A61196138BD00206F
:1041800038BD08B500220823852109F0B7FB28B106
:10419000836800221A715A719A71DA7108BD10B5DC
:1041A000002304461046CA1D02F0F802194601F029
:1041B000EBF920B182681470C368DB08537010BD3E
:1041C000F8B516460F461A46B11CFFF7E8FF04463D
:1041D00060B18568C2680235023A002128460AF0BB
:1041E00017FD3246394628460AF014FC2046F8BD31
:1041F00013460A4601460120FFF7E2BF13460A466E
:1042000001460220FFF7DCBF2DE9F04180460F4652
:1042100016461D46002210238621079809F06EFBE2
:1042200060B1069B846827F03F0776BA2DBA1BBAA7
:1042300084F804806771E680A560E360BDE8F081E2
:104240002DE9F0410746884616462021079A0320AB
:104250001C46FFF7A4FF0546C8B1806824BA0021B8
:10426000846028F03F0800F1100436BA01734173EE
:104270008173C173877080F80380466010222046E6
:104280000AF0C6FC3A460699204605F0F9F8284699
:10429000BDE8F08110B50A46044608210520FFF765
:1042A0007EFF28B18368002224BA9A70DA705C60BD
:1042B00010BD000008B5102203490AF079FBB0FADE
:1042C00080F0400908BD00BFAE13010810B50822F8
:1042D000094904460AF06CFB48B12378FF2B08D14A
:1042E000607800F00F00831E5842584110BD012035
:1042F00010BD002010BD00BF5E13010870B506465A
:1043000008461946FEF7F4FE0446A0B18368FF2272
:10431000DA7100231A461946184600F003FF0546D5
:1043200020B92146204600F0E1FF02E083685E806C
:104330004460284670BD70BD002101F017BA00002E
:10434000F7B51F46537C802B05460E46144603D90D
:1043500011490320FCF748FC1046FFF7ABFF08B1FA
:10436000002017E02046FFF7B1FF0028F8D1217C9C
:10437000CB07F5D43388607C626913F0010F14BF5A
:10438000002680268DE89000A3693143FFF758FF8F
:104390002860012003B0F0BDE509010830B585B003
:1043A000022300930D460DF10E0300220521044661
:1043B00000F08EFC002803DBBDF80E30062B10D871
:1043C0000823009300222B460221204600F080FCA7
:1043D000002802DBADF80E000EE00023ADF80E3031
:1043E0000AE00823009300222B460321204600F018
:1043F0006FFC0628E4DDEDE7BDF80E0005B030BD2A
:1044000038B5002009F0F2FB044658B1637E03F092
:104410000703013B012B03D90A4B00221A600EE06F
:104420002046EFE7074D286809F0E0FB034618B97E
:1044300009F0DCFB034610B12B60184638BD20465E
:1044400038BD00BF901900202DE9F7430A9C0F46A4
:10445000994680461646FEF7CDFFB0F8C63199075B
:1044600001D4002507E04046FEF7C4FFB0F8C6318E
:104470005A07F6D580253046FFF71CFF38B11022C9
:10448000334930460AF0C6FA0223737001E045F062
:104490004005B9F1000F0BD069464046FFF77EFF9B
:1044A00030B1C1B222466846FFF7A8FE68B10446A3
:1044B00024B13B7CDB0758BF45F020052246394636
:1044C0002846FFF73EFE814608B920463BE00146FC
:1044D000002332464046FFF711FF054608B948461B
:1044E00031E03B7CDFF8749013F0010F23D005F02E
:1044F000A7F9184BB0FBF3F7314607FB130740460B
:1045000009F02AFB044618B913490320FCF76CFB99
:1045100000F154063046FCF7E3FA40F20223A4F817
:104520006A30E566B9F9003004F168023946304670
:1045300008F074F909E00146B9F9000000F0ADFB9C
:10454000002802DC2846FFF7F7FE03B0BDE8F08341
:104550006E13010840420F00E5090108DC1000203D
:104560002DE9FF4707460D4690469946FEF742FF64
:10457000824618B92A490320FCF736FB35B92A468A
:1045800041463846FFF710F8054668B102A938469B
:10459000FFF704FF064650B1C1B2002202A8FFF7A0
:1045A00027FE044620B935E00646044600E00446EE
:1045B000BAF8C631DB0714D5082E0AD008230093B9
:1045C00000226B440321384600F082FB80B20828A9
:1045D0001FD1234602AA0F21002004F0A7F9C0B181
:1045E000044621464046FFF78FFD064688B1014646
:1045F0002B464A463846FFF781FE044608B9304646
:1046000008E0084B0146B3F9000000F046FB002823
:1046100002DC2046FFF790FE04B0BDE8F08700BF43
:10462000E5090108DC1000202DE9F041437E23F06C
:1046300007030B4305290446437620D0072903D0FE
:1046400004294BD1264E05E0B0F91A00FEF7D2FE40
:10465000D0F8D461234B04F13805B3F90070284633
:10466000FCF73EFA40F21723A4F84E3004F14C0256
:104670003B4631462846BDE8F04108F0CFB8B0F9D6
:104680001A00FEF7B7FE03230646224606F5E0753C
:1046900084F89430B4F91A0023460021FFF760FF34
:1046A00001212846FDF7FAFA0E4BD6F8D871B3F976
:1046B000008004F138063046FCF712FA40F212236B
:1046C000A4F84E303046434604F14C02394608F017
:1046D000A5F82846BDE8F041FDF710BBBDE8F08124
:1046E000404B4C00DC1000202DE9F3411B4D00290C
:1046F00018BF0D46002229468046FEF755FF0746A3
:1047000070B169464046FFF749FE38B1C1B2002298
:104710006846FFF76DFD044618B91AE0044600E04C
:1047200004462046FFF72DFD064688B101463B466C
:104730002A464046FFF7E2FD044608B9304608E045
:10474000074B0146B3F9000000F0A7FA002802DC8D
:104750002046FFF7F1FD02B0BDE8F0818E1301089D
:10476000DC1000202DE9F04F8BB0002791468A46DF
:10477000039302900797FEF73DFE964B064600F521
:10478000E07801214046B94508BF9946FDF786FA11
:10479000B6F8C65115F001051BD1344606F5E3778E
:1047A000B3465C4500F0ED80627C9BF811309A4284
:1047B00040F0E4805946204604F03CFE637C83428E
:1047C00000F2DC8000E01D463834A045E8D1079DAA
:1047D0004FE004F0FBF9054600284AD0846906F54D
:1047E000E37BECB163689E4218D1AB699C4200F058
:1047F000D780A268996892F811E0487C864540F01D
:10480000E38010460593049204F014FE049A059B7D
:10481000527C824200F2D88000E01F462468E0E724
:104820004FF0010B05EBD4039A7D04F007030BFA5C
:1048300003F31A420CD0E0B202F066FD428A417CDA
:104840000346007C009704F0DBFA079060B107464E
:104850000134102CE6D12A46A98A28693B4604F087
:10486000F5FA0546079020B94046FDF747FA384665
:1048700081E0B6F8C6311B0707D52946B6F8C8014E
:10488000FFF708FD0790F8B10546BAF1000F0FD108
:104890004046FDF733FA494601220298FEF784FEAE
:1048A000012182464046FDF7F9F9BAF1000F10D018
:1048B00008A90298FFF772FD58B1C1B22A4608A8AC
:1048C000FFF796FC079018B94046FDF717FA3DE050
:1048D0000546B6F8C62102F01004A4B20CB196F851
:1048E000CA4102F020039BB24BB1D6F8D4313A4909
:1048F0008B4206D84FF47A7BB3FBFBFB03E09B466D
:1049000001E0DFF8DCB002F04007BFB22FB1D6F80B
:10491000D8714FF47A73B7FBF3F7039B13B9B6F86A
:10492000CC2100E0002240460392FDF7E7F9B6F8FB
:10493000C611039A01950912204600975B4601F0C3
:10494000C001FFF761FC0446079008B9284612E051
:10495000014653464A460298FFF7D0FC01460790AD
:1049600008B9204607E01D4BB3F9000000F095F9A7
:1049700000282BDC0798FFF7DFFC27E00BF1380B52
:104980000FE72B462246394607A8FFF7D9FC002837
:104990003FF41AAF079B002B7FF415AF28460DE0BC
:1049A0003B46A268594607A8FFF7CAFC00283FF417
:1049B00035AF079B002B7FF430AF3846FFF7BCFCC8
:1049C0004046FDF79BF901E01B680FE70BB0BDE81F
:1049D000F08F00BF7E13010800A493D6DC100020E6
:1049E00080EE3600F8B51E469F1C5B7804461546DF
:1049F00013B96FF01500F8BD01F10800FFF75AFC7C
:104A00000028F6D17CB394F91030013304D1A368A7
:104A10001C78022C04D001E06468F3E7082C06D16E
:104A20007378012B14D0022BE3D1082411E0853DCB
:104A3000022D1BD884B9727808236FF0010413FB90
:104A4000024402FB036616F8013D2BB9013CFAE76C
:104A50000224853D022D09D822463946069809F0E0
:104A6000D9FF2046F8BD853D022DE4D96FF08500C1
:104A7000F8BD70B51D465B780446164613B96FF055
:104A8000150070BD01F10800FFF714FC0028F6D1F5
:104A9000882E27D1A91CA4B194F91030013304D178
:104AA000A3681C78022C04D001E06468F3E7082CAA
:104AB00006D16B78012B0ED0022BE0D108240BE03D
:104AC00054B96C78E408023CE4B20B1913F8013CC9
:104AD00013B9013CF8E702242246049809F09AFF32
:104AE000204670BD70BDF8B517460D46FEF782FC36
:104AF0007C78012C06460FD1862D0FD100F5E0758C
:104B000021462846FDF7CAF87B681BBAA6F8C831CB
:104B10002846FDF7F3F801E00020F8BD2046F8BD77
:104B20002DE9F0415378042B86B00746154671D124
:104B300086294ED102F110084046FFF7C7FB064612
:104B4000002846D13846FEF755FCB0F8C631DA07E2
:104B500003D595F90330002B3BDB41463846FEF781
:104B60009FFC044618B1427CAB789A422AD06B680D
:104B700043B31022002102A80AF04AF8EB785B0642
:104B800016D4AA78414602A804F07AFCEB78AA78F9
:104B900003F0C00302A93846FEF74AFC0446002889
:104BA00039D03846FEF726FC012103F0DFFF09E08B
:104BB0000821009104AB0022384600F089F8002853
:104BC000DFDA28E06B6833B91CB121463846FEF7BE
:104BD00057FC01261FE01BBA6361AA68013312BAB1
:104BE000A2610CD00E4B69680E481B8809BA41437C
:104BF0001BB204F1300204F11C0007F00FFE237C0D
:104C000023F07F03DBB22374EA7822F03F021343E0
:104C10002374DEE70026304606B0BDE8F08100BF11
:104C20000403002040420F002DE9F341044688466A
:104C300017461D4600F0F8FA064650B34146204696
:104C400000F0E0FA711E0446284600F07DFD04B332
:104C5000237A53B1012B17D1E068ADF8027000221E
:104C60006946019508F0F6FC07E0B4F90C10ADF8C0
:104C7000027068460195FDF7A7F9002804DD20467B
:104C800000F0E6FA0446E2E70021284600F06EFD57
:104C9000F5E7304602B0BDE8F08107B540F20223E7
:104CA000019101466846ADF80230FDF78DF903B079
:104CB0005DF804FB07B540F2012301910146684607
:104CC000ADF80230FDF780F903B05DF804FB000099
:104CD00000B589B006930A9BADF81C304FF4017300
:104CE0008DF81410ADF81620ADF80630024605AB6D
:104CF00003A901A80293FDF78BF9BDF80E2040F23D
:104D000005239A4203D004490320FBF76DFF049862
:104D100009B05DF804FB00BFE509010800B589B0E2
:104D200006930A9BADF81C3040F203238DF8141053
:104D3000ADF81620ADF80630024605AB03A901A870
:104D40000293FDF765F9BDF80E2040F205239A4263
:104D500003D004490320FBF747FF049809B05DF82E
:104D600004FB00BFE50901082DE9F043846807460C
:104D7000208F638D8FB000F0280EADF818304EF004
:104D8000010E0E4611B96FF015005DE091F910307B
:104D9000013354D18D682B792A7813F0C00F03BFEB
:104DA00002F108035B1995F801C0294B18BF4FF0B9
:104DB000020C12B105F1080107E0420747BF04F1F8
:104DC0002E01082204F12C01022294F8360000F191
:104DD000010884F8368004900DF12008BDF8180011
:104DE000ADF80800ADF80400CDF80CE0CDF800C037
:104DF000404604F0A3F981460028C4D0304607A9F4
:104E000000F048FA0646E8B1816881E800032B7992
:104E100013F0C00FBB6815BF1A69DA68013201329E
:104E200014BF1A61DA602368079A1B682046984706
:104E300000210446304600F099FC204604E06FF063
:104E40004C0001E06FF068000FB0BDE8F08300BFD8
:104E50005C1301082DE9F04387683B685C68002318
:104E600087B01A4619463846A047041E15DD0023B0
:104E700022461946184600F087FB054668B13B6894
:104E800081685E6822466B463846B047B0F100083C
:104E900005DC0021284600F069FC002466E03E8F16
:104EA00006F00206B6B2002E5BD1A86804F0DAF96B
:104EB000044608B9014637E00146C0EB080832460F
:104EC000284600F07BFB814608B90146E2E7866888
:104ED00001AA04A9304604F03BFA01AA044602A93B
:104EE000304604F0E3F9002C01DA00241BE000282E
:104EF000FBDBC1B2E3B204AA02A800F013F9064634
:104F00000028F2D0022C0CD19DF81030FF2B08D1D4
:104F10009DF81130FF2B01BF8268137963F07F0386
:104F20001371344626B90021284600F01FFC1DE00D
:104F3000B3689DF801209A719DF800205A710D4ABE
:104F400012885A8097F828302B744946284600F07A
:104F5000CDF9002373602B465A680AB11346FBE76C
:104F60005E604146284600F097FB2C46204607B07D
:104F7000BDE8F08304030020034B0360034B436050
:104F800081600020704700BF694D0008554E000841
:104F9000F0B5254E84683388838195B00821054695
:104FA00004A8FDF797F83088204B6360A56000B235
:104FB00000F090F8236820469B68984740F203274A
:104FC00041F234266846FDF782F8BDF80230BB4254
:104FD00013D0B3F5017F08D240F202229342F1D1FF
:104FE0002B68019928469847EAE70AD0B342E9D1ED
:104FF00023682046DB689847E2E7236801995E69E9
:1050000002E0236801991E690B894A6809782046E5
:10501000B04740F20523039002A96846ADF80A3074
:10502000FDF724F8CCE700BF04030020315000084E
:1050300013B50346806879B941F234230190B0F981
:105040000C10ADF802306846FCF79CFF002822DC0B
:10505000124809F06FFF1EE0042919D0072913D068
:10506000022918D1436898470446A0B103460C4969
:1050700090F9100040F20122FFF7D6FD014650B929
:10508000204600F073FB06E09A6901329A6102E063
:105090005A6901325A6102B010BD00BFA211010865
:1050A0000000FFFF30B585B0089C6CB1A5685DB10C
:1050B0000293074B009301940823FBF735FE002869
:1050C000D8BF6FF0150001E06FF0120005B030BDE1
:1050D000914F0008074B10B5B3F90040A04201D131
:1050E000002010BD14B16FF00B0010BD1880FEF74A
:1050F00055F9F5E794190020044BB3F9003013B1CA
:105100000380012070471846704700BF94190020A3
:10511000034BB3F900301B1A58425841704700BF87
:10512000941900202DE9F041174603F108020A44C2
:105130000E46002180461D4608464FF0FF3300F022
:1051400023FA00220446F8B183681E705D705A800D
:105150005A719A711A71B8F1000F08D03EB1806887
:105160000278B24203D14146083009F053FC5FB1E6
:1051700055B1A0684378AB4206D1037808332A467C
:105180003946184409F046FC2046BDE8F08100008D
:1051900008B50B7A53B9B1F90C200B4B53F82230F8
:1051A0001B6A1BB909490320FBF71EFDC3B2042B80
:1051B0009FBF074B53F820200A6043F8201094BF8C
:1051C00000206FF0150008BD50030020E50901081C
:1051D00098190020C3B2042B11D8094A52F8203084
:1051E0008B4206D11B6842F820307047914204D0B0
:1051F00013461A68002AF9D101E00A681A6070475C
:1052000098190020C3B2042B09D8064B53F820008C
:1052100020B143688B4203D00068F9E77047002053
:10522000704700BF98190020C3B2042B0BD8074B5E
:1052300053F8203000202BB15A681B688A4208BFFF
:105240000130F8E770470020704700BF9819002030
:1052500028B14368006810B142689342FAD17047A0
:1052600049B190F91030032B03D0042B06D103F081
:1052700007BF08F053BB6FF0150070476FF00100D7
:10528000704728B190F910308B4201D04068F8E7A0
:105290007047000070B504460E4619B91249032044
:1052A000FBF7A2FC10B90020306070BD014600255C
:1052B000496801350029FBD16FF00103EA0020465F
:1052C00000F062F90028EED08368002BE6D00833A6
:1052D000A26843F8082CE268646843F8042C083399
:1052E000002CF5D1356070BDE509010810B5044604
:1052F0008C42084601D1646808E023465A682AB106
:10530000904201D01346F9E742685A60002141609B
:1053100000F02CFA204610BD70B5556804460846CA
:10532000EDB129464B680BB11946FBE71CB91A4988
:105330000320FBF759FC0028F9D0002AF7D0436876
:105340005360844206D023465E6826B1B04219D02D
:105350003346F9E7144653684B60556015E0002C5E
:10536000E5D00029E3D0002AE1D04B6853608C429D
:1053700006D02346596841B1884205D00B46F9E76B
:10538000144602E05A60E6E75A600021416000F0EE
:10539000EDF9204670BD00BFE509010870B5034670
:1053A0001A4A072B88BF033310688CBF23F003030E
:1053B0000823002140B34468A34202D90146006893
:1053C000F8E7E41A072C0344114E05D8046809B91C
:1053D000146011E00C600FE0C6F108051D44B5F53E
:1053E000C05F02D90021116003E009B9136000E039
:1053F0000B60026883E81400064A9B1B11889BB26D
:10540000994201D2138070BD70BD00BFB019002059
:10541000B4190020AC19002001210148FCF73EBC62
:10542000B4310020204A38B5831AB3F5C05F39D2B1
:105430001E4D2C68002324B1844202D223462468E6
:10544000F9E707298ABF0331082121F0030104602D
:10545000141AC1F5C0522244072A98BF8918416026
:105460000BB9286011E05A6818601A44821A072A9A
:105470000BD818B90E490320FBF7B6FB0268416848
:105480001A60C21A0A445A601846036853B1426847
:1054900002449A1A072A05D81A6802601A1A5B6829
:1054A0001344436038BD00BFB4190020B019002078
:1054B000E50901082DE9F843814614200F461646F8
:1054C0009846FFF76BFF0446D8B15EB13046FFF750
:1054D00065FF054638B920461421FFF7A3FF28468B
:1054E000BDE8F88335460123C4F80490A560E66062
:1054F00084F81080236027B132463946284609F0E7
:1055000089FA2046BDE8F883F8B50F4D0446002619
:10551000CCB1631BB3F5C05F03D30C490320FBF789
:1055200063FB94E88800012B09D1E168A06826603C
:10553000FFF778FF14212046FFF774FF01E0013BDD
:1055400023603C46E4E7F8BDB4190020E5090108F2
:1055500008B5FFF761FF094A094B136018210022C3
:105560001A705A709A70DA701A7159719A71DA71E8
:105570000448BDE80840FCF7C1BB00BFB0190020DB
:10558000B4190020B4310020B2F5C05FF8B505466B
:105590000E4614461F460DD8FFF73EFF22463B46F7
:1055A00031462846FFF786FF04460348FCF7A6FB72
:1055B0002046F8BD0020F8BDB431002007292DE9B0
:1055C000F84388BFCF1C0D468CBF27F00307082780
:1055D00004469146FFF720FF2DB124B1E3689D42B8
:1055E00001D8A3682BB92B48FCF788FB0020BDE845
:1055F000F8831420FFF7D2FE06460028F3D0E368B4
:105600009D422ED0AF4202D85A1B072A29D82846DD
:10561000FFF7C4FE074610B9142130460BE0E068DE
:10562000401BFFF7BBFE804640B914213046FFF710
:10563000F9FE29463846FFF7F5FED4E72A46A16869
:10564000384609F0E7F9E268A168521B2944404650
:1056500009F0E0F9E168A068FFF7E4FEC4F808800B
:1056600005E0A7689D4214BF7B190023A360E3688F
:1056700008485B1BE360636873600123B760F560F3
:1056800086F8109033606660FCF738FB3046BDE862
:10569000F88300BFB4310020072970B588BFCE1C45
:1056A00004468CBF26F0030608260D46FFF7B4FE1D
:1056B0001CB922490320FBF797FAE368A06813B9E5
:1056C0000028F6D106E00028F3D01D4A821AB2F570
:1056D000C05FEED29D422CD02DB930B11946FFF7F4
:1056E000A1FEA56024E09D4202D8991B072917D886
:1056F0002846FFF753FE064620B91248FCF7FEFA8B
:105700000C2070BDA16829B1E268AA4228BF2A46D0
:1057100009F080F9E168A068FFF784FEA66007E061
:10572000033323F003039E4202D23044FFF77AFE94
:10573000E5600448FCF7E2FA002070BDE5090108C5
:10574000B4190020B431002038B504460D46FFF7E7
:1057500063FE24B123682B4423606468F9E70248A0
:10576000BDE83840FCF7CABAB431002010B5044691
:10577000FFF752FE2046FFF7C7FE0248BDE8104083
:10578000FCF7BCBAB431002038B50446FFF744FE3C
:105790000CB1E26822B90E48FCF7B0FA002038BD1F
:1057A0002368012B0FD994F91030A1686068FFF7C6
:1057B00081FE054610B12368013B23600448FCF7D5
:1057C0009DFA284638BD0248FCF798FA204638BDB5
:1057D000B4310020F8B50026074604463546002CB3
:1057E00048D02946E268294809F01AFB94F91010BC
:1057F0004B1C052B31D8DFE803F006030F182028D7
:10580000002123482AE04FF0FF31224809F008FB2D
:10581000A06808F0D3FA28E001211F4809F000FB36
:10582000E168A06806F048FC1FE002211B4809F06F
:10583000F7FAA06803F080FF17E00321184809F089
:10584000EFFAA06803F066FC0FE00421154809F0A8
:10585000E7FAA06806F06EFE07E0134809F0E0FAE8
:105860001022E168A06803F0B3FFE36864680135C3
:105870001E44B4E7294632460C4809F0D1FA2146C5
:105880003846BDE8F840FFF771BF00BFC8110108F6
:10589000ED11010801120108151201082D1201086D
:1058A0004012010855120108671201087D12010813
:1058B00000B595B0082104A8FCF70CFC6FF0850337
:1058C000039340F20523ADF80A306846FCF7FFFB6E
:1058D000BDF802306FF400721344032B11D8DFE8D7
:1058E00003F002040B0B094800E0094809F022FB11
:1058F0000198FFF76FFFE8E702A96846FCF7B6FBDF
:10590000E3E7044809F016FBDFE700BFAA1201082D
:10591000C2120108D91201081FB50A4CB4F90030AF
:1059200063B9094A0193094B0292009306220823A6
:105930004FF4C0610648FBF7F7F92080B4F9000086
:1059400004B010BDB831002000130108B1580008A0
:10595000BA31002007B501A8FFF7CEFBBDF904005E
:1059600000F006F903B05DF804FB00002DE9F043F8
:10597000082187B07648774C774FFCF7ABFB40F2B5
:105980000523ADF81230264602A8FCF7A0FBBDF8AF
:105990000A30B3F5017F09D840F20322934280F028
:1059A000CF8040F20122934277D0EDE7B3F5106F3C
:1059B00004D040F60112934264D0E5E7674D05F14B
:1059C000900815F8013CD3B1D5F81730022B0DD94A
:1059D000042B05D8D5F813302946986900F0E0FA71
:1059E000D5F81730023BC5F8173008E0D5F813900A
:1059F000681F01F0C7F80021484601F051F9303521
:105A0000A845DED16378ABB394F98C30002B20DC51
:105A100096F83730022B18D894F8351051BB94F80B
:105A20003430032B07D93C2384F8373084F8341002
:105A300084F835101EE0013394F82920206A84F898
:105A4000343000F0ADFD032300E0023B84F8373032
:105A500010E0E269002ADBD1218E4FF6FF729142FD
:105A6000D6D1023B5BB2002B84F88C30D0DC3948B5
:105A700001F0E3F8B7F90030394A3A493A4806F0FC
:105A8000CDFE81E7039800283FF47EAF4369002BE9
:105A90003FF47AAF06F0F0FC76E7039D1DB9334979
:105AA0000320FBF7A1F802212846FFF7EAFB4FF09D
:105AB000FF3180462846FFF7E4FBB8F1000FEED037
:105AC00018B18368B3F9021000E00146A868D8F85D
:105AD00008204378032B2ED8DFE803F0020D1823AB
:105AE00093885BBA9BB20093043002F1180308322A
:105AF00000F098FA1FE093885BBA9BB200930430E1
:105B000002F11803083200F0A9FB14E093885BBA95
:105B10009BB20093043002F11803083200F0AAFE91
:105B200009E093885BBA9BB20093043002F118033A
:105B3000083200F0F9FE00212846FFF717FE23E7A0
:105B40006FF0850304A902A80593FCF78FFA1BE701
:105B5000BC370020C03C0020BA3700201538002098
:105B60006402002080841E00A8380020E509010896
:105B70007FB51C4CB4F90050064625BB1A4B1B4898
:105B80001D701B4B02931B4B0093019508230522AC
:105B90004FF48061FBF7C8F8208000B316499B22C0
:105BA000888103204A60FFF7F3FA00F005FF134AEB
:105BB00013491448B4F9003006F030FE802229461B
:105BC000114809F025F80023802210493046FDF7DE
:105BD0002FFC00200D4900F0E3F9B4F9000004B0F7
:105BE00070BD00BFBA370020A0380020BC380020AC
:105BF000181301086D590008FC37002064020020CA
:105C000080841E00A8380020503D002008130108A1
:105C1000012380F82F30002380F82C3080F82D30BD
:105C200070473C2380F82F30002380F82C3080F818
:105C30002D30704710B5012104460948FCF72EF8B5
:105C4000084B1878421C1A7014B140F0800401E02F
:105C500000F07F040248FCF751F8204610BD00BF59
:105C6000A4380020A038002013B50C4612B1184605
:105C7000FFF7E0FF2146022201F0E2F8044678B384
:105C80000022032180F8252080F827100123142208
:105C90000A2180F8243080F8262080F8281084F823
:105CA0002F3084F832304FF48073238694F83630E6
:105CB000052043F0030384F8290084F836303C20A3
:105CC000094B6085F02084F82E00B3F900000191A3
:105CD0000092082340F6011204F1380106F0F2FBAD
:105CE000204602B010BD00BFBA3700200021FFF7E8
:105CF0003DBD10F0800F4BB202D0002B11DA01E055
:105D0000002B10DB884204D2C1F1800303440F2B27
:105D100009DD884205D9401A0F28CCBF0020012098
:105D2000704700207047012070470000F8B5074613
:105D300015461E460C4639B920461949FDF7D8FBD1
:105D4000044608B9384625E035B916492046FDF71E
:105D500009FC05460028F5D0114A2946002E18BF37
:105D600032463846FDF7C4F906460028EAD000233B
:105D70001A4619461846FFF7D5F983680A495C8028
:105D800005464660034640F202220220FEF74CFF21
:105D900020B92846BDE8F840FFF7A8BFF8BD00BF0E
:105DA000081301085E1301080000FFFF002370B50F
:105DB00010220C4619460646FFF7E6FB054618B9C1
:105DC0003046FFF793FF24E0836804221A70002115
:105DD0000E225A709970A27FDA70E27F1A7194F8DD
:105DE00020205A71A269B2F88A2052BADA80A269D8
:105DF000B2F8882052BA1A81A269D2F88420128897
:105E0000197352BA5A8194F821205A73628C52BA8B
:105E1000DA81284670BD002370B520220E4619464F
:105E20000446FFF7B1FB054618B92046FFF75EFFB1
:105E30001EE08068082303701E2343704023C37054
:105E400033695A6942609A6982605B7C8370002181
:105E500000F11004017341738173C1731022204655
:105E600008F0D6FE336931465A7C204603F008FB21
:105E7000284670BD2DE9F3410F460446002800F086
:105E8000898090F8363003F0020300F1080603F031
:105E9000FF0533B131460020FFF7BDFF054600285E
:105EA00078D094F83630DB070CD528463146FFF71A
:105EB0007DFF054600286DD094F8363023F00103AD
:105EC00084F836300023182219462846FFF75CFB79
:105ED000804608B9284637E0836822781A7094F81B
:105EE0002E205A7094F83220022A04D14FF0FF324B
:105EF0009A70DA7002E0228E52BA5A8094F88020AA
:105F000094F82F10D20042EAC11294F825100A43E7
:105F10001A7194F824205A7100229A71DA71354668
:105F2000083304F1180E2A4603CA724518605960F6
:105F3000154603F10803F6D1042301229B214046B4
:105F400007F0DCFC28B9404602B0BDE8F041FFF79D
:105F5000CDBE03460022D9685B680A44002BFAD103
:105F60000E4B17B13978FF290DD19969013199612B
:105F7000D9690A44DA61B4F92C1000963B46002234
:105F8000FFF7D4FE06E019690131196159690A4425
:105F90005A61F0E702B0BDE8F08100BF503D00203B
:105FA000F0B51E4B85B000220546186803900F46D9
:105FB0000A239B21104607F0A1FC064658B38068CF
:105FC000002404714471042203A9063008F022FD64
:105FD00032462346D16852680B44002AFAD1104A4F
:105FE00017B13978FF290FD1916B01319163D16BD2
:105FF0000B44D36305B10835002200953B4611469A
:106000003046FFF793FE06E0116B01311163516BCF
:106010000B445363EEE705B0F0BD00BF1C1301084D
:10602000503D002030B41948BDF808505BB11978D4
:10603000FF2908D0046A01340462446A2C44446293
:10604000052D07D820E0846A01348462C46A2C4498
:10605000C462F5E71B780E48FF2B09D143789BB14A
:1060600090F83230022B0FD0383030BC06F014BA22
:1060700043784BB190F8363043F0010380F8363066
:10608000114630BCFFF7F6BE30BC7047503D0020D3
:10609000C03C00202DE9F04F8BB00026159F0793E0
:1060A0003E600C46154600F048FF8246002800F08E
:1060B000CF80B0464FF47A7B079B434540F2C880BF
:1060C0002B78082B00F2BD80DFE803F0050FBBBB87
:1060D000147698BB4C003B6808F1010843F00103BB
:1060E0003B601FFA88F80135E6E73B6843F002039E
:1060F0003B60A6E03B6843F010033B6094F8363009
:1061000043F0010384F83630688940BA80B200F069
:106110005BFC10B1C4F8840003E000F055FCC4F847
:106120008400E87884F8260095F804E084F827E0F5
:10613000697984F82810EB885BBAA4F88A302B8937
:106140005BBAA4F888306B7B84F82930EA8984F83C
:106150003900012352BA03FA0EF36285E36384F82F
:1061600038106EE03B68B4F92C0043F480733B6058
:1061700094F83630082143F0020384F83630009159
:1061800008AB0022FEF7A4FD002802DAEB785B06DC
:1061900057D5082208A905F1100905F1180008F0E3
:1061A00039FC0023AA78B4F92C004946FDF740F9E0
:1061B000002846D0A06144E03B68B4F92C1043F0BD
:1061C00020033B6094F82900638DEA7843430BFB7E
:1061D00003F3002E08BF2E460493802A4FF00103DC
:1061E00094BF12060022149803931023019000928A
:1061F00002932A1D1848FCF7EBF822E03B6843F0B5
:1062000040033B600EB900261BE04FF010096A798D
:10621000638DCDF8009053430BFB03F3029395F984
:1062200002300D48DB43DB0F0193311D149B10221C
:10623000FCF756F9737802331E443378052BE6D009
:10624000E1E76B78023398441FFA88F81D4433E77E
:1062500050460BB0BDE8F08FA81000202DE9F047A4
:1062600086B017460022039204460D46BDF83860FA
:10627000A74A5BB11B78FF2B08D01368013313606A
:106280005368334453601B2E07D83DE193680133B4
:106290009360D3683344D360F5E71C3E03A92078AC
:1062A000B6B200F0ABFB002800F0898063885BBACF
:1062B0009BB24FF6FF72934200F023812379DDF801
:1062C0000C80C3F3C20388F88030002000F07CFB10
:1062D000C8F884004DB928468E49FDF709F90546EE
:1062E00018B98D490320FAF77FFC2A46002304F1F0
:1062F0000801039800F0B2FB039D06AA05F1080807
:10630000002342F8083D3946404600F0E7FB18B943
:10631000049B002B00F0F580637885F82E302379FC
:106320000399DB0985F82F30237903F0070385F8FB
:1063300025306388049A5BBAD38206AB002243F807
:10634000042D012001930097334604F11802FFF752
:10635000A1FE002800F0D580059810F0100407D1A8
:10636000039800F06AFC39462046FFF719FECBE09F
:10637000AB6943B94146B5F92C00FDF7F3F80028A5
:1063800000F0BF80A8614046FFF742FC634A95F8E1
:106390002730B2F9000095F82820019295F82620C0
:1063A0000092012202FA03F305F1380140F60112CE
:1063B00006F088F80499404600F072FCA4E0039DC2
:1063C000002D00F0A18005F10808102204F1080159
:1063D000404608F0EDFA8146002840F09580039A87
:1063E000237992F88020C3F3C2039A4240F08C8054
:1063F000627895F82EA010465146FFF77AFCC8B196
:1064000095F83230012B0FD1130601D5FF2A00E099
:106410007F2A1ABF0132D2B24A4685F82E2005F1F2
:10642000380006F039F80BE085F82E20404600F0E1
:1064300015FC05E011465046FFF75BFC002837D1FC
:1064400095F83230012B0BD163885BBA9BB24FF6C3
:10645000FF72934205F138002CD006F066F853E045
:1064600006AA002342F8083D3946404600F036FBB4
:10647000049B08B9002B47D01BB105F1380006F08A
:1064800054F8049900293FF42CAF63885BBACB829F
:10649000404600F005FC049B1A7972B963885BBA28
:1064A0009BB24FF6FF7293422ED12A8E9A422BD086
:1064B00005F1380005F0F0FF26E0EA69934223D1A8
:1064C0005A7D63799A4202D04046FFF7A1FB049BB4
:1064D00062795A7523790399DB0985F82F3023797E
:1064E00003F0070385F8253006AB002243F8042D9E
:1064F000012001930097334604F11802FFF7CAFD0B
:1065000010B9039800F099FB06B0BDE8F08700BF12
:10651000503D002008130108E5090108BA370020A2
:10652000F8B500230C461646194614220746FFF715
:106530002BF8054618B93846FFF7D8FB11E08368F9
:1065400005221A7012225A7000229A70DE702146BB
:10655000043304F1100251F8040B43F8040B914288
:10656000F9D12846F8BDF8B500230E461546194660
:1065700006220746FFF708F8044618B93846FFF721
:10658000B5FB0AE0836806221A7004225A70ED01F6
:1065900000229D70DA701A715E712046F8BD00000D
:1065A0002DE9F04F8DB00E4606920546002800F00A
:1065B000FD8090F83230012B00F0F88021B9C669D7
:1065C000002E00F0F38005360CA805F10803002426
:1065D000194640F8044D059309940A94FCF79CFF72
:1065E0000B9B002B00F0E28001217248DFF8D8B14C
:1065F000FBF754FBA04604940394DBF808309C425C
:1066000068D2DBF8007007EB4417D7E90223134385
:106610005ED0BB69DA070CD4039BD3B9012206997B
:106620001846FFF7A0FF0A9088B96248FBF766FB9F
:10663000BCE0049B83B91A4606991846FFF793FFFE
:10664000804609900028F0D00123049304E0012340
:1066500003930DF1280901E00DF124097B699A7873
:10666000FF2A03F1020A07D1D87800F00F00A0F149
:106670000E035842584120E008224F4907935046E4
:1066800008F096F9079B08B9002016E09A78FF2ACF
:1066900004D1DB7803F00F03022BF5D01022474919
:1066A000504608F085F90028EED0102244495046A3
:1066B00008F07EF9003018BF012048B1FA7CD9F803
:1066C00000005146FFF72CFFC9F800000028ACD0AD
:1066D000013492E73748FBF711FB0A9BB8F1000F32
:1066E00002D0C8F8043000E0099380220B99099881
:1066F000FFF716FF04460990002857D095F900705F
:10670000002F07DA002310220599FEF73DFF0A90BB
:1067100030B30990DDF82480002304221946404656
:10672000FEF732FF04460A9008B9404619E0836834
:106730002A781A70002FB4BF402200225A705A786B
:10674000099062F07F025A7095F83320DA700027C2
:106750009F70022204239B2107F0D0F80A9018B9F9
:106760002046FFF7C3FA21E0099002463B46D16874
:1067700052680B44002AFAD13278FF2A114A0ED00F
:10678000116D01311165516D0B445365059BB5F9D0
:106790002C10009300223346FFF7C8FA06E0916DF3
:1067A00001319165D16D0B44D365EFE70DB0BDE8C4
:1067B000F08F00BFB41000205E130108AE13010873
:1067C000BE130108503D0020A81000202DE9F7431A
:1067D0000E4691460446002846D090F90080B8F154
:1067E000000FACBF0823182303229B21002007F0D1
:1067F00085F80546002837D0876823783B71B8F1C3
:10680000000F09DA80237B71102204F1080107F1DF
:10681000080008F0FFF801E000237B71002387F8EF
:106820000690FB712A46D16852680B44002AFAD1BF
:106830000F4A16B13178FF290FD1916F013191675D
:10684000D16F0B44D367B4F92C100834009433464D
:1068500000222846FFF76AFA06E0116F013111673E
:10686000516F0B445367EEE703B0BDE8F08300BF00
:10687000503D00202DE9FF4117460546BDF8284050
:10688000284A8BB11B78FF2B0ED0136C0133136495
:10689000536C234453646B7813F0400F0CBF0823F0
:1068A00018239C423AD306E0936C01339364D36C73
:1068B0002344D364EFE7287800F0C2F8064668B3B3
:1068C0006B785B0605F1040106F1080801D4083C69
:1068D00007E01022404608F06BF8F8B905F1140102
:1068E000183C96F83220022AA3B217D004AA00203E
:1068F00042F8040D0097019202200A463146FFF744
:10690000C9FB58B195F90130002B04DAEA78394611
:106910003046FFF75BFF4046FFF77AF904B0BDE869
:10692000F08100BF503D002070B5224A0446BDF8FA
:106930001000A3B11978FF2911D0116E0131116631
:10694000516E014451661B78FF2B32D094F901300F
:10695000002BACBF0823182398422AD106E0916E81
:1069600001319166D16E0144D166ECE7207800F0E8
:1069700067F80546E8B194F90130002B05F10806E7
:1069800002DBE37843B90CE01022211D304608F009
:106990000FF80028F5D070BDA27895F833309A42F0
:1069A00007D1012385F835303046BDE87040FFF748
:1069B00038B970BD503D002008B500F021FB014BF7
:1069C000186008BDD03D0020054B1B680BB900F0D6
:1069D00017BB1A8882420CBF18460020704700BFC0
:1069E000D03D002090F83220022A02D1383005F044
:1069F00099BD0149FFF73EBA0813010810B50023FD
:106A00000E4A0B6054780CB90A6004E01478844292
:106A100001D10A600FE00B686BB118700B680120A0
:106A200058700B6800224FF48071A3F88A20A3F8F5
:106A30008810DA6110BD184610BD00BFC03C0020B0
:106A4000054A53782BB1137883420CBF10460020BF
:106A500070471846704700BFC03C0020F8B5044698
:106A600008B1407818B91B490320FAF7BDF80D4664
:106A700004F1080701F1100E286869683E4603C654
:106A8000083575453746F7D14FF6FF712186124913
:106A9000E164142184F82610032184F827100A21C8
:106AA00084F82810052184F829103C216185F02004
:106AB000002184F8330084F8321084F8241084F81C
:106AC0003410246584F835102462A285A361012066
:106AD000F8BD00BFE5090108E56900082DE9F843A4
:106AE0000026264F166080460D4614464FF00109D9
:106AF00017F8013C33B9B9F1000F14D07A1F2260A6
:106B0000994610E0D7F8133043450CD12946384652
:106B100002F07BFC38B11A4A302303FB06262660BC
:106B20000020BDE8F8830136032E07F13007DFD1DE
:106B3000206800B3C0F81880236800221A60D8F8D3
:106B4000143033B11A680AB11346FBE722681A60A1
:106B500002E02368C8F81430236801221A71236800
:106B60002946053305F1100251F8040B43F8040BD4
:106B70009142F9D10120BDE8F88300BF153800200B
:106B80001038002030B5044687B018B920490320DA
:106B9000FAF72AF885696B6998422AD110221D49B3
:106BA0001D48FBF7E6FC2368D3B10020FAF7EAFDA5
:106BB00022681A4BB0FBF3F0D369B5F92410181A08
:106BC0004FF47A7358430532012303930192102343
:106BD00000220490009202930E4A0F48FBF7F8FB44
:106BE0006B699C4205D123686B6108E0944204D034
:106BF00013461A68002AF9D101E022681A6030228F
:106C00000021204608F004F8012007B030BD00BF85
:106C1000E5090108AE130108A810002040420F004A
:106C200038B50446406920B10568FFF7ABFF284638
:106C3000F9E74FF6FF73238538BD10B504460830D9
:106C4000FFF7EEFF04F1380005F06CFC9022002104
:106C5000204607F0DDFF012010BD000010B5037FC6
:106C6000013303774369044633B1FFF7D9FF10229C
:106C700009490A48FBF77DFC228D4FF6FF739A42C3
:106C800008D0238504F1300005F006FCA369052235
:106C900083F88C2010BD00BFAE130108A81000209F
:106CA0002DE9F04F0A4689B00446E1B1438C90F8D3
:106CB00021105943D16141698A4214D1B0F924109D
:106CC00090F8210043434FF47A7043430532049314
:106CD0000123039301921023002200920293564A4B
:106CE0005648FBF775FB6369228D0692002B00F076
:106CF00099804FF0010B00226669626192469146CD
:106D0000002E36D00AF1010A354600272D680137DA
:106D10000DB9D84610E05F45F8D1FAE7B8F1000F99
:106D20000DD12A4635463668013FB9F1000F1CD017
:106D3000C9F80050A9461546002FEFDC01E02DB937
:106D4000EFE7B8F1000F12DD8DB157B1A2690793DB
:106D5000D2F884202946D268304690470028079B05
:106D6000DFDD2A6808F1FF38DFE76561E2E72E46DC
:106D7000C6E7B9F1000F01D0C9F80060BAF1010F00
:106D80004FEA4B0BB7DC6269D08A4FF6FF7188423D
:106D900048D0934223D0A06990F88020023A012A7B
:106DA00006D80022591DFFF7FBFB2046FEF730FFF7
:106DB000638C94F82120B4F9241020485A434FF4EE
:106DC0007A7353436269049305320123039301925A
:106DD0001023002200920293174AFBF7F9FAA369E5
:106DE0006069D3F8843000215B689847069B208552
:106DF000834203D004F1300005F04EFB606978B1A6
:106E0000A369228DB3F88810C38AB2FBF1F2B3FBF9
:106E1000F1F39A42056801D8FFF7B4FE2846EEE781
:106E200063692BB9204609B0BDE8F04FFFF716BFE4
:106E300009B0BDE8F08F00BFAE130108A810002014
:106E4000334BB3F900302DE9F34106460C461546A5
:106E50000BB9002058E0002301930B78FF2B0BD1D6
:106E60004B7803F00F030E2BF3D121466846FCF755
:106E70003FFB074608BBECE708222649204607F0FF
:106E800097FDA0B12378FF2B04D1637803F00F03A3
:106E9000022B0CD010222049204607F089FD30B18A
:106EA00010221E49204607F083FD0028DDD12378FB
:106EB0000433DBB2012BD8D9CBE7DDF80080B8F181
:106EC000000FC6D001A93046FFF798FD0028C0D0BA
:106ED0000020019EFFF778FDC6F8840001984FF46A
:106EE0008073A0F888300023A0F88A30214680F80B
:106EF000805043463A46FFF7B1FD0446019814B965
:106F0000FFF79BFEA5E7006202B0BDE8F08100BF7D
:106F1000BA3700205E130108AE130108BE13010842
:106F2000022380F82A3000218069FEF7A3BF0023E6
:106F300080F82A30303005F0AFBA70B500249C429A
:106F40002ED21578082D25D8DFE805F00524242455
:106F5000091319240E000134A4B20132EFE701280D
:106F600022D155780E2D14E001281DD155781E2D03
:106F70000FE0022818D15578122D0BD914E0022801
:106F800012D191F880505678012D14BF0425142594
:106F9000AE4209D1557802352C44A4B22A44CEE73A
:106FA0000CBF0120002070BD002070BD704711B9DA
:106FB00070B1C18A00E020B183699B69B3F8880091
:106FC00001E04FF480700844814201DC80B27047D8
:106FD0004FF6FF707047C28ACB8A9A4203D38CBFA8
:106FE0000120002070474FF0FF30704738B504464D
:106FF000FFF7F1FF0028CCBF0846204638BD704798
:10700000004870476C0200200021FEF7AFBB000073
:107010002DE9F0419EB0102200210AA807F0F8FDEA
:10702000804B0B93804B08211B88ADF834300EA8A1
:10703000FBF750F80AA90120FEF7AAF840F2052351
:10704000ADF81A3040F2032440F2012504A8FBF702
:107050003EF8BDF81230B3F5017F09D8A34280F0A5
:10706000D880AB420CD040F2022293426ED0EDE7C2
:1070700040F225229342E9D1059800F0EDF9E1E7CD
:10708000059D2846FEF780FB044600287ED001219E
:10709000FEF7F7F8054608B1C3681BB92046FFF7AD
:1070A000B3FFCFE783681B78412B11D1FEF76CFB50
:1070B00005460028F2D001221146FEF77FFA01466C
:1070C0000028EBD02046FEF711F90223044631E0F8
:1070D00003F0D802C02A03D1204600F0B1FAB1E78C
:1070E00003F0E003602BD9D10021022328220846B7
:1070F000FEF74AFA089010B9089890B9CEE703ABAA
:107100000093002321461A4608A800F0DFFC014640
:107110000028F1D001222046FEF750FA014618B9A6
:107120000898FFF771FFB9E72046089AFEF7F4F8D0
:10713000002304462B7440F20122234639490220E1
:10714000FDF772FD00287FF47DAFA7E7059DEDB147
:10715000EB68072B1AD96B68C3B193F91030022B77
:1071600014D12846FEF710FB044678B18768B7F9BA
:10717000020001F095FE61688046002619B1CB68D7
:1071800049681E44FAE7B8F1000F01D1284686E7A6
:1071900098F8043023B1204600F086FF70B97DE7EF
:1071A00001231A460846FEF7EFF900283FF476AFB0
:1071B000636843606060836841221A7062680023DC
:1071C0001AB1D16852680B44FAE7B8F80210994234
:1071D00008D32146B7F90200FDF75FFD00283FF70D
:1071E00031AF5BE7114B596800297FF457AFB6F513
:1071F000006FBFF453AF79889A8108A840F2252226
:1072000019805C609E60ADF822200993FAF77EFE3B
:1072100018E76FF0850306A904A80793FAF726FF7D
:1072200010E700BF0000FFFF04030020D43D002052
:107230001FB50A4CB4F9000000280DDC084B02937E
:1072400000230193074B0093032208234FF480612E
:107250000548F9F769FD208004B010BDE441002025
:107260002013010811700008E43D002038B50E4BD2
:10727000142404FB00340546638A63B10020FAF746
:1072800081FA0A4BB0FBF3F0094B53F825308342E7
:1072900006D800236382637C23F01003637438BD37
:1072A0001B1A638238BD00BFE641002000879303AC
:1072B000284300202DE9F041012180461048114D5E
:1072C000FAF7ECFC002426462746E0B2FFF7CEFF93
:1072D0002B7C53B14146284602F0ACF82B7C83420C
:1072E00003D8B84284BF2E4607460134102C05F15E
:1072F0001405EAD10248FAF701FD3046BDE8F081F5
:1073000068430020E64100200F2838B5044615D810
:1073100001210B48FAF7C2FC2046FFF7A7FF094BF3
:10732000142000FB043506482C7C1CB1FAF7E6FC5F
:10733000284638BDFAF7E2FC204638BD002038BDAB
:1073400068430020E64100202DE9F8430F28064657
:10735000884615461F469DF820903FD8002A40D009
:1073600001212148214CFAF799FC002F4FF014031A
:1073700003FB064308BF4FF00009802D88BF802221
:107380005F828CBF1A741D74B9F1000F02D046F0F1
:10739000100300E03346142000FB064441466374AA
:1073A000204602F032F8014640B91022204607F08C
:1073B0002FFC227C4146204602F062F80020FAF7BA
:1073C000E1F90B4BB0FBF3F00A4B0744064843F8D6
:1073D0002670FAF793FC2046BDE8F8830020BDE84C
:1073E000F8831046BDE8F88368430020E64100209A
:1073F00000879303284300200021FEF7B7B9F8B5B2
:107400000E4601784378174601F10802024405460A
:107410000830FDF787FE0446E0B18368B5F9022025
:107420005A802A791A716A795A71AA799A71B7427F
:107430004FF000013A464FF0010328BF324608469C
:10744000FEF7A2F8054620B92046FFF7D5FF2846EB
:10745000F8BD60602046F8BD2DE9F04F054685B0C7
:10746000B0F9000001F01CFDD5F80480D8F8044004
:1074700083464FF0000A1CB1E36864689A44FAE757
:10748000BBF1000F05D14046FFF7B6FFC5F804B0C9
:10749000D0E0B5F80C90B9F1000F42D1674FAE685B
:1074A0003B88D8F8080001333B80CAEB06039AB248
:1074B000BBF80230043B134403F0F8039B1A1FFA95
:1074C00083F909F104025146FFF799FF03460028AA
:1074D0003AD04268D2F808A076BAAAF800609AF8C2
:1074E000002062F03F028AF800203A8852BAAAF8D7
:1074F0000220D8F80470002F7CD0FA68B968009395
:10750000C4EB0906964228BF1646201D3444324675
:107510005044A4B207F07EFAA145009B6AD97F6867
:10752000E9E7D14580F08280BBF80260D8F8080016
:10753000AF68053E06F0F806C9F10501721D514419
:10754000FFF75DFF034628B96868FFF755FF002382
:107550006B606FE042689268511D009179BA1180AA
:10756000117861F01F01117034494F440988CAEB4A
:10757000070A49BA4FEADA0A518082F804A0D8F81B
:107580000470FFB1A1451BD0FA68A11889B28945E2
:1075900013D2C4EB09041FFA84F9C9EB0204B44204
:1075A000B9680098019328BF34462246494407F041
:1075B00031FAA4B27F68019B05E07F680C46E0E7E2
:1075C000002400E03C46A64214D99FB1FA6801931A
:1075D000C4EB06089045009BB96828BF904618196F
:1075E00044444246A4B207F015FAA642019B01D0DA
:1075F0007F68EAE71946BBF900000093FDF74DFBF1
:107600000028009B02DC1846FFF7F6FE002C9BD0FA
:10761000AB8903951C44AC8140F2252302A8ADF848
:107620000A30FAF773FCF9F745FB03E04046FFF731
:10763000E3FE6C6005B0BDE8F08F00BF6C43002036
:1076400010B58268137803F0F803C02B044606D007
:10765000E02B0DD11379C268DB00053A02E0C26865
:107660000023043A60682146806800F013F8204641
:10767000BDE81040FFF7C0BE002203682BB11968B7
:107680009A80DA801A600160F7E743607047002152
:10769000FEF76CB82DE9F04F8FB08146002092467E
:1076A00004911F468E68AA4DFAF76CF8A94A8346E2
:1076B00005F190082C46606858B1A368C3EB0B0332
:1076C000934206D90292FFF7E2FF2046FFF7D4FF6C
:1076D000029A24344445EED199F800B009F1080328
:1076E00007930BF108034B44069399F8013002937A
:1076F00033885BBAC3F30A03059373885BBAADF8AA
:10770000263000209BB20A93FAF73CF80023089039
:107710001C4603936A68A846002A00F02581D268B7
:107720000599914223D1EA8B0A998A421FD12A7F77
:1077300093451CD16A7F0299914218D15A46079904
:107740000B9305F10C0007F033F90B9B78B9029A03
:10775000069905F1140007F02BF90B9B38B97C4C06
:10776000039A242303FB0244089BA3604EE014B950
:107770006A6802B92C463BB1A9689A68521A7649E0
:107780008A4294BFA8469846039B0133042B039377
:1077900005F1240501D04346BCE784B9B8F1000FD8
:1077A00003D16E490320F9F71FFAD8F80400002826
:1077B000F7D0FFF76CFF4046FFF75EFF444600211D
:1077C0000223059A0846FDF7DFFE6060002800F0FE
:1077D000DD80836800210020C3E90001089BA360CD
:1077E0005A46079904F10C0007F014F9029A069919
:1077F00004F1140007F00EF99DF808306377BDF826
:107800002630E383002384F81CB0238425680FBB53
:107810003379412B03D105360AF1FF331FE003F022
:10782000E003602B06F1040618D10EAB204643F8A6
:10783000047D50F8042F0093D2680499042300F0CB
:1078400045F900287CD00D9A28320AEB0203064441
:107850001B1A05E005365346002201E053463A461E
:107860006068C16803EB070E8E456AD81FFA87FE71
:107870000EF1FF31194489B26DB1B5F8048041456C
:10788000C0F08280B5F806C0E6457DD8C6456FD108
:1078900061456DD178E01FFA83F80EF1FF31414464
:1078A000DFF8C0A089B2AC460AEBCC05B5F806B04B
:1078B000BBF1000F11D1ADB1E98021682960A5F8B5
:1078C00004E0218C256080684144174421849A1A81
:1078D0003146384407F09EF804E00CF1010CBCF18D
:1078E000340FE1D16368228CDB689A424ED1637F0A
:1078F000217F04F1140204F10C00FDF713FCF8B130
:107900008368B9F902205A8099F804201A7199F80D
:1079100006209A7199F805205A7100234360636824
:107920002BB15A680AB11346FBE7586000E060606B
:1079300063680B4940F201220220FDF775F910B986
:107940006068FFF7A4FE2046FFF796FE1EE000BF2A
:1079500070430020C0C62D00FEFFFF7FE50901082F
:107960000000FFFF00440020002C7FF404AF01E77B
:10797000FFF78DFE2046FFF77FFE3B4652460499F7
:107980004846FFF787FE01E02D6875E70FB0BDE8B8
:10799000F08F00BF037823F00F0343EA1113037045
:1079A000437803F00F0343EA011141707047000070
:1079B0000822014907F02EB85E13010810220021A9
:1079C00007F026B910B508220949044606F0F0FF71
:1079D00048B12378FF2B08D1607800F00F00831E98
:1079E0005842584110BD012010BD002010BD00BFFD
:1079F0005E13010873B51546194A04460E46106811
:107A000051686B4603C32CB3637CDB0624D4227C11
:107A1000802A1DD0402A1FD9D208D11F501C2944CA
:107A2000C2F10F02304406F0C3FFA8B9237CD90885
:107A30000D44725C15F8080C03F0070302A90B440F
:107A4000424013F8083C1A420CBF0120002004E019
:107A5000012002E0204600E0002002B070BD00BF1F
:107A6000241301080023042A10B54370037016D0B4
:107A7000082A02D0022A26D118E00B7883F00203EC
:107A800003704B7843708B788370CB78C3700B791D
:107A900003714B7943718B798371CB7911E00B784A
:107AA00083F0020303704B7843700223FF2400220B
:107AB000C470FE24827004714271CA5C82710B44EE
:107AC0005B78C37110BD184610BD00002DE9F74F5B
:107AD0001E464B6800920F46D3F808A0D1F808B0B4
:107AE000019018B9C0490320F9F77EF8019B1B6883
:107AF000002BF7D0DA68272AF4D90BEB06089D682B
:107B000098F90130002B2B7803F00F0343F060034A
:107B10002B701BF8063003F01803ACBF02240324BB
:107B2000082B27D017D8002B52D118F8041028465C
:107B3000FFF730FF08EB04014B7803F00F026B787E
:107B400013436B708978AA78E31C0A43AA7018F86B
:107B50000320043429E0102B2AD0182B38D100211F
:107B60002846FFF717FF6B7823F00F036B70002395
:107B7000AB702CE018F804309B099B0043F06003C5
:107B80002B706B7803F00F01697018F8043003F064
:107B90000F0308EB04020B436B705178AA78A31C07
:107BA0000A43AA7018F803200334EB7813430EE05D
:107BB00018F804102846621CFFF7ECFE6B7823F0DF
:107BC0000F036B700023AB70EB70144600E0EB709A
:107BD0001BF806305B075CBF18F80430AB711BF86C
:107BE000063003F0030358BF0134022B08D0032BE7
:107BF00008D0012B07D018F80430EB71013403E0F2
:107C0000402300E0FF23EB7198F8013003F04002BD
:107C100002F0FF0972B118064ABF98F8020000206E
:107C2000000913F0300905D0FFF76EFB81460028EC
:107C300000F0318298F8013003F07003302B42D00D
:107C40000FD8102B1CD0202B26D0002B40F08C807E
:107C500008EB0401102205F1080006F0DBFE1034E9
:107C600082E0502B3BD006D8402B7DD105F1080097
:107C7000FFF7A4FE78E0602B45D0702B62D073E054
:107C800005F10800FFF794FE082208EB040105F156
:107C9000100006F0BFFE34E005F10800FFF788FE93
:107CA0004FF0FF320023EA746FF001022A752B7443
:107CB0006B74AB746B75022208EB040105F11600BE
:107CC00006F0A8FE3CE0514605F1100011F8082B23
:107CD000FFF7C8FE05F10800FFF76AFE44E0B9F1BE
:107CE000000F3FF4FFAE082208EB040105F110007D
:107CF00006F090FE99F81020494605F1080001F0C1
:107D0000BFFB083430E0B9F1000F3FF4EBAE4FF0A9
:107D1000FF320023EA746FF001022A7508EB0401B8
:107D200002222B746B74AB746B7505F1160006F0B0
:107D300071FE99F81020494605F1080001F0A0FBFA
:107D4000023411E0B9F1000F3FF4CCAE514605F119
:107D5000100011F8082BFFF785FE99F8102049460E
:107D600005F1080001F08CFB98F8013059070FD598
:107D70001A064ABF98F80200002000F00F0013F026
:107D80000B0F05D0FFF7C0FA8146002800F0838171
:107D900098F8013003F00F030C2B00F27C81DFE830
:107DA00013F00D001600250042007A015100610019
:107DB00082000D009400A600B800C60008EB040184
:107DC000102205F1180006F025FE1034D9E005F167
:107DD0001800FFF7EDFD082208EB040105F1200073
:107DE00006F018FE3CE000BFE509010805F11800A7
:107DF000FFF7DEFD4FF0FF32002385F823206FF000
:107E0000010285F8242085F8203085F8213085F896
:107E1000223085F82530022208EB040105F1260006
:107E200006F0F8FD3DE09AF800109AF801200831BC
:107E3000514405F12000FFF715FE05F11800FFF78A
:107E4000B7FD9EE0082208EB040105F1200006F0D2
:107E5000E1FD99F81020494605F1180001F010FBEA
:107E600008348EE04FF0FF32002385F823206FF0B6
:107E7000010285F8242008EB0401022285F8203055
:107E800085F8213085F8223085F8253005F1260067
:107E900006F0C0FD99F81020494605F1180001F0E0
:107EA000EFFA02346DE09AF800109AF801200831D8
:107EB000514405F12000FFF7D5FD99F810204946FF
:107EC00005F1180001F0DCFA5BE005F11800FFF79E
:107ED00075FDFF232B7618F804306B76611C0522A4
:107EE000414405F1230006F095FD063449E005F113
:107EF0001800FFF763FDFF232B7618F804306B762C
:107F0000611C0322414405F1250006F083FD043481
:107F100037E005F11800FFF751FDFF232B76022310
:107F20006B7618F8043085F82730013429E005F124
:107F3000180099F810A0FFF741FD99F81030402B78
:107F400084BF402389F81030FF232B7618F80430C3
:107F50006B7608EB040349465B78AB7699F81030F2
:107F6000EB7699F8102005F1580001F089FA211DEF
:107F70000422414405F1240006F04CFD063489F842
:107F800010A0009B13B9FB681B1B01E0009B283B62
:107F90005BBAAB801BF806305B077ED518F804305F
:107FA00003F0F803F02B78D1019BBD68D3F800A053
:107FB000009BDAF80890344404F1010815F804B085
:107FC0004BB90099042308220846FDF7DDFA002882
:107FD00065D0826802E009F1280200200BF003035B
:107FE000022B14D0032B1FD015F808101170012B91
:107FF00005EB04039978517004D0D9789170053459
:108000001B790FE0DB780434A3F5805318E015F8F2
:108010000830A3F580535BBA13802B190434997888
:108020009170DB78D3700DE015F808301909A1F5CF
:10803000756149BA03F00F0302341180A3F575632B
:108040005BBA53801BF0040F03D00021FDF78EFBB9
:1080500025E02B5D9371A31C2C446178D17118B17C
:10806000F9680831C91A01E00099283949BA9180A4
:10807000112189F806109288A9F8042018B1019AF4
:10808000C0F804A0106053B19C1B0C9B0C9A1B6899
:108090000833136001E0002003E0204601E00024E3
:1080A000F3E703B0BDE8F08F2DE9F04F4268D0F858
:1080B00008909668D268002189B08246012308465C
:1080C000FDF762FA029038B38568AB4960232B70E4
:1080D00006F1080B00236B701022584606F068FC6E
:1080E00038B15846FFF7E6F8804610B1437CD90610
:1080F00001D44FF00008337EFF2B00F0628206F1BE
:108100001800FFF7D7F80746002800F05A82437C92
:10811000DA0640F1568201E0029858E2B8F1000F09
:1081200004D098F811301B0703D15FB17B7C1C078A
:1081300008D06B7863F07F036B700023AB7003246F
:1081400001E04746022431683378727821F47041A7
:1081500021F0FF011B01A9B943EA121313F0FF0F2D
:108160002B7803D143F018032B7036E043F0100353
:108170002B70737831781B09621C43EA01132B556D
:1081800094B22AE05BB203F030011209114304F10A
:1081900001010ED12B7843F008032B7032688BB2AB
:1081A000317812BA8910C2F3034242EA81122A5589
:1081B00009E013432B55326889B212BAC2F3034265
:1081C000A31C6A549BB2326812BA120AEA549C1C6D
:1081D00001339BB20022EA54A4B2B379112B6DD1C2
:1081E000DAF80430586883681A88B3F802E052BAA3
:1081F00092B222F00F0C1FFA8CFC4FF2B0018C45AA
:108200001AD19EFA9EF121F00F010904090C614573
:1082100012D10322B271598849BA1FFA81FE198816
:1082200049BA89B20EEB011101F5AA611970997969
:108230005970D979997026E09EFA9EFE0EF47F4E11
:10824000BEF5704F04D10122B2715A8852BA0CE0C7
:1082500002F47F42B2F5704F0ED10222B2711A8839
:1082600052BA1A709A785A70DA789A709A79DA70E3
:10827000DA791A71052206E00022B2719A791A7130
:10828000DA795A710622B17961F00F01C2F1080E54
:10829000B1711A44C168C3EB020CCEEB01018C45ED
:1082A00004D212F80E1002F8011BF3E7FDF7F4F9FF
:1082B0002B7843F004032B70012303E0621C2B5541
:1082C00094B200230393F379402B07D0FF2B0AD0FD
:1082D000012B0CD12B7843F0010302E02B7843F003
:1082E00002032B7006E02B7843F00303F9E7621CCE
:1082F0002B5594B210222049584606F059FB18B964
:108300006B7843F0400335E0B8F1000F0CD06B7888
:1083100043F040036B7098F8112010070AD0AB7837
:1083200043EA0213AB7005E05846FFF74BFB002809
:1083300000F0408108AB0020002163E9040199F8B6
:108340000020082A00F224814FF48A71D140C90725
:1083500040F11E8109F108011846FFF783FBDDE9B2
:10836000042371693069994208BF904206D16B7845
:1083700043F030036B7021E0AE13010804AA5946A4
:108380004046FFF737FB0028F1D13369B3F17F4F47
:1083900005EB04006B7840F00381B28A52BA92B2C6
:1083A000B2F57E4F40F0FC8043F020036B70022258
:1083B00006F1160106F02EFB0234A4B2337EFF2B29
:1083C00072D16B7843F008026A70728BCABBF26993
:1083D000BABB328CAABB727E022A0FD1326A6AB94A
:1083E000B28C5AB996F8262042B943F00B036B7051
:1083F00096F827202A55631C9CB2B4E0728C8AB987
:1084000096F8242072B943F00A036B70737E2B55E3
:10841000601C032206F1250115FA80F006F0FAFA35
:1084200004349FE096F82220002A40F0948043F024
:1084300009036B70737E2B55601C052206F1230126
:108440002CE0B38BADF81030F38BADF81230338CD9
:10845000ADF81430738CADF8163004A8FEF72AFF7F
:10846000002878D0437CDB0675D5027CF37E9A42E7
:1084700071D16B7843F004036B70437C13F00F03EE
:108480001EBFAA781343AB70737E2B55631C9BB23F
:10849000B27EEA54A01C042206F1240115FA80F0F1
:1084A00006F0B8FA06345DE01FB199F801303BB927
:1084B00051E006F11800FFF785FA0028F5D14AE0EF
:1084C00057B16B7843F004036B707B7C13F00F03A0
:1084D0001EBFAA781343AB7099F8001099F80120D9
:1084E0000831494404A8FFF7BDFADDE90423716AA5
:1084F000306A994208BF904204D16B7843F003037D
:108500006B7030E004AA06F118013846FFF772FAE2
:108510000028F2D1336AB3F17F4F05EB04006B788A
:108520000FD1B28C52BA92B2B2F57E4F09D143F05C
:1085300002036B70022206F1260106F06BFA023488
:1085400010E043F001036B70082206F1200106F0F1
:1085500061FA083406E02819102206F1180106F025
:1085600059FA1034A4B2039B1BB1631CB2792A558B
:108570009CB221460298FDF78FF8DAF804105046B5
:10858000FCF7B4FE029A43685360426001201EE08B
:108590000821B9F9020000910022FCF799FBDEE600
:1085A00043F010036B70082206F1100106F032FA56
:1085B000083402E728191022594606F02BFA103425
:1085C000FBE6B8F1000F3FF4BCAD0027A9E509B008
:1085D000BDE8F08F10B508220949044606F0E8F915
:1085E00048B12378FF2B08D1607800F00F00831E7C
:1085F0005842584110BD012010BD002010BD00BFE1
:108600005E130108F8B5B0F8C631DB07044603D4A1
:1086100015490320F8F7E8FA00F5E0760121002576
:1086200004F5EE773046F9F739FB384684F8CB513C
:10863000F8F756FA4FF40873A4F8F2310B4B0C49D3
:10864000B3F90030C4F8F44104F5F872384604F088
:10865000E5F83046F9F752FB2946B4F9C401BDE804
:10866000F840FCF741B800BFE5090108DC10002024
:1086700080969800F8B5B0F8C631DB07044603D4FD
:1086800024490320F8F7B0FA00F5E07601213046DE
:10869000F9F704FB94F8CB31022B03D8013384F8AB
:1086A000CB3116E0DD1E01F0CBF80123AB403B2BB4
:1086B000B0FBF3F505FB13009EBF94F8CB310133FB
:1086C00084F8CB31092804D93C2828BF3C20054632
:1086D00000E00A2504F5EE773846F8F701FA4FF482
:1086E0000873A4F8F2310C490C4BC4F8F441694307
:1086F000B3F9003004F5F872384604F08FF83046CC
:10870000F9F7FCFAB4F9C4010021BDE8F840FBF721
:10871000EBBF00BFE509010840420F00DC1000205C
:1087200010B50446B0F91A00FAF764FEB0F8C63185
:10873000DA0703D410490320F8F756FA637E1B07C3
:108740000BD4002005F052FAA8B9B4F91A00FAF7D0
:1087500051FEBDE81040FFF755BF102207492046E3
:1087600006F026F90028ECD02146B4F91A00BDE83D
:108770001040FBF7B9BF10BDE5090108AE130108B1
:108780002DE9F04380468DB01846894614461F46B1
:10879000FFF720FF0546B8B910230693029308AEF1
:1087A00007AB079003900093019706AB32460DF19B
:1087B00016014748F9F717FF002806DB069B102B28
:1087C0000CBF3546002500E000253946204605F05F
:1087D000C3F90646002D74D030B93946BDF91600EC
:1087E00005F0BAF90646E0B1B6F91A00FAF702FE4A
:1087F00018B1B0F8C631DA0706D5737E03F030033E
:10880000302B08BF3D4600E03D4645B93846FFF7EE
:10881000E1FE002851D03D46002D3CD00EB1AF42C4
:1088200004D02946204605F097F906462846FFF76A
:10883000D1FE58B326B1737E03F03003202B25D12F
:1088400007AE3046FCF758FC0822074689F800209E
:10885000A918404606F0DEF898F8003083F00203CD
:1088600088F80030CCB9BC4215D036F91400FAF7BC
:10887000C1FD48B1B0F8C631DB0705D50CAB03EB41
:10888000440434F9140C1FE00134ECE7737E03F068
:108890003002202A03D1002016E0204614E003F025
:1088A0000703032B03D104213046FBF7BDFE3246FC
:1088B0004946404605F0D0F906E0FBF7A1FD054624
:1088C000AAE70028A2D08FE70DB0BDE8F08300BF73
:1088D000A810002070B50E4618B911490320F8F70A
:1088E00083F90029F9D0B0F91A00FAF783FD00F5F1
:1088F000EE7504462846F8F7F3F84FF40873A4F829
:10890000F2310849084BC4F8F44104F5F872714398
:108910002846B3F90030BDE8704003F07FBF00BFC8
:10892000E509010840420F00DC100020F8B50746B9
:108930000D46164610211A462120FBF730FC04464E
:1089400060B1806800236DBA08228770437103719B
:10895000C370C5803146104406F05CF82046F8BD6F
:108960002DE9F04F85B080460E9E7578022D0F469A
:1089700092461C4640F0B8800823009300226B44C6
:108980000321FCF7A5F90028C0F2AE804046FAF7B3
:1089900031FD21468146404605F0DEF8BAF1870FE9
:1089A00004464ED0BAF1880F40F09E80B9F8C63127
:1089B000D90740F19980DDE90223D6F80CB0D6F84A
:1089C00008A05B4508BF524540F08E80002800F0AB
:1089D0008B80B578012D2ED00BD3022D40F08480F2
:1089E000404607F1080105F0DFF84846FFF70AFEA8
:1089F0007AE009F5E07901214846F9F74FF9F68860
:108A00003D4B04F13807384676BAB3F90080B6B268
:108A1000F8F766F8394940F21223013EA4F84E30C7
:108A20003846434604F14C02714303F0F7FE4846D2
:108A3000F9F764F95BE007F118014046FAF720FD09
:108A400052E0B9F8C6319A074ED0B378002B4BD11B
:108A5000083710222A49384605F0AAFF002843D0DB
:108A6000D4B1637E9B060CD5D4F88C20D4F890301A
:108A700052EA030105D0F168B0688B4208BF824218
:108A800034D1B6F80690B9F1000F05D13946404609
:108A900005F08AF84D462AE0F3882BB384B9032306
:108AA00000930F9A109B3946404604F0E7FF0446B6
:108AB000E8B1324600F18C0352F8080F516803C345
:108AC000637E0E4823F0300343F030036376F18871
:108AD000094B49BA89B24143B3F9003004F1840229
:108AE00004F1700003F09AFE002500E001252846FD
:108AF00005B0BDE8F08F00BFDC10002000879303B5
:108B0000AE13010813B58A784B78402A01D8022B9E
:108B100000E0032B0ED186280ED1C878CB88C0F395
:108B200000145BBA00949BB2083100F00F00FEF70E
:108B30000BFC01E0002000E0012002B010BD0000AD
:108B400008B50146074800F060FC48B91022064904
:108B5000044805F02DFF0028024818BF002008BD7A
:108B6000004808BDA0450020AE13010838B50446F2
:108B7000E1B1012380221449B0F9C401FAF758FC8D
:108B8000A0B104F5E07528460121F9F787F8B4F89B
:108B9000C63143F00403A4F8C6314FF4E163A4F8EE
:108BA000CC312846BDE83840F9F7A8B8B4F8C6314A
:108BB000B4F9C401044923F00403A4F8C631BDE8A4
:108BC0003840FAF75DBC00BF8E13010808B51022CB
:108BD0000449054805F0ECFE0028034808BF0020C2
:108BE00008BD00BFAE130108A04500202DE9F047E5
:108BF0000024054600F116074FF00109A2464FEA8E
:108C0000D40804F0070617F8083009FA06F63342CC
:108C10000AD0E0B2FEF778FB80F810A017F8083011
:108C200023EA060607F808600134102CE7D1002675
:108C3000AC695CB12368AB616368A168B3F9C40136
:108C4000FAF71EFC26606660A660F1E71022214656
:108C5000284605F0DDFF2C61BDE8F0872DE9F04FD7
:108C600087B003F1080A02905046039117461E464A
:108C7000FFF766FF0446002800F0B480F3885BBA73
:108C80009AB21AB942F210738382ABE0DFF86091B6
:108C90008382103F4FF00008002F70DD08F11003B1
:108CA000039AD518D35C032B02D0222B4AD05EE066
:108CB0000298FAF79FFB6B780190042B42D105F1E3
:108CC000100B08224949584605F072FE002839D099
:108CD0002A7CFF2A04D16A7C02F00F02022A31D0DA
:108CE000EA7851062ED413062CD46A6852B359463A
:108CF0000298FAF737FCAA7804905946D9F8080088
:108D0000059200F097FB059A824209D8D9F80830FD
:108D10005B7C9A4204D1D9F80430019A9A4207D078
:108D2000334B986820B11022324905F041FE48B912
:108D30002F4B5A6832B9019A5A60049A9A60A26914
:108D40001A60A361AB783F2B6B7801D8022B00E04F
:108D5000032B0CD1EA7804F11603C2F3C001012001
:108D600002F0070200FA02F2585C02435A546B7890
:108D700008EBC3081FFA88F8A7EBC3078CE77388D2
:108D80005BBA9BB22361B28852BA43EA02432361C1
:108D9000DAF80000DAF80410234603C356F8100F7F
:108DA0007168022203C3002104F1160005F030FFB0
:108DB0000023A361A58A104B04F11C0630465D43D5
:108DC000F7F78EFE40F2232363860C4B6463B3F9FE
:108DD000003004F130022946304607B0BDE8F04FBC
:108DE00003F01CBD07B0BDE8F08F00BF5E130108A3
:108DF000D8450020AE13010800879303DC10002043
:108E00002DE9F0418846C108064614460831069A05
:108E100022201F46FBF7C3F90546A0B18068002158
:108E200064BA01714171C480867080F80380EA6879
:108E300000F10804083A204605F0EAFE32463946B9
:108E4000204600F01DFB2846BDE8F08170B50546C0
:108E50000E46144618211A462320FBF7A0F980B1CC
:108E600083686ABA2D0C6DBA76BA5A809D80DE800E
:108E700022689A606268DA6054F8082F1A616268A2
:108E80005A6170BD054BB3F90020904204D01AB965
:108E90000122188059801A71704700BFE4450020F4
:108EA000034BB3F9002082420CBF184600207047E4
:108EB000E44500200021FCF759BCF8B50746848939
:108EC0000E46154600204DB900230822B96800F06F
:108ED00075FA96F91030022B25D10DE0BD42F3D082
:108EE000B542F1D02346AA89A96800F067FAEB6879
:108EF0006D681C44A4B2E6E702194FF6EE739A427D
:108F0000C4BF013080B2B168113420440023202254
:108F1000083180B200F052FA4FF6FF73984203D046
:108F2000C04380B2F8BD0020F8BD000070B510222B
:108F300098B000210DEB020005F06AFE4D4B059341
:108F40004D4B1B88ADF81C3040F20523ADF80A30BC
:108F500008216FF0850308A80393F9F7BBF804A96B
:108F60000420FCF715F96846F9F7B1F8BDF80230AE
:108F70006FF400721344032BF5D8DFE803F0023BD3
:108F80007575019D2846FCF7FFFB044608B9284685
:108F900067E00221FCF775F9064618B93749032046
:108FA000F7F722FE606830B190F91030042B02D13F
:108FB000C368082B06D0042208212046FCF7FEFADD
:108FC00000284DD0002385682374EB885BBA9BB2E0
:108FD000002B45D022463146FFF76FFF4FF6FF7357
:108FE00098423DD1698849BA234640F2012289B2AC
:108FF000042031E0019E304696F91050FCF7C4FB86
:10900000044608B930462CE0406826460028C5D002
:1090100090F91030042B07D0FCF7B6FB0346F8B1EB
:10902000706040681E46F1E7FCF7AEFBC0B1826895
:1090300070600023C16840680B440028FAD15BBA15
:1090400093806B1C08BF63680A4908BF93F91050EE
:1090500040F2022223462846FBF7E6FD002882D193
:109060002046FFF727FF7EE702A96846F8F7FEFFD4
:1090700079E700BF0000FFFF04030020E5090108B5
:1090800010B5044668B161B190F91030042B0BD1D2
:109090004268FFF712FF50B1A36840BAD8800020A1
:1090A00010BD6FF00D0010BD6FF04C0010BD6FF0E3
:1090B000010010BD38B50D461446042308220021D6
:1090C000FCF762FA38B1836800226DBA64BA1D8079
:1090D0005C809A71DA7138BD1FB50A4CB4F9003062
:1090E00063B9094A0193094B0292009305220823B0
:1090F0004FF480610648F7F717FE2080B4F90000AE
:1091000004B010BDEA490020030D01082D8F0008AE
:10911000EA45002010B5044601784278054805F07C
:109120007FFE6188044849BA89B2BDE8104005F065
:1091300077BE00BF2C13010849130108F8B5044697
:109140009DF8245025701E4605F0070310250F4694
:10915000657006989DF8281015460AB1002F68D052
:1091600018B1002E69D13046F8BD23B1022B02D0D0
:109170000DB9002873D0A17080B39DF82030E37042
:1091800002289DF82130237104D0082816D0002829
:1091900051D120E002463249304605F009FC18B9A9
:1091A000237823F020032370637843F0080363706F
:1091B000737863713378A371072040E01C236370D8
:1091C000221D06F1080313F8011D02F8011F9E423B
:1091D000F9D10D2033E005201DB9F8BD0320002D85
:1091E0003DD0431C9DF81C2022549DF81D20E254C4
:1091F0000230022D03D0082D0CD0E5B9F8BD6378FC
:1092000063F07F0363707A782254431C3A78E25407
:109210000230F8BD637863F03F03637007F1080321
:10922000044413F8012D04F8012BBB42F9D1083096
:10923000F8BD3846F8BD0020F8BD63B90DE075B142
:10924000BDF81C20BDF820309A42CAD1237843F0E3
:1092500040032370CDE7022B8AD1A1708DE7F8BDC2
:109260005C130108427802F00C03082B07D00C2B8A
:1092700007D0CBB90178490614D4032302E00723B1
:1092800000E00D2312F0C0020CD00178490658BF4F
:109290000233802A01D1981C7047C02A04D103F1FF
:1092A00008007047184670470020704770B501B13C
:1092B0001AB926490320F7F797FC437803F00C030B
:1092C000082B07D103785C0617D5C3781370037990
:1092D000537012E00C2B07D103785B060FD5C378CF
:1092E0001370037953700AE013B16FF0150070BD6D
:1092F00003785E06F9D4032302E0072300E00D2380
:10930000447814F0C00411D005786D0605D4C65C0D
:1093100016705D1C0233455D5570802C08D1C25C0F
:109320004A70034402205B780B7070BD204670BD0C
:10933000C02CDAD1034401F1080213F8010B02F842
:10934000010D8A42F9D1082070BD00BFE50901086E
:1093500008B501B11AB918490320F7F745FC43785D
:1093600003F00C03082B09D1C378137003795370F1
:1093700043794B7083790B70022008BD0C2B0ED102
:10938000C378137010F8043F537001F1080310F80C
:10939000012F03F8012D8B42F9D1082008BD3BB9FC
:1093A000037813F0400F14BF6FF01500002008BDC4
:1093B0006FF0150008BD00BFE5090108F0B51AB34C
:1093C000DC0705D511F8014B013A204492B2013374
:1093D000570801EB47054C1C03350234AC4207D05B
:1093E00014F803EC14F8026C06EB0E263044F4E794
:1093F0001A44D30703D511F8173000EB0320030CF0
:1094000080B201D01844FAE7F0BD30B54B6845682A
:1094100004680A689D4208BF944209D1C568CB68B8
:1094200084688A689D4206BF94420120002030BDB6
:10943000002030BD30B510B3E1B188421CD00138F6
:109440000139002210F8015F11F8014FA54202F125
:10945000080303D1DAB2802AF4D10FE085EA0401CF
:10946000D8B20B060AD40132D2B249008242C9B244
:10947000F7D130BD084630BD802030BD104630BD2C
:10948000802A28BF8022F8B5D50814462A46064609
:109490000F4605F0BFFA63070ED0A4EBC504725D5A
:1094A000FF23C4F1080403FA04F422EA040272550B
:1094B0007B5D1C4014437455F8BD10F8013F43B167
:1094C0008B42FAD100230370437813B1013004F0CA
:1094D000F7BF1046704700002DE9F04707468AB0F5
:1094E00008B90020A8E00029FBD000204FF0FF348D
:1094F00006462346054631F810E0BEF1000F07D1BD
:10950000B3F1FF3F13BF013503B201252DB20BE0CC
:10951000B3F1FF3F08D0B4F1FF3F01D0B54201DD08
:109520002E461C464FF0FF3301300828E3D1581C6B
:1095300004D0601C7DD0B54202DD7AE0601C03D00F
:10954000012ED8BF4FF0FF343D4800256B46E8465A
:109550004FF03A09AC4203D183F80090A5194EE0D0
:1095600015B183F80090013311F815E01EF0F00FEB
:109570004FEA450C17D04FEA1E1A0EF00F0E10F8E6
:109580000AA010F80EE083F801E001EB0C0E83F85E
:1095900000A09EF801E04FEA1E1E033310F80EE013
:1095A00003F801EC21E0BEF1000F10D010F80EA07E
:1095B0009E460EF802AB01EB0C0A9AF801A04FEAA6
:1095C0001A1A10F80AA083F801A073460DE001EB07
:1095D0000C0E9EF801E01EF0F00F1FBF4FEA1E1E9A
:1095E00010F80EE083F800E001338C4401359CF85C
:1095F00001E00EF00F0E10F80EE083F800E0072DEA
:1096000003F10103A6DD611C05D03444082C02BF20
:109610003A2119700133002103F8011BC8EB030341
:1096200093423FF65EAF4146384605F0E7FE3846C6
:1096300002E02E461C4683E70AB0BDE8F08700BF73
:10964000CE1301082DE9F0470F46054610B900205A
:10965000BDE8F0870029FAD01022002105F0D8FAE1
:109660003B783A2B04D00024A1462646A04619E0B8
:109670007A783A2A07F10103E9D11F46F3E7514608
:109680002B4805F0DDFC98B951462A4805F0D8FC76
:1096900080B1284BC01A40EA0616B6F5803FD6D2F4
:1096A0004FF0010917F801ABBAF1000FE7D119E04B
:1096B0001F4BEFE7BAF13A0FC9D1B9F1000F05D14D
:1096C000B8F1000FC3D105EB0408EBE7A21C102A88
:1096D000BDD8631CDBB2310A29558146EE54D4B2A1
:1096E0000646DFE7B9F1000F08D0A21C102AAED859
:1096F000631CDBB2310A2955EE54D4B2B8F1000F25
:1097000010D02C44C8EB040805F1100201230021FD
:10971000434504F1FF3407DC207802F8010D0133E2
:109720002170F5E7102C92D12846BDE8F08700BFE4
:10973000CE130108DF13010810B5017801F0F00322
:10974000602B8AB0044603D009091B4805F068FB6A
:1097500022786378110149B21B0901F030001943E6
:10976000C2F381020343C9B2144805F059FB2168D2
:10977000134809BAC1F3130105F052FBA188E3793C
:10978000A279104849BA89B205F04AFB282204F1AF
:1097900008016846FFF7A0FE01460B4805F040FBB4
:1097A000282204F118016846FFF796FE0146074893
:1097B00005F036FB0AB010BDF01301080D140108C6
:1097C0003E14010853140108801401089414010880
:1097D0002DE9F8431546814613480F4603F0EEFF86
:1097E000002D08BF1025002407F1FF38A74218D02C
:1097F0000E4803F0E3FF661C19F8040003F0C6FFEF
:10980000B6FBF5F305FB13630BB1A04507D1084880
:1098100005F090FBA04502D0304603F0C3FF34466C
:10982000E4E7BDE8F88300BFAD140108D01E0108CD
:10983000593801080146014802F0BABDEC49002040
:10984000124BF0B593E83400D8681E691C6084EAB6
:10985000050122F000424A4082EA420280EA5000BA
:1098600050405969D86040F3000782EA80223940AD
:109870004A4004EB12249A609A693E40604044F3E7
:109880000004754014405D606040F0BDEC4900206C
:109890000C4B0146186882689368013B002B10B49A
:1098A000936005DA9469A34208DBCBB20A2B05D09A
:1098B0001368581C1060197010BC704710BC06F07B
:1098C0000FB800BF9402002008B53E20FFF7E0FF6C
:1098D0002020FFF7DDFF034B1B689868BDE80840B8
:1098E00004F0C6BE940200202DE9804885B0814670
:1098F00000AF0E469246FFF7E7FFB0460AF1FF348D
:109900000025C6EB0803A342F5DA844B18684168CA
:109910004B68013B002B4B6004DA05F013FB002879
:1099200004DAE8E70B685A1C0A6018780D2801D0A1
:109930000A280FD100240D2088F80040FFF7A8FF67
:109940000A20FFF7A5FF4645D5D0334622462546D7
:1099500020462BE0082801D07F280DD14645D0D0E5
:10996000082008F8015CFFF793FF2020FFF790FF25
:1099700008F1FF3B082003E008F1010B88F8000024
:10998000FFF786FFD846BCE7222913D15C781CB3C9
:109990005C2C25D001331C788C42F7D159782029D2
:1099A0001AD80135197811B303F8010B1978202959
:1099B000F8D9E9E7272906D1E8E74B1C497822299D
:1099C0000AD02029EDD91C785C2C1946F5D1591CF8
:1099D0005B780132002BF0D1514805F0ABFA8AE7F1
:1099E0009C1C9B780132002BF6D02346D3E7002D38
:1099F00081D0AB000E3323F00703EB46ADEB030D34
:109A00006C464DF82510304690F800E003460130D2
:109A1000BEF1000FF8D0BEF1220F02D0BEF1270F29
:109A200000D1013344F821301846013390F800E0AA
:109A3000BEF1000FF8D101318D42E5D1201FBAB13E
:109A400050F8043FA3B1194613F801EBBEF1000F23
:109A5000F5D0BEF15C0FF6D191F800E0BEF1000F39
:109A600004D091F801E001F801EBF5E7013AEAD101
:109A70002C4B2268FB60C7F80890002307F108010F
:109A800051F82380B8F1000F0DD10133022B16D00D
:109A9000F4E711463B607A6005F046FB7A683B6864
:109AA00030B108F10C08D8F800000028F1D1ECE73B
:109AB000D8F808301BB12146284698472CE0216889
:109AC000194805F031FB054610BB184A18491948DA
:109AD00005F0A6F9184805F02DFA124BC7F80890C2
:109AE000FB602C4607F1080353F824500DB10C35E8
:109AF00003E00134022CF5D10EE00C3555F8181CAA
:109B00000029F6D055F8142C0A4805F089F9F4E735
:109B100021680A4805F084F9DD46ECE6940200204D
:109B2000B61401089C160108CF140108D4140108CA
:109B3000E0140108E8140108552E0108F214010888
:109B400008B503F0D1FD002008BD08B5F7F7AEF960
:109B5000002008BD012810B506D10020F7F712FE3D
:109B600004460146074805E0486804F0A9FC04469D
:109B70000146054805F054F92046FFF75BFE00203A
:109B800010BD00BF201701084617010808B5FFF7F0
:109B900057FE0146024805F043F9002008BD00BF0A
:109BA0007A1001080146062814D8DFE800F0040600
:109BB0000B0D0F110900094800E0094805F030B904
:109BC0000848FBE70848F9E70848F7E70848F5E7D9
:109BD0000848F3E7084805F023B900BF68170108F3
:109BE0006C170108721701087A1701087F1701081E
:109BF00082170108851701088B170108102828D043
:109C00000BD803281BD003D8E8B1022815D0704721
:109C1000052816D006281AD07047262815D004D853
:109C2000162818D0202818D070472A2817D02B289B
:109C300017D0272818D10D4814E00D4812E00D4820
:109C400010E00D480EE00D480CE00D480AE00D480C
:109C500008E00D4806E00D4804E00D4802E00D481C
:109C600000E00D4805F0DCB8704700BF1718010888
:109C700090170108A0170108AD170108C3170108C4
:109C8000CB170108D0170108E3170108F5170108E1
:109C90000A1801082E1801083918010808B50146EC
:109CA000034805F0BDF80348BDE8084005F042B997
:109CB000481801086D18010813B5044601A8FBF700
:109CC0001BFA20B1BDF90400031B5842584102B0F1
:109CD00010BD00001FB504AB012403F8012D009452
:109CE0000022FBF71BF8002804DA094805F022F9E6
:109CF00020460BE09DF80F10064B074A0748002945
:109D000014BF1146194605F08BF8002004B010BDB1
:109D1000FB1B0108F81B010859380108171C010832
:109D2000A0F13003DAB2092A04D9A0F16103DAB252
:109D3000052A01D8184670474138C3B2052B88BFA1
:109D40004FF0FF30704700007FB50C4608210546F4
:109D50000DEB0100164603F0C9FF08B911480FE0EA
:109D6000009002AB002221462846FAF7D7FF0028D0
:109D70000ADA0D4805F054F82046FFF73FFF0B487C
:109D800005F0D8F801200BE0094805F049F8204615
:109D9000FFF734FF32462946064805F041F8002017
:109DA00004B070BD2E1C0108A11C0108593801081F
:109DB000B71C0108C51C01087FB5064610460D46B4
:109DC00004F07EFB04AB012403F8010D0022009493
:109DD00029463046FAF7A2FF00280ADA0C4805F0B7
:109DE0001FF82846FFF70AFF0A4805F0A3F82046A7
:109DF0000CE0094805F014F82846FFF7FFFE9DF82F
:109E00000F200648314605F00BF8002004B070BD65
:109E1000A11C010859380108B71C0108DE1C010803
:109E20007FB506460D461046531E13F8014F1CB170
:109E3000303C092CF9D908E00A22214605F038FD0A
:109E40000390013009D11C481CE01022002105F0CC
:109E50002FFD03900130F6D00124039BB3F5803F22
:109E6000F1D202230093002203AB29463046FAF7D1
:109E700055FF00280ADA114804F0D2FF2846FFF700
:109E8000BDFE0F4805F056F8012012E00D4804F021
:109E9000C7FF2846FFF7B2FE31460B4804F0C0FF6B
:109EA000039924B1094804F0BBFF002001E00848F1
:109EB000F9E704B070BD00BFF71C0108A11C010840
:109EC00059380108B71C0108451D01085B1D010830
:109ED000BF400108022808D0FF2808D0054A064BD9
:109EE00001280CBF184610467047044870470448C4
:109EF000704700BF741D0108631D01086B1D010838
:109F0000701D010870B5012988B00C46164609D1AC
:109F100004230093002207AB2921FAF7D9FE051E7E
:109F20000EDA09E0022905D1F9F7BCFC079008B167
:109F3000012505E06FF08505154804F0FBFF24E0DE
:109F4000E4B266B11C220021079804F061FE2046AD
:109F5000FFF7C0FF01460F4804F062FF15E02046FE
:109F6000FFF7B8FF079AD368516804939368039387
:109F700013690293019113680B440093936952692A
:109F80000146054804F04CFF3546284608B070BD30
:109F90007C1D0108B61D0108D71D01082DE9F047F9
:109FA00090B002AF00260446FE70F9F723FA21466E
:109FB0000546CB4804F034FF082300933246FB18D3
:109FC00002212046FAF784FE061E1CDB06EB46083B
:109FD00008F1070323F00703E946ADEB030D0DF18C
:109FE000080AC04804F01CFF334607F10802414646
:109FF000504603F04FFE0146BB4804F011FFBB483A
:10A0000004F00EFFCD4602230022009311463B1DB3
:10A010002046FAF75DFE002803DBB988B44804F057
:10A02000FFFE0223009300223B1D26212046FAF763
:10A030004FFE002803DBB988AE4804F0F1FE02238E
:10A04000009300223B1D06212046FAF741FE00281E
:10A0500003DBB988A84804F0E3FEA84804F0E0FE5A
:10A06000082300930022FB1803212046FAF730FE54
:10A07000061E1EDB06EB460808F1070323F0070364
:10A08000E946ADEB030D0DF1080A9D4804F0C8FE4A
:10A09000334607F108024146504603F0FBFD0146F6
:10A0A000984804F0BDFE9848CD4604F0B9FE01265C
:10A0B00000E00026022300930022BB1D1021204651
:10A0C000FAF706FE002804DBB7F906108F4804F003
:10A0D000A7FE012300930022BB1C18212046FAF79B
:10A0E000F7FD002808DB8A4804F09AFEB878FFF7ED
:10A0F00059FD7E4804F094FE012300930022FB18D2
:10A1000016212046FAF7E4FD002803DB7978814820
:10A1100004F086FE4FF00108CDF8008007EB08033D
:10A12000002220212046FAF7D3FD002810DBCDF8CD
:10A130000080FB1C00221F212046FAF7C9FD0028E1
:10A1400006DBFB78434503D17978734804F068FE59
:10A150006A4804F065FE012300930022FB1C1321D2
:10A160002046FAF7B5FD002808DB97F80380B8F120
:10A17000010F03D1694804F053FE464601230093C2
:10A180000022FB1C14212046FAF7A2FD002808DB60
:10A1900097F80380B8F1010F03D1614804F040FE45
:10A1A0004646012300930022FB1C15212046FAF7A6
:10A1B0008FFD002808DB97F80380B8F1010F03D169
:10A1C000584804F02DFE4646012300930022FB1C54
:10A1D00012212046FAF77CFD002808DB97F803805F
:10A1E000B8F1010F03D1504804F01AFE464601238E
:10A1F00000930022FB1C19212046FAF769FD002874
:10A2000008DB97F80380B8F1010F03D1474804F049
:10A2100007FE4646012300930022FB1C1F21204617
:10A22000FAF756FD002808DB97F80380B8F1010F14
:10A2300003D13F4804F0F4FD464601230093002279
:10A24000FB1C1E212046FAF743FD002808DB97F887
:10A250000380B8F1010F03D1364804F0E1FD464612
:10A26000012300930022FB1C23212046FAF730FD36
:10A27000002808DB97F80380B8F1010F03D12E48BE
:10A2800004F0CEFD4646FDB1B5F8C8112B4804F0E8
:10A29000C7FD95F8CA112A4804F0C2FDB5F8C631C9
:10A2A000D80702D5274804F0BBFDB5F8C631990799
:10A2B00002D5254804F0B4FDB5F8C6315A0702D5D9
:10A2C000224804F0ADFD01262046FEF7E9FD0028F6
:10A2D00040D00379002B3DD01D4804F0A1FD3AE0A9
:10A2E000821E0108B91E0108C91F0108D11E0108FC
:10A2F0008E1E01089D1E0108A91E0108B11F01083C
:10A30000B51E0108C31E0108C71E0108D31E01089F
:10A31000E61E0108EF1E0108031F0108161F0108B1
:10A32000201F01082A1F0108341F01083E1F0108D1
:10A33000481F01084F1F0108591F0108681F010825
:10A34000721F01087A1F0108801F0108861F01087B
:10A35000901F010816B1394804F062FD02230093F2
:10A3600000223B1D05212046FAF7B2FC002803DB42
:10A37000B988334804F054FD002D58D0B5F8C631E3
:10A380003049314813F0800F304B08BF194604F0B4
:10A3900047FD2A4804F044FD05F5E07610222C49DB
:10A3A000284604F005FB002831D02A4804F038FD87
:10A3B0002822294607F11000FFF78EF808B36A7CBF
:10A3C000254807F1100104F02BFD082223492846F7
:10A3D00004F0EEFA38B12B78FF2B06D16B7803F03E
:10A3E0000F03022B01D11E4800E01E4804F018FDA7
:10A3F0002B7CDB0708D52B78FF2B0CBF1A481B489A
:10A4000000E01B4804F00CFD0C4804F009FD383551
:10A41000B542C3D1174804F08DFD0022012120462A
:10A42000FFF770FD002202212046FFF76BFD114867
:10A4300004F080FD3837BD46BDE8F087B11F010844
:10A44000971F0108731E0108BE1F0108791E01082D
:10A45000AE130108CC1F0108D91F01085E130108C3
:10A46000E81F0108EE1F0108F51F0108022001087E
:10A470000D200108593801082DE9F04F012889B055
:10A48000804602AF0E460BDC07F10800FAF734FEF7
:10A4900018B1B7F90800FFF781FD002400F06EBC89
:10A4A0004868431E13F8014F3CB3303C092CF9D9DE
:10A4B0003168A94804F0B4FC3068FFF7EFFB31685D
:10A4C000A64804F0ADFC3168A54804F0A9FC316849
:10A4D000A44804F0A5FC3168A34804F0A1FC31684D
:10A4E000A24804F09DFC3168A14804F099FCA14801
:10A4F00004F020FD012400F041BC03F0E1FF05B2AF
:10A500002846FFF7D9FB002800F01984B8F1020FA4
:10A5100004D12846FFF742FD00F030BC9649B068F0
:10A5200004F002FE002840F02482B8F1040F01DCA0
:10A5300030681BE2D6F80C809048D6F80090366957
:10A54000414604F0F1FD10B9324602210CE04146CB
:10A550008B4804F0E9FD0028F6D04146894804F014
:10A56000E3FD28B9324603212846FFF7EDFBACE3B3
:10A570004146854804F0D8FD10B93246002151E02B
:10A580004146824804F0D0FD0028F6D0414680487C
:10A5900004F0CAFD10B93246262143E041467D4809
:10A5A00004F0C2FD10B9324606213BE041467A482C
:10A5B00004F0BAFD0028F6D04146784804F0B4FD16
:10A5C0000028F0D04146764804F0AEFD044610BBAA
:10A5D000304603F075FF07F11803022223F8100D2F
:10A5E0001021009228462246FAF798FB002807DA45
:10A5F0006C4804F015FC6C4804F012FC6B4877E7DB
:10A600006B4804F00DFC684804F00AFCB7F9082018
:10A610006848294607E34146674804F085FD28B9A4
:10A62000324605212846FFF7FBFB4EE341466348CF
:10A6300004F07AFD0446002863D13146604804F0F6
:10A6400073FD08B9002332E031465E4804F06CFD2A
:10A650000028F7D031465C4804F066FD08B90123B4
:10A6600025E03146594804F05FFD0028F7D0314617
:10A67000574804F059FD08B9022318E031465548FF
:10A6800004F052FD0028F7D03146534804F04CFD49
:10A6900008B905230BE03146504804F045FD002879
:10A6A000F7D031464E4804F03FFDB8B906230126E5
:10A6B0003B720022009607F1080318212846FAF79A
:10A6C0002DFB002812DA474804F0AAFB387AFFF77E
:10A6D00069FA364804F02EFC34464FE331464248CE
:10A6E00004F022FD0028E1D0404801E72946404817
:10A6F00004F096FB387AFFF755FA2C4804F01AFC60
:10A700003CE341463B4804F00FFD10B932461621A8
:10A710000EE04146384804F007FD10B932462021CA
:10A7200006E04146354804F0FFFC28B932462721AF
:10A730002846FFF741FBC8E24146314804F0F4FCEB
:10A740000446002840F0978031462E4804F0ECFC87
:10A75000002859D1012363E064270108442401083B
:10A7600009250108F7260108F2220108F72301084C
:10A7700079270108A4270108FE200108BC20010850
:10A78000C1200108CC200108C3170108D620010808
:10A79000CB170108DB200108DF200108E3200108B6
:10A7A000EA200108A11C0108E31701085938010833
:10A7B000B71C0108DE1C0108F0200108AC0A0108E2
:10A7C000F820010868170108D22501086C17010854
:10A7D000730A01087A170108FC200108851701088F
:10A7E000022101084B210108721701080A21010802
:10A7F0006A210108922101089A210108A721010874
:10A80000B52101081E2001083146B04804F08CFC37
:10A8100000289FD03146AE4804F086FCC8B900231A
:10A820004FF001083B720022CDF8008007F10803C9
:10A830002A212846FAF772FA002812DAA54804F00D
:10A84000EFFAA54804F0ECFAA44804F073FB444680
:10A8500094E23146A24804F067FC0028DFD0A1480A
:10A8600046E6A14804F0DCFA9B4804F0D9FA3246E7
:10A8700029469E48D7E141469D4804F055FC0446D0
:10A88000002872D1304604F01BFE4FEA500909F14E
:10A89000070323F00703EA460E28ADEB030D8346BA
:10A8A0000DF1080801D1934806E0102801D1924823
:10A8B00002E0202804D1914804F0B2FA002117E008
:10A8C000302801D18E48F7E7402801D18D48F3E7C1
:10A8D000802801D18C48EFE78C4804F0A1FA17E0FA
:10A8E000421C12D04A0800EB031008F802000231A3
:10A8F0008B450FD9705CFFF713FA721878605078A7
:10A90000FFF70EFA7B685A1CEAD1814804F012FB6B
:10A91000012428E0CDF80090434600222B21284650
:10A92000FAF7FCF9002807DA6A4804F079FA79485E
:10A9300004F076FA6948E9E76B4804F071FA754863
:10A9400004F06EFA2946744804F06AFA4546C14498
:10A95000A94505D015F8011B704804F061FAF7E726
:10A960005E4804F0E7FAD54608E24846FFF796F954
:10A97000C0E56B49B06804F0D7FB044600286AD1F3
:10A98000B8F1030F01D1316827E0A8F10308B8F14D
:10A99000010FD6F80C9022D06249D6F800A04846A4
:10A9A00004F0C2FB20B9D6F810904FF0020A17E06D
:10A9B0005D49F06804F0B8FB20B9D6F810904FF06C
:10A9C000010A0DE05949F06804F0AEFB20B9D6F851
:10A9D00010904FF0000A03E051465548ABE1824623
:10A9E0002F2140224846FEF768FD431E802B064675
:10A9F000494628BF402607F108005FFA86FBFEF7AC
:10AA000021FE00283AD0B8F1010F07D03B7AFF2B86
:10AA100004D1BAF1010F07D0464869E5BAF1020F37
:10AA200014BF4023412300E040235A4607F10801A8
:10AA30002846F8F7FDFC18B93F4804F0F1F959E54C
:10AA40004FF0FF334361836132462B4649463B4812
:10AA500004F0E6F992E13A49B06804F065FB044677
:10AA6000B8B9B8F1030F02D13168364863E1F6682E
:10AA700007F108003146FEF7E5FD08B9324837E531
:10AA800007F108012846F8F7FBFC2A4631462F4813
:10AA9000C9E02F49B06804F047FB0446002869D19B
:10AAA000B8F1030F02D131682A4844E1F06803F09D
:10AAB00007FDA0F5A063B3F57B4F06464ED34FF6D6
:10AAC000FF724FF4A06124489FE000BFBD21010840
:10AAD000F8200108A11C01082E18010859380108A6
:10AAE00068170108C0210108B71C0108C51C01082E
:10AAF000D3220108F02101080D2201082A220108B1
:10AB0000482201086622010884220108A2220108C5
:10AB1000BC22010839180108D72201080A100108CF
:10AB2000EE2201083E2301084623010850230108B4
:10AB3000F22201087D230108A9230108CC23010882
:10AB4000F3230108F7230108582301081A240108F8
:10AB500040240108442401085F2401082846F8F72E
:10AB600049FC08B98848C3E4A0F8C8612A463146C0
:10AB7000864858E08649B06804F0D6FA044670BBAF
:10AB8000B8F1030F17D08349F06804F0CDFA00281C
:10AB900000F0EA808049F06804F0C6FA002800F06E
:10ABA000E6807E49F06804F0BFFA002800F0CA8011
:10ABB000F1687B48BAE04FF0FF0919F0010F04D0AB
:10ABC000224601212846FFF79DF919F0020F3FF4B4
:10ABD00091AC224602212846FFF794F98AE4714994
:10ABE000B06804F0A1FA044600BBB8F1030F02D12B
:10ABF00031686D489FE0F06803F062FCFF2806466C
:10AC000006D96A484FF6FF72002104F009F971E491
:10AC10002846F8F7EFFB08B9654869E480F8CA618F
:10AC200064482A46314604F0FBF8A7E0D6F80880CD
:10AC3000614998F80030D6F800902D2B08BF08F134
:10AC4000010840460CBF0026012604F06DFA10B939
:10AC50003246132136E05949404604F065FA10B9EE
:10AC6000324612212EE05649404604F05DFA10B9F2
:10AC70003246142126E05349404604F055FA10B9F3
:10AC8000324615211EE05049404604F04DFA10B9F5
:10AC90003246192116E04D49404604F045FA10B9F4
:10ACA00032461F210EE04A49404604F03DFA10B9F1
:10ACB00032461E2106E04749404604F035FA30B9D5
:10ACC000324623212846FFF705F8044656E042495C
:10ACD000404604F029FA044678B92846FEF7E0F821
:10ACE00008B93E4804E426B10123037129463C48D3
:10ACF0001CE0067129463B4818E03B49404604F0F9
:10AD000013FA0446A8B92846F8F774FB10B9374877
:10AD1000FFF7EEBB2EB10121F8F783FB294634483B
:10AD200004E03146F8F77DFB3248294604F078F814
:10AD300024E03148494604F073F8FFF7DBBB2F48A5
:10AD4000FFF7D6BBB8F1040F0AD04FF00209052275
:10AD50002B49306904F022FCB0FA80F464092CE736
:10AD600004464FF0020930E74FF0FF0901E04FF0D1
:10AD70000109B8F1040FEAD1002421E720461C376D
:10AD8000BD46BDE8F08F00BF87240108A12401085B
:10AD9000C4240108701D0108CA2401089A11010881
:10ADA000CD240108062501080925010823250108ED
:10ADB00051250108712501089A250108A2250108DD
:10ADC000AA250108B2250108BA250108BE250108F7
:10ADD000C3250108CB250108D8250108DD25010878
:10ADE000FB250108222601084A26010852260108EF
:10ADF00086260108BE260108F72601084A20010818
:10AE0000FC2001082DE9F04F87B006AF05468846C3
:10AE100091469A4604F054FB28448542A0EB050471
:10AE200013D010F801392F2B05D1601C284403F0F2
:10AE300047FB06460BE03A2B01D02E2BEDD12846DE
:10AE400004F03EFB0026044601E00024264604F1FF
:10AE5000080323F00703ADEB030D0DF1180B621C83
:10AE60000021584603F0D4FE29462246584603F0F6
:10AE7000D1FD404604F024FB59461648FEF7E2FB9C
:10AE8000D0B1144D102441461348FEF7DBFBD0B17E
:10AE9000114B102200213606039102920193CDF846
:10AEA00010A0009623462A4649460C48F7F790FA28
:10AEB0000437BD46BDE8F08F03F00AFB6A23036048
:10AEC000074D0424DFE703F003FB6A230360042239
:10AED000044BDFE7184A0020084A0020A810002091
:10AEE0002C4A0020284A002001282DE9F34105467C
:10AEF0000C4603D17A48F7F715FCBBE002281AD1BB
:10AF00004968784804F010F9002800F0B1806168C1
:10AF1000754804F009F908B97448B8E061687448E4
:10AF200004F002F9014620B96D48F7F740FB71487B
:10AF3000ADE07148ABE053DD49686A4804F0F4F8CD
:10AF400058B16168684804F0EFF830B1616868484A
:10AF500004F0EAF808B1694899E0032D25D1616849
:10AF6000634804F0E1F8054690B9A06803F0A8FA38
:10AF700004B22046FAF7CCF8214628B15848F7F732
:10AF800016FB21465E4800E05E4803F049FFA2E060
:10AF9000A1685D48FEF756FB054600286CD01022DC
:10AFA00059494F48F7F7E5FA64E0052D18D1616873
:10AFB0004C4804F0B9F8002868D1E168534804F01F
:10AFC000B3F80546002861D101A8FAF795F80128E1
:10AFD00031D14FF0FF33BDF904202169A0683DE075
:10AFE000072D3ED161683F4804F09EF8C8B9E1687A
:10AFF000464804F099F8A0B96169454804F094F80E
:10B00000054670B901A8FAF777F8012813D1A069AD
:10B01000BDF90480A668276903F052FA4246034648
:10B020001AE061682F4804F07FF820B9E1683748DA
:10B0300004F07AF808B1374829E06169364804F02D
:10B0400073F805460028F6D1A069A668276903F0C1
:10B0500037FA4FF0FF3302B239463046FFF7D2FEDF
:10B0600039E0092D12D161681E4804F05DF890B1F5
:10B070002A480CE000252EE003F02AFA6A23036038
:10B08000042227491648F7F774FA24E0254803F00C
:10B0900051FF01251FE0E1681C4804F045F8002835
:10B0A000E6D161691C4804F03FF80028E0D1E1696D
:10B0B000174804F039F805460028D9D1A069A668D8
:10B0C000276903F0FDF98046206A03F0F9F90FFAC9
:10B0D00088F20346C0E7284602B0BDE8F08100BF11
:10B0E000A8100020EE220108F3230108BE29010860
:10B0F000522A0108582A0108792A0108F62A01086B
:10B10000462B01087A2B0108184A0020982B0108C9
:10B110000E2D01089C2B0108172D0108DE270108C0
:10B120002C4A00201B2D010813B5044601A8F9F78D
:10B13000E3FF20B1BDF90400031B5842584102B09F
:10B1400010BD000000F00700072813D8DFE800F06A
:10B150000406080A0C0E121008480CE008480AE021
:10B16000084808E0084806E0084804E0084802E00B
:10B17000084800E0084803F053BE00BF6B2D0108EB
:10B18000782D0108852D0108922D01089F2D0108B9
:10B19000AC2D0108B92D0108C62D010800F03000C2
:10B1A000202805D0302805D0102805D1044804E017
:10B1B000044802E0044800E0044803F031BE00BF48
:10B1C000D32D0108D62D0108DB2D01087B2E0108A7
:10B1D000F0B5012893B006460D4607D16B4803F041
:10B1E000A9FE6B4803F0A6FE002005E04968694807
:10B1F00003F09AFF30BBF1E702F0E0FC04460028C0
:10B2000000F0C1802822214608A8FEF765F9237EB8
:10B21000B4F91A60054604F11002182102A802F0E0
:10B2200039FD3246034629465B4803F0F9FD607E4E
:10B23000FFF788FF607EFFF7B1FF584803F07AFE02
:10B240002046D9E7012E40F39680022E74D069681B
:10B25000534803F069FF0446002857D1023E012EEF
:10B2600002D0022E0CD022E008A8F9F745FF0128F1
:10B2700098BFBDF92060AF6888BF264600251CE056
:10B28000AF6808A83946FEF7DDF928B9A86803F0C9
:10B2900017F9EF6806B2F1E702A8F9F72DFF0128C8
:10B2A00098BFBDF90860ED6888BF264605E0A8682C
:10B2B00003F006F9EF682D6906B23046FFF734FF58
:10B2C00008B9384805E0394608A8FEF7BBF920B9A7
:10B2D000354803F02FFE012455E04DB108212A46E0
:10B2E0000DEB010002F002FD034610B92F48F0E714
:10B2F0002B460022009208A902AA304602F0BEFBAB
:10B3000008B92B48E5E739462A4812E069682A4817
:10B3100003F00AFF044678B9AD6808A82946FEF78D
:10B3200091F90028D4D008A9204602F03DFC23481A
:10B33000294603F075FD26E06968214803F0F4FE14
:10B340000446C0B902F03AFC2146054655B119B190
:10B35000B1F91A0002F028FC284602F02FFC294619
:10B360000546F3E719B1B1F91A0002F01DFC1548C2
:10B3700003F056FD07E02B6800931A461946124861
:10B3800003F04EFDA7E7204613B0F0BDDF2D010806
:10B390002E2E01085A1601087D2E01085938010881
:10B3A000EE220108922E010858230108B22E01084E
:10B3B000DD2E01080D2F0108F32301083F2F01089E
:10B3C000FC200108682F0108872F010870B50128AB
:10B3D0008AB00C460DDD486803F072F805B22846C5
:10B3E000FFF7A2FE30B92168164803F019FD0120CD
:10B3F00025E00025144803F09DFD144803F09AFD54
:10B40000002002F0F3FB0446C8B1B4F91A600DB194
:10B41000AE4212D1282221466846FEF75DF8314639
:10B4200002460B4803F0FCFC607EFFF78BFE607E5B
:10B43000FFF7B4FE074803F07DFD2046E1E70AB0C0
:10B4400070BD00BF333001084C300108492E01089F
:10B45000803001085938010808B501460B4803F04F
:10B46000DFFC0B4803F066FD0A4803F063FD0A4861
:10B4700003F060FD094803F05DFD094803F05AFD43
:10B480000848BDE8084003F055BD00BF8E300108F4
:10B49000EA300108F4300108023101085C3101088A
:10B4A00070310108813101080C4AF0B51488083068
:10B4B000260AE5B200238B4209D2FF2C85BFC718AC
:10B4C000C654C5547D708CBF02330133F3E781BF8E
:10B4D000138809181B0A01F8013CF0BD90020020F6
:10B4E0002DE9F0430D4685B002210446F9F7C9FE67
:10B4F000032107462046F9F7C4FE07B108B92748DB
:10B5000045E08668264AB388F48812885BBA9BB205
:10B5100064BA9A42A4B239D12249234B0A881B88C3
:10B520009A4203D9944203D3012307E0944204D3FF
:10B530009C428CBF0023012300E0002333B3BF688B
:10B54000D0F80C901948944298BF013207F10808CE
:10B5500098BF0A8028224146FDF7BEFF4FF47A7259
:10B56000B388B5FBF2F102FB115502910395FA790C
:10B5700001925BBA02469BB2494600940C4803F024
:10B580004FFC404602F03AFB012003E0094803F07B
:10B59000D1FC002005B0BDE8F08300BF9C3101085C
:10B5A00090020020584A00205A4A0020304A0020C9
:10B5B000D3310108163201082DE9F04F99B08146C8
:10B5C0000C461022002114A803F022FB81231593BE
:10B5D000994BB9F1010F1B88ADF85C303BDDB9F137
:10B5E000020F00F0C281606802F06AFF051ED4BF3E
:10B5F0004FF000084FF0010808F101034FEA8307FC
:10B6000054F82330089308F10203D8BF0325994565
:10B6100005DDE319586802F053FF049001E00423AC
:10B62000049308F10303994505DDE319986802F0D6
:10B6300047FF064601E04FF47A7608F10408C14559
:10B6400005DD2744F86802F03BFF099000E009950A
:10B65000049B002B03DA2068FFF7FEFE3FE04FF06B
:10B66000FF3225210898FDF728FF04B2621C0899D3
:10B6700010A808BF0024FDF7E5FF08B96F482CE0CB
:10B6800008226F4910A803F093F950B19DF840309B
:10B69000FF2B05D19DF8413003F00F03022B00D0A2
:10B6A000A4B10EA8F9F728FD44B1002800F0588194
:10B6B000BDF938309C4240F0538106E0012802D1A8
:10B6C000BDF9383001E05F4807E01C4614A90320AB
:10B6D000F9F75EFD002804DA5B4803F02BFC01203B
:10B6E0004BE1F5F787F94FF47A7373430D9300221A
:10B6F0000023CDE90A010027CDE906234FF0FF33EF
:10B700002E460593BA46BB46013E731C4F4A00F0D5
:10B7100006814E4B19884E4B1A88013292B21A801C
:10B72000049B00938020002302F012F9804698B118
:10B7300004998068FFF7B8FE10AA00214046F7F789
:10B74000D7FC814640B1ACB14FF0FF330822002155
:10B75000F9F71AFF814618B93E4803F0EBFBD3E72F
:10B76000836800221A705A705A719A711A715A803D
:10B7700083685C800020F6F705F84B46804640F26F
:10B78000022235490220F9F74FFA0C9038B93348B4
:10B7900003F0D0FB0C994846F9F7E8FFB4E7304ACC
:10B7A00000230EA801F054F800282DDBBDF83A2044
:10B7B00040F201239A4220D10020F5F7E3FFDDF8A3
:10B7C0003C90C8EB000841464846FFF789FE00213F
:10B7D00083444846F9F7CAFF059B474538BF4746AB
:10B7E000434528BF43460593DDE9062312EB0802D3
:10B7F00043F10003CDE906231AE00F4B19880EA888
:10B8000009B2F6F7BFFB13E0164803F093FB0FE015
:10B810000EA8F6F759FC002828DDBDF83A3043455C
:10B82000F6D1114803F0FCFA00210F98F9F79EFFBA
:10B8300040F20128ECE700BF040300203332010886
:10B840005E1301084C3201089A3201089002002070
:10B850005A4A00208C2001080000FFFFBA3201087C
:10B8600040420F00E5320108F23201081EB100210A
:10B870000D9800F0A9FF099B0AF1010A534502D077
:10B88000002E7FF441AFF5F7B5F8089980463C48A3
:10B8900003F0C6FABBF1000FC6EB050A38DD5246CD
:10B8A000DDE90601D31702F07FFCDDE90A23B8EBDE
:10B8B00002029046334AB8FBF2F1642302FB118284
:10B8C0008DE806000C905A46514603FB0BF32E48B8
:10B8D00093FBFAF3C3F1640303F0A2FA4FF47A7214
:10B8E000B7FBF2F002FB107E01900C980C9BB3FBAF
:10B8F000F2F302FB1300009005980599CDF808E0DB
:10B90000B1FBF2F102FB1102204803F089FA03E0D7
:10B9100051461F4803F084FA4FF0000AF4E61D4B2D
:10B9200000211980138814A9013303201380F9F72B
:10B9300051FC40F201240EA8F6F7C6FB00280BDDEF
:10B94000BDF83A30A342F6D1134803F069FA00215A
:10B950000F98F9F70BFFECE7BBFA8BF040090CE00E
:10B9600021460E4803F05CFAB9E6636808930427A1
:10B970004FF000080325049753E619B0BDE8F08F97
:10B980003733010840420F00533301089C3301084C
:10B99000D03301085A4A0020F23201080734010866
:10B9A0009368013B002B10B4936008DA9469A342BA
:10B9B00002DBCBB20A2B02D110BC03F091BF13689B
:10B9C000581C10601970C8B210BC704710B502F056
:10B9D00077FD04B22046F7F70DFD20B9064803F0C5
:10B9E000A9FA012010BD2046FAF7C2F82146034803
:10B9F00003F016FA002010BD2D3401084934010867
:10BA000030B58FB00D4602F05BFD2946C4B26846E2
:10BA1000FDF718FE18B90E4803F08CFA10E0002369
:10BA20001A4669462046FAF71FF958B9282269468E
:10BA300004A8FDF751FD22460146064803F0F0F93F
:10BA4000012003E0044803F0EBF900200FB030BD03
:10BA500077340108A6340108D834010810B502F083
:10BA60002FFDC4B22046FAF7EBFF10B92146084873
:10BA700004E0FBF7E2F8214620B9064803F0D0F9CC
:10BA8000012010BD044803F0CBF9002010BD00BF19
:10BA9000FC340108253501084C35010830B58BB060
:10BAA00002F00EFDC5B22846FAF7CAFF044620B9D7
:10BAB0000A4803F03FFA01200EE0383000F0ECFCB9
:10BAC000282204F108016846FDF706FD2A460146D2
:10BAD000034803F0A5F900200BB030BD6C35010818
:10BAE0009435010830B58BB002F0EAFCC5B22846A7
:10BAF000FAF7A6FF044620B90A4803F01BFA012012
:10BB00000EE0383000F00EFD282204F108016846EE
:10BB1000FDF7E2FC2A460146034803F081F90020C4
:10BB20000BB030BD6C350108D335010870B58CB051
:10BB300002F0C6FCC6B23046FAF782FF0125044681
:10BB400020B9134803F0F6F928461EE0114A90F890
:10BB50002730B2F9000094F82820019294F82620AA
:10BB6000009205FA03F340F6011204F1380100F0E7
:10BB7000A9FC282204F1080102A8FDF7ADFC324619
:10BB80000146054803F04CF900200CB070BD00BF21
:10BB90006C350108BA3700201436010808B504498D
:10BBA0000020FAF7FDF9034803F0C4F9002008BDAE
:10BBB000081301085536010813B5234C234803F038
:10BBC000B9F9A36900932269A3682168204803F0AA
:10BBD00027F9E36900936269E36861681D4803F02F
:10BBE0001FF9A36B0093226BA36A216A1A4803F022
:10BBF00017F9E36B0093626BE36A616A174803F01D
:10BC00000FF9A36D0093226DA36C216C144803F00F
:10BC100007F9E36D0093626DE36C616C114803F00A
:10BC2000FFF8A36F0093226FA36E216E0E4803F0FE
:10BC3000F7F8E36F0093626FE36E616E0B4803F0F9
:10BC4000EFF8002002B010BD503D00206A36010818
:10BC5000AD360108DF360108113701084337010806
:10BC600075370108A7370108D93701080B380108D3
:10BC70002DE9F041514C524892B003F0D1F863786D
:10BC80000BB9504800E05048504DDFF86C8103F08C
:10BC9000C7F8286809218268FFF782FE28680A2110
:10BCA0008268FFF77DFE4A4803F0BAF8002606EBEB
:10BCB00008031B790BB9434800E04348434F03F0A6
:10BCC000AFF82868092182683036FFF769FE902EA8
:10BCD000EDD13868394D82680A21FFF761FE386876
:10BCE0000A218268FFF75CFEF4F784FE637806465B
:10BCF0000F46002B5DD0B5F88A0095F88030297882
:10BD0000B5F92C200290B5F888000190D5F8840090
:10BD1000008800902F4803F083F8E86E296F801B9D
:10BD200061EB0701002871F1000305DB2A4A0023BB
:10BD300002F03AFA064600E00026236A274993F902
:10BD40008C50282208A8FDF7C7FB94F8363094F8E9
:10BD50003270228E069613F0020F214B214918BF34
:10BD60001946638F059394F83830049394F826307D
:10BD7000039394F8273001269E4025EAE5758DE867
:10BD80006200194B1949022F08BF0B46014618489B
:10BD900003F046F8E46964B1611D282208A8FDF7A4
:10BDA0009BFBE369E28A0146124803F039F82468F4
:10BDB000F1E7002012B0BDE8F08100BFC03C0020D8
:10BDC000493801085A3801085E38010894020020F9
:10BDD000623801087138010840420F00C83C002059
:10BDE0001E200108F8200108423801083D380108EA
:10BDF000B53801080C3901081038002038B505465F
:10BE0000084602F05DFBC4B22046FAF719FE28B9D5
:10BE100021460B4803F004F8012038BD083015B165
:10BE2000FBF77EF801E0FBF782F8064B064A07486D
:10BE3000002D08BF1A46214602F0F2FF002038BD4F
:10BE4000FC340108423901083D390108493901082B
:10BE500038B50C4602F034FBC5B22846FAF7F0FDBF
:10BE600028B929460B4802F0DBFF012038BD90F8C5
:10BE70003630094923F0020343EA440380F83630A0
:10BE8000064B0748002C08BF194602F0C9FF0020E6
:10BE900038BD00BFFC3401085938010824150108D9
:10BEA00072390108012838B505460C4603DCBDE8A7
:10BEB0003840FFF7DDBE6349606803F035F90028BC
:10BEC000F5D0032D09D16049606803F02DF988B9D8
:10BED000A068BDE83840FFF779BD042D0AD15B4961
:10BEE000606803F021F928B9E168A068BDE838402E
:10BEF000FFF786BD5649606803F016F930B9032D87
:10BF00007AD1A068BDE83840FFF7A8BD5149606804
:10BF100003F00AF900BB042D6ED14F49A06803F06D
:10BF200003F920B9E068BDE83840FFF7B7BD4B49D9
:10BF3000A06803F0F9F820B9E068BDE83840FFF7E1
:10BF4000D1BD4749A06803F0EFF8002854D1E0685C
:10BF5000BDE83840FFF7EABD4249606803F0E4F805
:10BF600058B9032D48D14049A06803F0DDF80028F6
:10BF700042D1BDE83840FFF711BE3C49606803F08C
:10BF8000D3F820B9032D37D1A168012007E0384943
:10BF9000606803F0C9F830B9032D2DD1A168BDE860
:10BFA0003840FFF72BBF3349606803F0BDF8D0B9C4
:10BFB000022D21D03049A06803F0B6F8E0B9052D74
:10BFC0001AD12E49E06803F0AFF808B9012105E065
:10BFD0002B49E06803F0A8F8014668B92069BDE87C
:10BFE0003840FFF735BF2749606803F09DF818B95E
:10BFF000BDE83840FFF7E0BD234802F09BFF23482F
:10C0000002F098FF224802F095FF224802F092FFCA
:10C01000214802F08FFF214802F08CFF204802F0F7
:10C0200089FF204802F086FF1F4802F083FF1F4867
:10C0300002F080FF1E4802F07DFF1E4802F07AFFEA
:10C04000002038BD9A390108711501089F3901088F
:10C05000A4390108A7390108FC2001084F0F010885
:10C06000B90E0108CC0B0108AF3901083D390108B0
:10C0700042390108FE200108B33901081E200108D9
:10C08000F8200108C4240108B7390108CF39010894
:10C09000093A0108423A01087B3A0108B43A01081A
:10C0A000EB3A01082E3B0108773B0108B43B01083D
:10C0B000D93B0108243C0108F8B506460F46044662
:10C0C00023783D1B412B35440ED17B4802F032FFD3
:10C0D000282D40F2EF80601CFDF72EFB1022A5F109
:10C0E000290104F12900E1E013F0C00F06D17348E3
:10C0F00002F020FF102229462046D7E003F0F80284
:10C10000C02A11D16E4802F015FF21886D4849BA46
:10C11000C1F30A0102F084FE61886B4849BA89B212
:10C1200002F07EFE0434CBE7E02A17D1674802F024
:10C1300001FF2188634849BAC1F30A0102F070FE89
:10C140006188614849BA89B202F06AFE2179604883
:10C1500002F066FE1022691F601DA7E003F0E003F5
:10C16000602B40F0A7805B4802F0E4FE237803F0E8
:10C170001803082B09D002D863B9574808E0102BE0
:10C1800005D0182B06D1554802E0554800E0554827
:10C1900002F0D0FE237803F0040303F0FF0213B192
:10C1A00022B1514800E0514802F0C4FE237803F068
:10C1B0000303022B06D0032B06D0012B14BF4C48DF
:10C1C0004C4802E04C4800E04C4802F0B3FE637873
:10C1D00059060BD54A4802F023FE637803F030037A
:10C1E000102B15D00ED8C3B9464814E0464802F0CB
:10C1F00017FE637803F03003102B09D002D863B91F
:10C20000424808E0202B05D0302B06D1404802E000
:10C21000404800E0404802F08DFE637813F0080FBC
:10C2200003F004031FD05BB13C4802F083FE637847
:10C2300003F00303013B022B8CBF3948394822E04D
:10C24000394802F077FE637803F00303022B06D02F
:10C25000032B06D0012B14BF3448354813E0354872
:10C2600011E035480FE03BB1344802F0D9FD637866
:10C270009A070AD1324806E0324802F0D1FD6378CD
:10C280009B0702D1214802F055FE94F90130002BA2
:10C2900008DAA1782C4801F00F02090902F0C0FD6C
:10C2A000032000E00220291A10222044BDE8F840B3
:10C2B000FDF78EBAF8BD00BF503C0108693C01088B
:10C2C000833C0108A03C0108B43C0108C03C0108C3
:10C2D000E23C0108F03C0108FE3C01085C3D01081D
:10C2E000243D0108433D01088F3D0108843D0108BC
:10C2F0009E3D0108AB3D0108B33D0108BC3D01086E
:10C30000C63D0108EC3D01083B3E0108623E0108C4
:10C31000233E0108053E0108143E0108723E010853
:10C32000A53E0108D73E0108E43E0108183F010878
:10C33000343F01084F3F01086A3F0108843F01086C
:10C34000DB3E0108AE3F0108D93F010830B5036864
:10C3500045688468C168056085EA040223F00043EB
:10C36000534083EA430381EA510183EA010242F325
:10C37000000583EA8223C2600169426929402A409C
:10C380004C4053404460836030BD036823F0004359
:10C3900063B9436853B9836843B9C36833B9542157
:10C3A00049224E234FF0590C80E80E1070470000D0
:10C3B00038B503694360436983608369016004465B
:10C3C000C3600F4801256B1E03F0030305F0030251
:10C3D00054F8233054F8221083EA937300FB03537C
:10C3E00001354B40082D44F82230ECD12046FFF7B0
:10C3F000CCFF2046FFF7AAFF013DFAD138BD00BFB0
:10C400006589076C2DE9F341856804461DB9194912
:10C410000320F4F7E9FB427843689340C268C2EB1B
:10C4200005086A0093424FF000072CBF82608360CA
:10C43000478038BF5D088668FDF702FA711BB0FBC4
:10C44000F1F202FB11000544B4F91030E5604FF43D
:10C450007A7245446A43019304F11C030093A2627B
:10C46000E7623B4604F1300000F0E2F902B0BDE8BB
:10C47000F08100BFE509010810B5428803789A42AF
:10C48000044600D313B96369A06998472046BDE804
:10C490001040FFF7B7BF0000826843689A4210B5AA
:10C4A000044603D806490320F4F79EFB3030F4F726
:10C4B00017FB6368A3602046BDE81040FFF7A2BFEA
:10C4C000E5090108F8B50C46174606469DF8181010
:10C4D0009DF81C201D461BB910490320F4F784FB6E
:10C4E00003FA01F00E4B9842F6D8002363802270C5
:10C4F000656026826170FDF7A3F9C5EB8503B0FB8B
:10C50000F3F202FB13000544E560A5602682246275
:10C51000E7832046BDE8F840FFF774BFE50901084E
:10C52000FEFFFF7F3030F4F7DBBA438801334380EE
:10C530007047000010B501884288044649BA52BAD3
:10C5400092B289B2064802F06BFCA188E2880548E5
:10C5500049BA52BA92B289B2BDE8104002F060BC4A
:10C56000EF3F01081240010801210148F5F796BB91
:10C570005C4A00202DE9F04780460E46FFF7F4FFA5
:10C58000294C002514F8013C9E420AD1324641460E
:10C59000204602F00DFA20B9244B122404FB053486
:10C5A00028E00135282D04F11204EBD1204B1B6843
:10C5B000272B33D81D4B0025122202FB05F91B4FF8
:10C5C00019F803A0BAF1000F25D107EB090463782D
:10C5D0009E4207D010225146A01C02F019FB07F81A
:10C5E00009A06670122000FB0570324641460230F9
:10C5F00002F010FA23780F480133DBB2012B08BF99
:10C600000B4A237002BF136801331360F5F776FB02
:10C610002046BDE8F0870135282DCED10548F5F735
:10C620006DFB0020BDE8F087664A0020644A0020C8
:10C63000604A00205C4A002010B50446FFF794FFD2
:10C640004CB123783BB1013BDBB223701BB9044AE8
:10C650001368013B13600348BDE81040F5F74EBB7B
:10C66000604A00205C4A002070B5154606460C461C
:10C67000FFF77AFF72782B6893420AD3B11C2046E9
:10C6800002F0C8F973782B600548F5F737FB2046B0
:10C6900070BD2A600248F5F731FB002070BD00BF75
:10C6A0005C4A00202DE9F041174606468846FFF710
:10C6B0005BFF72783B68B3EBC20F05D1B01C00255D
:10C6C00001244FF0FF3316E02648F5F717FB6FF013
:10C6D0000100BDE8F081591C37D190F800E018F84E
:10C6E0000510714537D02B46C4B1BEFA8EF46409EB
:10C6F000A4B1013501309542EDD33CB100233B603C
:10C700001848F5F7FBFA0220BDE8F0815D1C05D161
:10C710001448F5F7F3FA2046BDE8F0811E4418F8F6
:10C720000310B2784A40072142FA01F4E40748B204
:10C7300002D40139F8D1084600EBC3033B60094835
:10C74000F5F7DCFA0120BDE8F081002CE6D0047892
:10C75000B4FA84F4CBE7002CCBD0B1FA81F46409AD
:10C76000C7E700BF5C4A002070B5FFF7FDFE0A4C2A
:10C77000002504F5347604F8025C04F8015C2046D8
:10C7800010220021123402F043FAB442F3D10348DC
:10C79000BDE87040F5F7B2BA664A00205C4A002056
:10C7A000F5F7ACBAB0F90010F5F7C8BB38B50446D8
:10C7B0000020F4F7E7FF05460020F4F7E3FF401BF5
:10C7C000A042F9D338BD000030B587B004460D460D
:10C7D000F3F751FE40B11DB10E490320F4F704FAFE
:10C7E0002046FFF7E3FF13E00B4B0090039002900D
:10C7F000012168460493CDF814D0F5F74FFA21468D
:10C8000001A82A46F4F79EF901216846F5F746FA91
:10C8100007B030BDE5090108A1C7000830B4034DD9
:10C82000C560026130BC1380F4F76CB9A5C700087D
:10C8300070B41146039ABDF91050044EC6600261EF
:10C8400015801A4670BCF4F77DB900BFA5C7000873
:10C8500070B58AB00021079106911049098803AC90
:10C8600009B2054643F23906019105A80094ADF8D6
:10C870000E600494FFF7DCFF2846F5F728FC6B8870
:10C88000B34202D16B68A34204D005A8F4F728F99B
:10C89000012001E04FF0FF300AB070BD040300201A
:10C8A00010B5084B0446182240F83C3B02F0B2F8A1
:10C8B000082384F85630002384F8543084F8573025
:10C8C00010BD00BF6840010837B5044600F03CFBCE
:10C8D00094F854301BB90321204600F060FA00257B
:10C8E0000821684684F83650258701F0E9FA9DF85A
:10C8F0000030019A23F0010343F002038DF8003069
:10C90000009B12BA1BBA204600F000F9BDF80010D7
:10C9100049BA204689B200F0E5F82046232100F00C
:10C9200028F920461A2100F015F92946204600F082
:10C930003DF920460122202100F0B8F920460122CD
:10C940004FF4807100F0B2F92A4620464FF40051AE
:10C9500000F0ACF9204601224FF4804100F0A6F926
:10C96000204601224FF4805100F0A0F9012384F801
:10C970002830802220460C2100F057FA042120465E
:10C9800000F065FA042100F0FD02204600F04DFAA7
:10C990000321204600F05BFA032100F0F00220465C
:10C9A00000F043FA082220460E2100F03EFA0F2143
:10C9B000204600F04CFA1621204600F0F0F903B0B2
:10C9C00030BD10B590F857300133044680F8573029
:10C9D000204600F094FAA0F11103DBB2012BF7D945
:10C9E000192818BF84F856001921204600F0D7F9FD
:10C9F000022384F8553010BD70B51D4690F85530AF
:10CA00006E1C1344144680F8553013460A46F1B2A2
:10CA100000F02FFA601970BD10B5012300F1550226
:10CA20000021044600F025FA02221146204600F0BB
:10CA3000FCF963683BB1228F120504D5204603211F
:10CA4000BDE81040184710BDF8B50821044600F0B5
:10CA5000A6F915210746204600F0F9F960F07F029B
:10CA6000D2B215210646204600F0DFF90621204605
:10CA700000F095F90821204600F0E9F960F07F0206
:10CA8000D2B20821204600F0D0F90121204600F062
:10CA9000DEF903060546F8D532462046152100F09A
:10CAA000C4F90821204600F07AF93946204600F002
:10CAB00076F9C5F38010F8BD38B50D46022104465D
:10CAC00000F0B3F9162D07D0204600F018FA854281
:10CAD000FAD184F8545038BD204600F010FA1F28CF
:10CAE000FAD0F6E710B50A0A044601F07F0180F893
:10CAF0002D2080F82C10202100F097F994F82C209C
:10CB000020462121BDE8104000F08FB92DE9F843FF
:10CB1000054616461F4600F12D0800246FF0070950
:10CB2000E2003046394601F033FB09FB04F208F815
:10CB3000010F38323046394601F02AFB04F1240156
:10CB4000C2B2C9B22846013400F06FF9082CE7D10F
:10CB5000BDE8F883A1F10B020F2A07D890F837201F
:10CB60008A4203D080F8371000F00ABA70470020DC
:10CB7000704737B50D0A4185CAB22221044600F03C
:10CB800054F92A462321204603B0BDE8304000F086
:10CB90004CB9000008B5052100F059F9024B00F02E
:10CBA0000F0033F9100008BD48400108113109B2E7
:10CBB0001429A8BF142121EAE171024B5A5C052116
:10CBC00000F033B93240010808B52C2100F03FF9DC
:10CBD000C0F3071008BD38B50C462C21054600F0FF
:10CBE00036F9072C28BF072400F00F0040EA041292
:10CBF000D2B228462C21BDE8384000F016B908B55D
:10CC00002C2100F024F9C0F3420008BD0529A8BF7B
:10CC10000521002938B50C46A8BF0C464FF02C0161
:10CC20000546B8BF072400F012F920F00E0040EAD4
:10CC30004402D2B228462C21BDE8384000F0F5B8B5
:10CC400038B505460C4699B10A782D2100F0EDF86B
:10CC50002E21284600F0FBF8637800F0F80203F07C
:10CC600007031A4328462E21BDE8384000F0DDB8FE
:10CC700038BD08B5092100F0EAF800F00F004000C7
:10CC80005B3840B208BD0029C4BF494249B25B319C
:10CC9000C1F3430242F0C002092100F0C6B808B552
:10CCA000072100F0D4F85B3840B208BD10B5038FFF
:10CCB0000446B2B30B43B1F5807F03870AD002D894
:10CCC000202925D010BDB1F5007F0ED0B1F5005F51
:10CCD00020D010BD00F12E01FFF7B2FF0421204645
:10CCE000FFF794FF53222F2153E02E2100F0AFF8DD
:10CCF00040F01002D2B22E21204600F096F8172103
:10CD0000204600F0A4F840F00202D2B2172140E021
:10CD10002E212BE00E2100F09AF840F00402D2B24E
:10CD200036E023EA0103B1F5807F03870AD002D8F9
:10CD3000202921D010BDB1F5007F09D0B1F5005FE9
:10CD400021D010BD4FF0FF31BDE81040FFF75EBFAE
:10CD5000172100F07CF8172100F0FD02204600F0BA
:10CD600064F8238F9B0619D52E21204600F06FF81A
:10CD700000F0EF022E210CE02E2100F068F840F0C8
:10CD80001002D2B2F6E70E2100F061F800F0FB02CB
:10CD90000E212046BDE8104000F047B810BD70B528
:10CDA00004460D46204600F0AAF8A0F11103DBB2BC
:10CDB000012B0646F6D91F28F4D0032D02D12A46AE
:10CDC000082126E0A84227D0162801D1192D02E01B
:10CDD000192807D1162D0AD1092211462046FFF73E
:10CDE0006BFE04E00F2802D1204600F094F80F2DCE
:10CDF0000DD103212046FFF7D2FF2946204600F03F
:10CE000026F8E06CF4F734FC84F8545004E02A4629
:10CE100029462046FFF750FE304670BD90F840305E
:10CE2000416CC06B0022F4F793BA70B504460D460E
:10CE30001646FFF7F3FF334645F0C002616CE06B26
:10CE400001F08FF9E06BBDE87040F4F7C1BA38B576
:10CE500004460D46FFF7E2FF45F080020023616CB7
:10CE6000E06B01F07EF90546E06BF4F7B1FA284675
:10CE700038BDF7B504460F4615461E46FFF7CEFFF0
:10CE8000616CE06B4023012201F05AF93B46616C72
:10CE9000E06B012201F054F90022E06B0196009250
:10CEA0002B46616CF4F7B0FAE06B03B0BDE8F040DC
:10CEB000F4F78EBA10B50446FFF7B0FF616CE06B73
:10CEC00020230122BDE8104001F03AB907B58DE8F2
:10CED00006000023416CC06B0122F4F795FA03B001
:10CEE0005DF804FB10B50446416CC06B01230022C1
:10CEF00001F026F9E06BBDE81040F4F769BA08B517
:10CF000090F854300F2B04D00121FFF7A0FF00F060
:10CF10001F03184608BD10B50446FFF7F0FF0F28A1
:10CF200011D1E06CF4F7ADFB00214FF49970FFF7DD
:10CF30004BFC01212046FFF78AFF00F01F00082864
:10CF400084F85400F5D110BD10B50446006DF4F717
:10CF500098FB00213E20FFF737FC206DF4F788FB9B
:10CF600000213E20FFF730FC01212046FFF76FFF34
:10CF700000F01F0310F0170F84F85430F4D110BDE7
:10CF800038B508210446FFF70AFF08210546204668
:10CF9000FFF75DFF94F8373000F0E00203F01F0365
:10CFA00020461A430821FFF740FF29462046BDE8E6
:10CFB0003840FFF7F4BE43680BB1002118477047B3
:10CFC0002DE9F0470446884616461F46FFF797FFAF
:10CFD0008146002C00F0D3800F2840F0DF80B8F1AC
:10CFE000180F66D02046FFF796FFB8F1270F00F222
:10CFF0002B81DFE818F042002901280033002901C5
:10D0000029013B00290129012901290129012901BF
:10D01000290129012901550029018B008F007E007B
:10D0200029018400290129012901930097009B000F
:10D030009F002901A300AA00290129012901290132
:10D0400029014E00BA00022F03D98B490320F3F7C0
:10D05000CBFD31882046FFF745FD94E0082FF4D83A
:10D06000D6E900232046FFF751FD8CE0022FECD8D3
:10D0700031882046FFF77DFD85E0012FE5D031782E
:10D08000A1F10B030F2B00F2EC802046FFF762FDAD
:10D0900079E0012FD9D03378002B40F0E2806CE0AA
:10D0A000022FD2D8B6F900102046FFF77FFD0225E7
:10D0B000D9E0012FC9D83378013B052B63D8DFE8CD
:10D0C00003F00507620C1403082102E00F2100E0C1
:10D0D00016212046FFF763FECBE0238F5A0540F16F
:10D0E000C8802046FFF798FCC3E02046FFF7ECFB22
:10D0F000BFE0327820212046FFF7D8FD43E0012F22
:10D10000A3D831782046FFF766FD36E032784FF439
:10D11000806116E032784FF4007112E032784FF4FB
:10D1200000510EE032784FF480410AE032784FF43B
:10D13000006106E032784FF4805102E032784FF41B
:10D1400080712046FFF7B2FD17E0012F3FF67DAF5B
:10D15000238FDB0503D43378052B40F2828096F9C8
:10D1600000102046FFF752FD07E0012F3FF66DAF9C
:10D1700096F900102046FFF786FD012573E06FF059
:10D180001200BDE8F087B9F10F0F5DD03B46324683
:10D1900041462046BDE8F04700F054BFB8F1270FE4
:10D1A000F4D801A353F828F07BD000088DD10008F3
:10D1B00047D000085DD000088DD100088DD100084F
:10D1C0006DD000088DD100088DD100088DD10008E8
:10D1D0008DD100088DD100088DD100088DD10008B7
:10D1E0008DD100088DD10008A1D000088DD1000894
:10D1F0000DD1000815D10008F3D000088DD100082A
:10D20000FFD000088DD10008B3D000088DD10008F0
:10D210001DD1000825D100082DD1000835D1000806
:10D220008DD100083DD100084BD100088DD10008F8
:10D230008DD100088DD100088DD100088DD1000856
:10D2400093D000086BD10008B8F1180F9ED06FF092
:10D2500085050F212046FFF7A2FD15F1860F05D1A8
:10D2600094E76FF01505B9F10F0FF2D02846BDE82D
:10D27000F0870120BDE8F087E50901082DE9F041BC
:10D280000446FFF73CFE0F2806464CD00F212046EF
:10D29000FFF7DDFD022107462046FFF7D8FD7B079B
:10D2A000054603D5636801212046984738073AD5DB
:10D2B000162E01D0112E05D1238F590433D5636862
:10D2C00002212CE0192E01D0122E2CD194F85730C7
:10D2D0001BB916490320F3F787FC013BDBB284F846
:10D2E000573023B994F856102046FFF758FD63686D
:10D2F000CBB1228FD20416D505F0E000202809D04A
:10D3000002D838B1BDE8F081602807D0A02803D04A
:10D31000BDE8F081042102E0062100E0072120465B
:10D32000BDE8F0411847BDE8F08100BFE5090108FC
:10D3300013B50446416CC06BF3F7DCFF0121E06CD0
:10D34000F4F7D2F8E06CF4F79CF90121206DF4F7C2
:10D35000CBF8206DF4F78CF90D4B009401220021DD
:10D36000A06CF4F7FBF82046FFF7AEFA1C2120462C
:10D37000FFF76DFD032807D11C22002104F10C00EA
:10D3800001F046FC002001E04FF0FF3002B010BD7C
:10D39000B7CF00082DE9F34104460F4690461E46DC
:10D3A000FFF788FD01220DF103012046FFF78EFDF6
:10D3B0009DF8035005F07F05023D37B3454505D97B
:10D3C0002046FFF78FFD6FF0680521E0236A0133E7
:10D3D0002362636A2B442A46394620466362FFF77C
:10D3E00075FD022201A92046FFF770FD6EB10122F2
:10D3F000B1182046FFF76AFD2046FFF773FD0721AD
:10D400002046FFF724FD307002E02046FFF76AFD5A
:10D41000284602B0BDE8F0812DE9F04106460D46F0
:10D420009046FFF7CEFA00273C46474512D06A687F
:10D43000A31C13447F2B05F1080514D8F36955F894
:10D44000081C2344F36130462346FFF7D5FA013721
:10D450000446EAE7338F5B0502D43046FFF7DCFA77
:10D460002046BDE8F0816FF08A00BDE8F081000041
:10D4700008B5FFF744FD0838C0B211289ABF024B27
:10D48000185C022008BD00BF804001082DE9F84368
:10D490000F46164698460546002800F0B780A1F1D1
:10D4A0001103152B4DD8DFE803F01827344C4C4CF2
:10D4B0004C204C383C40444C484C4C4C4C4C4C0B55
:10D4C000B8F1010F03D857490320F3F78DFB002370
:10D4D0007370FFF74CFB307004E0B8F1010FF2D924
:10D4E000662333800220BDE8F883B8F1000FEAD04C
:10D4F000FFF7BEFF307009E0038F13F4806F03D095
:10D5000001203070BDE8F883002333700120BDE8AE
:10D51000F883038F13F4007FF1E7038FC3F34033E5
:10D52000F3E7038FC3F38033EFE7038FC3F3C02325
:10D53000EBE7038FC3F30033E7E7038FC3F3002365
:10D54000E3E74346324600F0C9FC10F1860F04467B
:10D5500060D12846FFF7D3FC0F28814611D1284619
:10D56000FFF7D9FC162F1CD004D8012F35D0102F6F
:10D570000ED046E0272F28D02F2F36D0202F1DD0B9
:10D580003FE0162F0DD013D8012F26D0102F44D1F5
:10D59000B8F1010F97D92846FFF7FCFA0224308032
:10D5A0002CE0B8F1000F8ED02846FFF70DFB23E0EA
:10D5B000272F0AD02F2F18D0202F2ED1B8F1000FEF
:10D5C00081D02846FFF71BFB16E0B8F1000F3FF4AF
:10D5D0007AAF2846FFF74DFB0EE0B8F1000F3FF49D
:10D5E00072AF2846FFF730FA06E0B8F1000F3FF4BB
:10D5F0006AAF2846FFF753FB30700124B9F10F0FD3
:10D6000008D10F212846FFF7CAFB03E06FF0120094
:10D61000BDE8F8832046BDE8F8836FF08500BDE8DB
:10D62000F88300BFE5090108094B70B51C68064680
:10D630000D4620460821F2F719FE21463046F3F741
:10D6400053FB2846F2F714FFBDE87040F3F732BBF6
:10D65000080300202DE9F04104460E461546F2F776
:10D66000FFFE27688046A7B13B68236096E8030069
:10D670007B6883E803000A21A7F10800F2F7F6FDB2
:10D6800017F8034C4046F2F7F3FE2046F2F72EFE61
:10D690001FE0A268E3689B1A2269934207DDDDB1AF
:10D6A0004146201DFFF7C0FFF2F7DAFE80460D4B22
:10D6B000E1681B8833804B1CE360236962690B407F
:10D6C00096E8030002EBC30383E803004046F2F749
:10D6D000CFFE0120BDE8F081F2F7CAFE2846BDE882
:10D6E000F08100BF04030020BFF34F8F0549064BB4
:10D6F000CA6802F4E0621343CB60BFF34F8F00BFF0
:10D70000FDE700BF00ED00E00400FA0538B1054B6D
:10D710000A0901F00F019A5C5B5C02704370022001
:10D72000704700BF9240010803461A78591C0AB19D
:10D730000B46FAE7181A7047F8B505460F46164625
:10D740008C18BC4206D0284614F8011DFFF7DEFFF6
:10D750000544F6E77000F8BD07B502AB042243F8B4
:10D76000041D1946FFF7E8FF03B05DF804FB38B568
:10D7700005460C464CB122462946012002F0A4F889
:10D78000002802DB241A0544F4E738BD07B501463A
:10D7900001A8FFF7BBFF022101A8FFF7E8FF03B0D4
:10D7A0005DF804FB07B501466846FFF7D5FF082181
:10D7B0006846FFF7DCFF03B05DF804FB10B50446D4
:10D7C000FFF7B2FF01462046BDE81040FFF7CFBF8C
:10D7D000F8B5064684890F46154600206DB900232A
:10D7E000B289B168FBF7EAFD4FF6C57302199A4298
:10D7F00039680EDD013080B20BE0AE42EFD0234637
:10D80000AA89A968FBF7DAFDEB686D681C44A4B22D
:10D81000E4E73A34204400232022083180B2FBF7A9
:10D82000CDFDC04380B2F8BD2DE9F3410C468046E2
:10D8300003212046F7F725FD054618B92E49032098
:10D84000F3F7D2F90221F7F71CFD07460028F5D0BF
:10D85000EB68032B4CD900F1080122462846AE683C
:10D86000FFF7B6FF002843D13378803B082B30D830
:10D87000DFE803F0052F2F2F2F0C151E2700AB8993
:10D88000B9683246404600F081F822E0EB68009328
:10D89000BA68334621464046F6F7D8F919E0EB68F6
:10D8A0000093BA68334621464046F6F751FA10E035
:10D8B000EB680093BA68334621464046F6F730F8E5
:10D8C00007E0EB680093BA68334621464046F6F716
:10D8D000F3F83178234640F201220320F7F7A4F948
:10D8E000014628B9204602B0BDE8F041F7F73EBF37
:10D8F00002B0BDE8F08100BFE509010838B50D466A
:10D90000144600211A460323F7F73EFE28B1836828
:10D9100000221D705C709A70DA7038BD10B5044634
:10D9200068B190F91030032B0CD142680831FFF731
:10D930004FFF50B1A36840BA5880002010BD6FF06F
:10D940000D0010BD6FF04C0010BD6FF0010010BD58
:10D950002DE9F041DDF81880154600220E461F46DD
:10D96000014608F108031046FFF7C8FF044650B10E
:10D97000806876BA6DBA8680C58027B1424639463E
:10D98000083001F047F82046BDE8F081F7B50646BB
:10D990000C46002A38D0072B36D99188D088083B0E
:10D9A00040BA49BA009389B202F1080382B28120D9
:10D9B000FFF7CEFF074638B3237EFF2B04F10802A2
:10D9C0000CBF002104F11801F5F792FB054610B9D0
:10D9D0000146384613E000231A4619461846F7F761
:10D9E000A1FB836809495E8004464560034640F216
:10D9F00002220220F7F718F9014628B9204603B0A1
:10DA0000BDE8F040F7F7B2BE03B0F0BD0000FFFF85
:10DA100038B505460C4619B301F17000F3F760F80C
:10DA20002846F5F7E7FC38B1D0F810329C4203D114
:10DA300000F5FC70F3F754F804F11C00F3F750F80C
:10DA400004F13800F3F74CF804F15400F3F748F808
:10DA500010220021204601F0DBF800236383637667
:10DA600038BD000008B51022034900F0A1FFB0FA4C
:10DA700080F0400908BD00BFAE1301082DE9F74F43
:10DA8000904600901E469DF83070894609B90020E6
:10DA90005CE0082BFBD80846FFF7E4FF0028F6D12E
:10DAA000824604464FF0980B2A4B0BFB0AF29D1856
:10DAB000494628460192FBF7A8FC019A78B1B8F1D3
:10DAC000000F42D0002E40D0224B02F11000414600
:10DAD0003246184400F09EFF2E766F7635E02846D9
:10DAE000FFF7C0FF10B1002C08BF2C460AF1010A55
:10DAF000BAF1080FD8D1002CC9D0BDF8003063832B
:10DB000010224946204600F085FFB8F1000F07D0EB
:10DB100036B13246414604F1100000F07BFF267614
:10DB2000677607F00707022F04BF032384F89430B9
:10DB30004FF40973A4F886304FF40473C4F8884096
:10DB4000638664632465204600E0284603B0BDE890
:10DB5000F08F00BF344D00202DE9F04107460E46FE
:10DB600011B90020BDE8F0810846FFF77BFF0028CF
:10DB7000F7D10C4D0446A846B5F91A3013B10FB1D0
:10DB8000BB4209D131462846FBF73FFC20B1982023
:10DB900000FB0480BDE8F0810134082C05F19805F4
:10DBA000EAD1DEE7344D002010B50446FFF7D4FF7C
:10DBB00001462046BDE81040FFF72ABF38B510B136
:10DBC00000F1980400E0074C074DAC4205D2204616
:10DBD000FFF748FF18B19834F7E7002038BD20461A
:10DBE00038BD00BF344D0020F451002008B5FFF7C8
:10DBF000E5FF10B1437E1B07F9D508BDF8B5014616
:10DC00000020FFF7A9FF044610B3437E13F0050F71
:10DC10001ED0B0F91A00F5F7EDFB0E4BD0F8D46129
:10DC2000B3F9007004F138052846F2F759FF40F2C5
:10DC30001723A4F84E3004F14C023B4631462846E7
:10DC4000FEF7ECFD637E23F0070343F007036376E2
:10DC50002046F8BDDC10002010B5144600B119B9FB
:10DC60000B490320F2F7C0FF2AB1537E03F00703EC
:10DC7000013B012B01D8002010BD137E0B70127EDA
:10DC800004F1100100F0C6FEB4F91A0010BD00BF87
:10DC9000E5090108F0B503EB43048C424FF00001A5
:10DCA00022D8017005465E1E0F464FF03A0E99428B
:10DCB00019D014782409092C94BF30345734944671
:10DCC0002C709CF8004004F00F04092C94BF3034F1
:10DCD0005734B1426C700CBF3C467446AC70013294
:10DCE00001310335E3E7F0BD0846F0BD2DE9F04111
:10DCF00012B90020BDE8F0811378002BF9D014464A
:10DD0000264601347378002BFAD107464FF0010CF8
:10DD1000964217D33478A4F130055FFA85F8B8F14C
:10DD2000090F06F1FF3E23D9A4F14105052D02D8C4
:10DD3000A4F137051CE0A4F16105052D11D8A4F16B
:10DD4000570515E0BCF1000FD3D1013FB84205D211
:10DD50003A780178397000F8012BF6E71846BDE8EB
:10DD6000F081BCF1000FC4D14FF0010C7646CFE733
:10DD7000724518D8A6F1020E16F8016CA6F130040F
:10DD80005FFA84FCBCF1090F0ED9A6F14104052C01
:10DD900002D8A6F1370407E0A6F16104052C02D8E9
:10DDA000A6F1570400E0002401338B42A1D845EAD4
:10DDB00004143C704FF0000C0137D7E710B504464F
:10DDC00086B0B0F90210214801F02AF861792048A4
:10DDD00001F026F8A1791F4801F022F81E4801F051
:10DDE0001FF8237963B11A0602D51C4801F018F810
:10DDF00023795B0602D51A4801F012F8194800E0B1
:10DE0000194801F097F8237853B104F1080218215A
:10DE10006846FFF73FFF0146144801F001F802E0B1
:10DE2000134801F087F863785BB122780832224406
:10DE300018216846FFF72EFF01460E4800F0F0FF5C
:10DE400002E00D4801F076F806B010BDA2400108CE
:10DE5000AF400108BA400108C3400108CB400108A7
:10DE6000D640010859380108E1400108E5400108A1
:10DE7000F540010807410108174101087FB50C462C
:10DE8000054600B119B90D490320F2F7ADFE0A4667
:10DE900001AE232100F0BCFE304600F04BF9002318
:10DEA000B3FBF4F204FB1232F15CA85C0133414095
:10DEB0000C2BA954F4D104B070BD00BFE5090108D2
:10DEC00010B50446FFF7DAFF034B1A78511C19709E
:10DED00023785340237010BD92020020062938B5E4
:10DEE00004460D46104636D006D8032922D029D83C
:10DEF000B1B3022911D09DE017294AD004D80829CE
:10DF000051D0152932D095E0252948D0292900F093
:10DF10008980192940F08E8035E0012B03D84849CB
:10DF20000320F2F761FE0A4604F12C0100F072FDB5
:10DF3000284638BD072BF2D9082204F12E0100F043
:10DF400069FD7AE0022BEAD1228F520701D508221F
:10DF500004E003806CE0022BE1D1628D028067E077
:10DF6000022BDCD194F8373013800AE0012BD6D194
:10DF7000238F13F0200F02D00123037058E00023F9
:10DF80000370012038BD012BC9D1238F13F0020F7C
:10DF9000F1E7012BC3D194F92820027048E0022B4D
:10DFA000BDD10322DAE7072BB9D9238F5B074CBF1A
:10DFB0002B4602234FF000024CBF04F12E0104F166
:10DFC0002C01042B4270027018D0082B03D0022BB6
:10DFD00033D1134619E00A7882F0020202704A78BF
:10DFE00042708A788270CA78C2700A7902714A795E
:10DFF00042718A798271CA79C27119E00B7883F013
:10E00000020303704B7843700223FF240022C47084
:10E01000FE24827004714271CA5C827119444B788B
:10E02000C3710AE0042B7FF47AAF04F10C01116094
:10E03000184638BD6FF0850038BD082038BD00BFD8
:10E04000E509010870B515461C4619296AD8DFE8AC
:10E0500001F00D691929393949696969696969697D
:10E06000696969696969694E69616958022C03D0F7
:10E070002F490320F2F7B8FD1388FF2BF8D880F85A
:10E0800037304DE0022CF3D800F12C06022200219B
:10E09000304600F0BDFD22462946304600F0BAFC6D
:10E0A000022070BD082CE3D800F12E0608220021C2
:10E0B000304600F0ADFD22462946304600F0AAFC6D
:10E0C000082070BD022CD3D11388022B06D0082B58
:10E0D0002BD1038F43F00403038721E0038F23F048
:10E0E00004030CE0022CC3D11388438518E0127896
:10E0F000038F12B143F0200301E023F020030387D4
:10E10000CEE71278038F12B143F00203F7E723F052
:10E110000203F4E7012CABD192F9003080F82830EB
:10E12000204670BD6FF0850070BD6FF0690070BD56
:10E13000E50901080C22014900F06CBC107AFF1FB0
:10E1400010B586B006AC04F8093D012301930DF12A
:10E15000170300932346F3F757F99DF8170006B00D
:10E1600010BDF0B585B01F4604AB002403F8012DA7
:10E17000012205460E4601920094F3F745F93B460D
:10E18000224631462846FFF7DBFF05B0F0BD000010
:10E19000D0400B1CD1409C46203AD34018435242F9
:10E1A000634693401843704753B94AB9002908BFE2
:10E1B00000281CBF4FF0FF314FF0FF3000F07EB958
:10E1C000ADF1080C6DE904CE00F006F8DDF804E0CE
:10E1D000DDE9022304B070472DE9F0478C460E4676
:10E1E0000446089D002B50D18A4217466CD9B2FADA
:10E1F00082FEBEF1000F0BD0CEF1200420FA04F411
:10E2000001FA0EF644EA060C02FA0EF700FA0EF4D2
:10E210004FEA1749220CBCFBF9F01FFA87F809FBFB
:10E2200010C642EA064600FB08F3B34209D9F619C4
:10E2300000F1FF3280F02281B34240F21F810238A8
:10E240003E44F61AA2B2B6FBF9F309FB136642EAA2
:10E25000064403FB08F8A04509D9E41903F1FF328D
:10E2600080F00A81A04540F20781023B3C44C8EBA4
:10E27000040443EA00400021002D62D024FA0EF489
:10E2800000232C606B60BDE8F0878B4207D9002D1E
:10E2900055D0002185E841000846BDE8F087B3FA73
:10E2A00083F1002940F09080B34202D3824200F211
:10E2B000F880841A66EB03060120B446002D40D096
:10E2C00085E81010BDE8F08712B90127B7FBF2F717
:10E2D000B7FA87FEBEF1000F35D1F31B4FEA17489E
:10E2E0001FFA87FC0121B3FBF8F0220C08FB103663
:10E2F00042EA06460CFB00F3B34207D9F61900F1D7
:10E30000FF3202D2B34200F2CE801046F61AA2B219
:10E31000B6FBF8F308FB136642EA06440CFB03FC69
:10E32000A44507D9E41903F1FF3202D2A44500F253
:10E33000B5801346CCEB040443EA00409CE7294631
:10E340002846BDE8F087CEF1200106FA0EF307FA61
:10E350000EF720FA01F94FEA1748CE4049EA0309BF
:10E36000B6FBF8FA4FEA194408FB1A661FFA87FC55
:10E3700044EA06430AFB0CF29A4200FA0EF40AD968
:10E38000DB190AF1FF3180F087809A4240F28480E5
:10E39000AAF1020A3B449B1A1FFA89F9B3FBF8F170
:10E3A00008FB113349EA034301FB0CF69E4207D9EF
:10E3B000DB1901F1FF326BD29E4269D902393B442D
:10E3C0009B1B41EA0A418EE7C1F1200E22FA0EF4AE
:10E3D0008B40234320FA0EF706FA01F44FEA134C60
:10E3E00026FA0EF63C43B6FBFCF9270C0CFB19662B
:10E3F0001FFA83F847EA064609FB08F7B74202FA14
:10E4000001F200FA01FA08D9F61809F1FF3041D2F9
:10E41000B7423FD9A9F102091E44F61BA0B2B6FBD0
:10E42000FCF40CFB146640EA064704FB08F8B84508
:10E4300007D9FF1804F1FF3028D2B84526D9023C8D
:10E440001F4444EA0940C8EB0707A0FB02894F4577
:10E4500044464E4614D329D065B3BAEB040367EBA8
:10E46000060707FA0EFECB40CF404EEA030385E8CD
:10E4700088000021BDE8F0871346F8E61046E0E684
:10E48000B8EB020469EB03060138E5E70446D8E778
:10E49000114695E78146C0E78A467CE7023B3C444B
:10E4A00048E708460AE702383E442FE7C245E7D36B
:10E4B0003E46D1E72946BDE8F08700BF704700BF60
:10E4C0000A22002101F04EB90A23002201F0B6B859
:10E4D000014B1868704700BF940200208B891A070F
:10E4E0002DE9F0410D46804635D44A68002A6BDD9F
:10E4F000EC6A002C47D003F48052002192B2D8F885
:10E500000060C8F80010002A62D06A6D5F0705D568
:10E5100069686B6B521A0BB12B6CD21A0023296AF3
:10E520004046A047441C39D0AB892A692A60DB04E5
:10E530004FF000026A6045D4696BC8F8006011B3FF
:10E5400005F14403994202D0404600F0AFFB0020A1
:10E550006863BDE8F0810E69AEB10C680E60980783
:10E560000CBF4B690023A41B8B600AE02346324694
:10E57000AF6A296A4046B8470028A4EB0004064465
:10E5800004DD002CF2DC0020BDE8F081AB8943F013
:10E590004003AB814FF0FF30BDE8F081D8F8002098
:10E5A0001D2AF3D8184BD34003F0010383F0010177
:10E5B000002BEBD0AB892C696960D9042C60BBD5EA
:10E5C000002AB9D16865B7E70A6C002A90DCDAE75F
:10E5D0000123296A4046A047431C024602D0AB896A
:10E5E000EC6A93E7D8F80030002BF8D01D2B01D04F
:10E5F000162B02D1C8F80060C5E7AB8943F0400391
:10E60000AB81BDE8F08100BF010040200B6933B34E
:10E6100010B5044682B008B18369ABB1114B994281
:10E6200019D0114B994218D0104B994208BFE1689C
:10E63000B1F90C3013B9002002B010BD204602B071
:10E64000BDE81040FFF74ABF019100F019F90199A8
:10E65000044B9942E5D16168EAE7A168E8E7002048
:10E66000704700BF6C4101084C4101082C41010872
:10E6700020B1054B01461868FFF7C8BF034B04499A
:10E68000186800F043B900BF940200208C410108D3
:10E690000DE6000800207047014900F037B900BFBF
:10E6A0000DE600080020704770B568234D1E03FB7F
:10E6B00005F50E4605F1740100F03EFB044640B13D
:10E6C00000210C30666005F168022160A06000F056
:10E6D0009FFA204670BD00BF1F4B70B51D68AB6927
:10E6E000064613B9284600F039F848356B68AC681F
:10E6F000013B05D521E0013B5A1C04F168041CD004
:10E70000B4F90C20002AF6D1002501234FF6FF7240
:10E71000E281A38165662560A5606560256165610C
:10E72000A5612946082204F15C0000F071FA6563D6
:10E73000A563A564E564204670BD2B680BB11D463A
:10E74000D4E704213046FFF7AFFF286008B1054643
:10E75000CCE70C23336070BD8C4101083D4B3E4932
:10E760001A682DE9F04F90424FF000038364C364B0
:10E77000036508BF012383B008BF83618162074638
:10E78000FFF7AAFF78603846FFF7A6FFB860384663
:10E79000FFF7A2FF7D68F86000240423AB812C60A2
:10E7A0006C60AC606C66EC812C616C61AC61214684
:10E7B00005F15C00082200F02BFABE68DFF89CB07F
:10E7C000DFF89CA0DFF89C90DFF89C80C5F824B0AF
:10E7D00001230922C5F828A0C5F82C90C5F830807F
:10E7E0002D622146F381B28134607460B460746636
:10E7F00034617461B46106F15C000822019300F099
:10E8000007FAFD68366212200222C6F824B0C6F864
:10E8100028A0C6F82C90C6F830802146A881EA814D
:10E820002C606C60AC606C662C616C61AC6105F155
:10E830005C00082200F0ECF9019B2D62C5F824B0C1
:10E84000C5F828A0C5F82C90C5F83080BB6103B08E
:10E85000BDE8F08F8C41010899E60008B5EF00088B
:10E86000DDEF000819F0000839F00008024B0349F9
:10E87000186800F04BB800BF8C4101080DE6000895
:10E88000836903B96AE77047704700BF704700BFEC
:10E89000704700BF704700BF024B0349186800F083
:10E8A0000FB800BF94020020A5E60008024B034900
:10E8B000186800F005B800BF9402002095E6000833
:10E8C0002DE9F04110F148071BD0884600267D68ED
:10E8D000BC68013D0FD4A389012B05F1FF3506D992
:10E8E000B4F90E300133204601D0C04706436B1CFB
:10E8F00004F16804EFD13F68002FE8D13046BDE84D
:10E90000F0813E463046BDE8F08100BF2DE9F84376
:10E9100010F148071FD0884606464FF000097D6871
:10E92000BC68013D11D4A389012B05F1FF3508D93D
:10E93000B4F90E3001332146304602D0C04749EACF
:10E9400000096B1C04F16804EDD13F68002FE6D18B
:10E950004846BDE8F883B9464846BDE8F88300BF9D
:10E9600070B50F4E0F4D761BB61018BF002405D0A2
:10E97000013455F8043B9847A642F9D10A4E0B4D95
:10E98000761BF1F703FCB61018BF002406D0013443
:10E9900055F8043B9847A642F9D170BD70BD00BF41
:10E9A000D4420108D4420108D4420108D4420108EB
:10E9B000032A70B426D940EA01039B0711D00478DA
:10E9C0000D78AC4222D10244431C05E013F8014B00
:10E9D00011F8015FAC4219D19342F7D1002070BC0D
:10E9E00070470C4603461E682568AE42184621460D
:10E9F00003F1040304F10404E1D1043A032A1846A4
:10EA00002146F0D8002ADAD11046E8E7601B70BC36
:10EA1000704700BF844641EA000313F003036DD141
:10EA2000403A41D351F8043B40F8043B51F8043BD1
:10EA300040F8043B51F8043B40F8043B51F8043BD8
:10EA400040F8043B51F8043B40F8043B51F8043BC8
:10EA500040F8043B51F8043B40F8043B51F8043BB8
:10EA600040F8043B51F8043B40F8043B51F8043BA8
:10EA700040F8043B51F8043B40F8043B51F8043B98
:10EA800040F8043B51F8043B40F8043B51F8043B88
:10EA900040F8043B51F8043B40F8043B51F8043B78
:10EAA00040F8043B403ABDD2303211D351F8043B18
:10EAB00040F8043B51F8043B40F8043B51F8043B58
:10EAC00040F8043B51F8043B40F8043B103AEDD2C7
:10EAD0000C3205D351F8043B40F8043B043AF9D218
:10EAE000043208D0D2071CBF11F8013B00F8013BEB
:10EAF00001D30B8803806046704700BF082A13D3F8
:10EB00008B078DD010F003038AD0C3F10403D21A0F
:10EB1000DB071CBF11F8013B00F8013B80D331F843
:10EB2000023B20F8023B7BE7043AD9D3013A11F8C3
:10EB3000013B00F8013BF9D20B7803704B7843702E
:10EB40008B788370604670478842F0B50DD98B187A
:10EB500098420AD28118002A51D09A1A13F8014D0E
:10EB600001F8014D9342F9D1F0BD0F2A48D941EA8D
:10EB700000039B0746D100F1100401F11003154674
:10EB800053F8106C44F8106C53F80C6C44F80C6C8F
:10EB900053F8086C44F8086C103D53F8046C44F8C2
:10EBA000046C0F2D03F1100304F11004E8D8A2F156
:10EBB000100323F00F0302F00F0E1033BEF1030F0A
:10EBC0001944034421D91E1F0D467446043C55F8D0
:10EBD000047B46F8047F032CF8D8AEF1040424F03B
:10EBE000030404342344214402F0030262B1013BD4
:10EBF0000A4411F8014B03F8014F8A42F9D1F0BDE4
:10EC00000346F3E70346F2E7F0BD7246EEE700BFC6
:10EC100070B4840746D0541E002A41D0CDB20346BA
:10EC200002E0621EE4B3144603F8015B9A07F8D1D0
:10EC3000032C2ED9CDB245EA05250F2C45EA054512
:10EC400019D903F110022646103E0F2E42F8105C2F
:10EC500042F80C5C42F8085C42F8045C02F11002D5
:10EC6000F2D8A4F1100222F00F0204F00F041032C7
:10EC7000032C13440DD91E462246043A032A46F8B3
:10EC8000045BFAD8221F22F003020432134404F07A
:10EC900003042CB1C9B21C4403F8011BA342FBD1ED
:10ECA00070BC704714460346C2E700BF30B481B160
:10ECB00051F8043C0439002BB8BFC9181D4B1A6821
:10ECC0002AB18A420AD908680C18A24225D04A60A3
:10ECD000196030BC70478B4203D81A465368002B2A
:10ECE000F9D1146815198D420CD007D808680C1892
:10ECF0009C4218D04B6030BC516070470C230360BD
:10ED000030BC704709680C44111999421460E0D175
:10ED10000ACB0C4453601460DBE7146852684A6005
:10ED200020440860D4E71C685B684B60204408609E
:10ED30005160CEE7F451002070B5CD1C25F00305DD
:10ED400008350C2D38BF0C25002D06463BDBA942AB
:10ED500039D827490A6852B113685B1B04D436E0DE
:10ED600023685B1B1AD522465468002CF8D14968E9
:10ED70001F4C002936D029463046F1F70BFA431CC8
:10ED800021D0C41C24F00304A04205D0211A30462F
:10ED9000F1F700FA013016D0256004E00B2B0DD9F5
:10EDA00023601C44256004F10B0020F00700231DA4
:10EDB000C31A02D05A42E25070BD70BD94420ED0C8
:10EDC00063685360EFE70C233360002070BD0B2BAA
:10EDD00003D8536814460B60E5E71446E0E7134692
:10EDE0001446F8E73046F1F7D5F96060C3E700BF95
:10EDF000F45100200EB410B5044683B018B18369F5
:10EE00000BB9FFF73DFD06A803460190059AA168DE
:10EE1000204600F0EFFE03B0BDE8104003B070479D
:10EE20000FB410B50A4B1C6882B024B1A36913B9A2
:10EE30002046FFF725FD05A803460190049AA16826
:10EE4000204600F0D7FE02B0BDE8104004B0704785
:10EE5000940200202DE9F0410E46804600283ED065
:10EE60008369002B39D084682F4B9C4243D02F4BB1
:10EE70009C4256D02E4B9C4208BFD8F80C40A38928
:10EE80001B073DD52369002B3AD0013EA36816F835
:10EE9000015F013BA360B5B1002B04DB23685A1C62
:10EEA00022601D70F2E7A769BB4222462946404610
:10EEB00001DB0A2DF2D100F013FD0130E6D14FF055
:10EEC000FF30BDE8F081002B21DB23680A22591CAA
:10EED00021601A701046BDE8F081FFF7D1FCD8F828
:10EEE0001830D8F80840002BBED14046FFF7C8FCC8
:10EEF0000D4B9C42BBD1D8F80440A3891B07C1D459
:10EF00002146404600F04EFD0028BED0D7E72246FD
:10EF100040460A2100F0E4FC0130D0D00A20BDE8D0
:10EF2000F081D8F80840AAE76C4101084C4101087B
:10EF30002C410108024B01461868FFF78BBF00BF48
:10EF40009402002038B50C46054608B18369B3B178
:10EF5000114B9C4218D0114B9C4217D0104B9C4235
:10EF600008BFEC682846214601F07AF980B994E898
:10EF70000C00013B511C84E80A00107838BDFFF7F3
:10EF80007FFC054B9C42E6D16C68EBE7AC68E9E797
:10EF90004FF0FF3038BD00BF6C4101084C41010803
:10EFA0002C410108024B01461868FFF7CBBF00BF98
:10EFB0009402002010B50C46B1F90E10F1F708F9D3
:10EFC000002803DB636D0344636510BDA38923F44C
:10EFD0008053A38110BD00BF002070472DE9F04190
:10EFE0001646B1F90C201F46D3050C46054607D539
:10EFF00000220223B1F90E10F1F7F7F8B4F90C2052
:10F00000B4F90E1022F48052A2813B4632462846C3
:10F01000BDE8F041F1F7E0B810B50C46B1F90E10BB
:10F02000F1F7E3F8A389421C0EBF23F4805343F4A5
:10F0300080536065A38110BDB1F90E10F1F7D0B80F
:10F0400070B411F0FF0434D085070FD00378002B83
:10F050005AD09C422BD0431C05E013F8012B002A08
:10F060004FD0944223D09A071846F6D10E0206F4E8
:10F070007F462643036846EA064601E050F8043F0F
:10F0800086EA0305A5F10132A3F1013122EA050266
:10F0900021EA0303134313F0803FEFD0037823B931
:10F0A00032E010F8013F002B2ED09C42F9D170BC09
:10F0B000704784070BD00378002BF8D0431C03E083
:10F0C00002780133002AF2D099071846F8D1026875
:10F0D000A2F1013323EA020313F0803F08D150F874
:10F0E000042FA2F1013323EA020313F0803FF6D08C
:10F0F0000378002BDBD010F8013F002BFBD170BC54
:10F100007047104670BC7047184670BC704700BF0F
:10F1100000000000000000000000000000000000EF
:10F12000A2EB0300704700BF02780B78012A28BFCA
:10F130009A42F5D16DE9044540EA0104CDE9026740
:10F140006FF0000C4FEA447212B380EA010414F02D
:10F15000070F6AD100F0070420F0070004F0030550
:10F1600021F007014FEAC505F0E8042314F0040F6D
:10F17000F1E804670CFA05F462EA040266EA0406A0
:10F180000AD063EA0403624667EA0407664603E0BE
:10F19000F0E80423F1E8046782FA4CF582EA0604F9
:10F1A000A4FA8CF46CBB83FA4CF583EA0705A5FA44
:10F1B0008CF595B950E9022351E9026782FA4CF5C2
:10F1C00082EA0604A4FA8CF483FA4CF583EA070574
:10F1D000A5FA8CF52543DBD09CB92DBAB5FA85F498
:10F1E00024F0070427FA04F1DDE9026723FA04F3A7
:10F1F00003F0FF0001F0FF01FDE80445A0EB010072
:10F20000704724BAB4FA84F424F0070426FA04F10F
:10F21000DDE9026722FA04F202F0FF0001F0FF01CB
:10F22000FDE80445A0EB0100704714F0030F3CD14A
:10F2300010F0030428D150F8082B51F8083B82FA4B
:10F240004CF582EA0305A5FA8CF55DB950F8042C5B
:10F2500051F8043C82FA4CF582EA0305A5FA8CF5D4
:10F26000002DE8D02DBAB5FA85F424F0070423FA6E
:10F2700004F122FA04F202F0FF0001F0FF01FDE8C0
:10F280000445A0EB010070474FEAC40420F00300DE
:10F2900050F8082B21F0030151F8083B0CFA04F454
:10F2A00062EA040263EA0403C9E710F003041AD017
:10F2B000A1EB040120F00300E40750F8042B06D072
:10F2C0000FD28B785FFAA2F4E41A06D12BB1CB7877
:10F2D0005FFAB2F4E41A00D11BB920465DF8104B76
:10F2E000704701F1040150F8042BCC0721F0030111
:10F2F00051F8043B48D824D222F07F4482FA4CF5DE
:10F3000094EA1325A5FA8CF50AD165B951F8043BA6
:10F3100084EA0204B4EB036F0ED150F8042BEBE740
:10F320004FEA132355E035F07F454DD10878FDE8CD
:10F330000445C0F1000070474FEA126203F0FF037A
:10F3400047E002EA1C4482FA4CF594EA1345A5FA18
:10F350008CF50AD165B951F8043B84EA0204B4EB98
:10F36000034F0CD150F8042BEBE74FEA134330E086
:10F3700015EA1C4528D10B884FEA124229E04FEAD2
:10F38000124203EA1C4324E002F0FF0482FA4CF527
:10F3900094EA1365A5FA8CF50AD165B951F8043BD6
:10F3A00084EA0204B4EB032F09D150F8042BEBE7F5
:10F3B0004FEA13630DE015F0FF0F05D10B684FEA1C
:10F3C000122223F07F4304E04FF00000FDE80445E3
:10F3D000704712BA1BBA82FA4CF482EA0304A4FA08
:10F3E0008CF5B5FA85F402FA04F203FA04F34FEA55
:10F3F0001260FDE80445A0EB1360704780EA01024B
:10F40000844612F0030F4FD111F0030F32D14DF8A3
:10F41000044D11F0040F51F8043B0BD0A3F101325D
:10F420009A4312F0803F04BF4CF8043B51F8043B70
:10F4300016D100BF51F8044BA3F101329A4312F0E8
:10F44000803FA4F101320BD14CF8043BA24312F0EF
:10F45000803F04BF51F8043B4CF8044BEAD02346EC
:10F460000CF8013B13F0FF0F4FEA3323F8D15DF89E
:10F47000044B704711F0010F06D011F8012B0CF866
:10F48000012B002A08BF704711F0020FBFD031F8DE
:10F49000022B12F0FF0F16BF2CF8022B8CF8002065
:10F4A00012F47F4FB3D1704711F8012B0CF8012BE8
:10F4B000002AF9D1704700BF0000000000000000E2
:10F4C00090F800F06DE9024520F007016FF0000CA4
:10F4D00010F0070491F820F040F049804FF000044C
:10F4E0006FF00700D1E9002391F840F000F1080027
:10F4F00082FA4CF2A4FA8CF283FA4CF3A2FA8CF35F
:10F500004BBBD1E9022382FA4CF200F10800A4FAC5
:10F510008CF283FA4CF3A2FA8CF3E3B9D1E9042319
:10F5200082FA4CF200F10800A4FA8CF283FA4CF350
:10F53000A2FA8CF37BB9D1E9062301F1200182FA0A
:10F540004CF200F10800A4FA8CF283FA4CF3A2FA10
:10F550008CF3002BC6D0002A04BF04301A4612BA1E
:10F56000B2FA82F2FDE8024500EBD2007047D1E921
:10F57000002304F00305C4F100004FEAC50514F0B0
:10F58000040F91F840F00CFA05F562EA05021CBF81
:10F5900063EA050362464FF00004A9E7002A41D060
:10F5A00040EA010313F00303F0B425D1032A23D961
:10F5B00004680D68AC421FD1043A35D0A4F101357E
:10F5C00025EA040414F0803F31D1071D0D1D0DE024
:10F5D00057F8043B0E68A3F10134B34224EA030454
:10F5E0000AD1043A20D014F0803F23D1032A2946BF
:10F5F000384605F10405EBD803780C789C4202F1FB
:10F60000FF320CD182B114B916E06AB17BB110F8A7
:10F61000013F11F8014FA34202F1FF32F5D0181B50
:10F62000F0BC7047104670471046F0BC7047184653
:10F63000F0BC70470020F3E72046F1E72DE9F04FDA
:10F64000474C83460E46D4F800E000E02646344698
:10F6500014F8015B0EEB0500407800F0080000F0A4
:10F66000FF080028F2D12D2D5CD02B2D04BF75781A
:10F67000B41C002B3ED0102B60D09A46B8F1000F7E
:10F680000CBF6FF000404FF000400027B0FBFAF9CC
:10F69000BC460AFB19000CE0303DAB4219DD7E1C74
:10F6A00005D0CC4523D820D00AFB0C5C012714F8E8
:10F6B000015B0EEB0506767816F0040FECD116F020
:10F6C000030606D0012E14BF57263726AD1BAB42CA
:10F6D000E5DC7B1C16D0B8F1000F10D16046002A83
:10F6E00039D0DFB91160BDE8F08F8542DCDD4FF025
:10F6F000FF37DCE7302D1AD00A239A46BEE7CCF15B
:10F70000000CEBE7B8F1000F4FF022030CBF6FF0D5
:10F7100000404FF00040CBF80030F2B1611E1160A4
:10F72000BDE8F08FB41C75784FF00108A1E723788D
:10F7300003F0DF03582B08D008239EE7302D9CD11F
:10F74000207800F0DF00582897D14FF0100A657834
:10F750005346023492E7BDE8F08FBDE8F08F00BF5A
:10F76000F802002010B4044C13460A4601462068F3
:10F7700010BCFFF763BF00BF940200202DE9F04FDB
:10F78000494C82460E46D4F800E000E02646344656
:10F7900014F8015B0EEB0500407800F0080000F063
:10F7A000FF0C0028F2D12D2D54D02B2D04BF7578DD
:10F7B000B41C5BB1102B5ED04FF0FF38B8FBF3F8F0
:10F7C00003FB08FB6FEA0B0B994607E0302D46D090
:10F7D0000A23DFF8D88099464FF0050B00273846FA
:10F7E0000CE0303DAB4219DD7E1C05D0404522D8EF
:10F7F0001FD009FB0050012714F8015B0EEB050632
:10F80000767816F0040FECD116F0030606D0012E20
:10F8100014BF57263726AD1BAB42E5DC002F0FDBAC
:10F82000BCF1000F00D0404242B17FB91160BDE889
:10F83000F08F5D45DDDD4FF0FF37DDE7BDE8F08F90
:10F840002223CAF800304FF0FF305AB3611E116016
:10F85000BDE8F08FB41C75784FF0010CA9E7237850
:10F8600003F0DF03582B0DD0082399464FF0070B08
:10F870006FF06048B2E7302D0ED1207800F0DF0045
:10F88000582809D14FF0100965784B464FF00F0BFF
:10F8900002346FF07048A1E74FF00F0B6FF0704823
:10F8A00099469BE7BDE8F08FF802002099999919D5
:10F8B00010B4044C13460A460146206810BCFFF7FA
:10F8C0005DBF00BF9402002010B4044C13460A46EA
:10F8D0000146206810BCF0F77FBC00BF94020020F6
:10F8E000F8B50E461446054610B18369002B41D089
:10F8F000254B9C4243D0254B9C4242D0244B9C42FA
:10F9000008BFEC68A389A269A2601A0721D5236900
:10F91000FBB122686169D31A8B42F7B221DA013355
:10F92000A168501C0139A1602060167062699A427A
:10F9300006D0A389DB0701D50A2F01D03846F8BDD0
:10F9400021462846FEF762FE0028F7D04FF0FF3729
:10F95000F4E72146284600F025F80028F6D123696F
:10F96000D7E721462846FEF751FE0028EED122684F
:10F970000123D5E7FEF784FF034B9C42BBD16C68A3
:10F98000C0E7AC68BEE700BF6C4101084C4101080C
:10F990002C410108024B0A4601461868FFF7A0BF38
:10F9A00094020020384B70B51D6806460C4615B110
:10F9B000AB69002B42D0354B9C4245D0344B9C4226
:10F9C00058D0344B9C4208BFEC68B4F90C2093B279
:10F9D00019070CD52069A8B113F001021ED0636984
:10F9E00000225B42A361A260F0B1002070BDDD0681
:10F9F00042D558072AD4206942F00803A3819BB25C
:10FA00000028E9D103F42072B2F5007FE4D030463B
:10FA1000214600F06FF8A3892069DDE7990758BFF8
:10FA20006269A2600028E0D1B4F90C301A06DDD575
:10FA300043F04003A3814FF0FF3070BD2846FEF72E
:10FA40001FFF124B9C42B9D16C68BEE7616B51B18C
:10FA500004F14403994204D03046FFF727F9B4F982
:10FA60000C200023636300232069636022F02402DA
:10FA70002060C1E7AC68A8E742F040020923336088
:10FA80004FF0FF30A28170BD940200206C4101084C
:10FA90004C4101082C41010870B50C46B1F90E101B
:10FAA000002990B015461E4613DB01AAF0F7A2FB11
:10FAB00000280EDB029A02F47042A2F50052B2FA5C
:10FAC00082F252094FF48063002032602B6010B044
:10FAD00070BDA38900221B06326004D5402300209C
:10FAE0002B6010B070BD4FF4806300202B6010B00D
:10FAF00070BD00BF8A8992070B4606D501F1470207
:10FB000001211A601A6159617047F0B583B001ABE9
:10FB10006A460C460546FFF7BFFF00990646284691
:10FB2000FFF70AF9B4F90C30D0B1019A124F0099DD
:10FB3000AF6243F08003A3812060206161611AB944
:10FB40003343A38103B0F0BD2846B4F90E10F0F79B
:10FB500056FBB4F90C300028F2D043F00103EFE774
:10FB60009A05EFD404F1470243F002030121A38177
:10FB7000226022616161E5E799E600089368013B34
:10FB8000002B10B4936007DBCCB21368581C1060D4
:10FB90001970204610BC70479469A34202DBCCB2B6
:10FBA0000A2CF2D110BCFFF79BBE00BF93B1F8B591
:10FBB00014460F460646D51801E0AC4208D03A4636
:10FBC00014F8011B3046FFF7D9FF431CF5D1F8BDEF
:10FBD0000020F8BD00207047936810B5144613B993
:10FBE0005360184610BD00F0D1FB0023A360636092
:10FBF00010BD00BF2DE9F04F9DB088461446039319
:10FC0000814618B18369002B00F00B818B4B98451E
:10FC100000F00D818A4B984500F00C81894B984586
:10FC200008BFD9F80C80B8F80C301D0740F1EF8000
:10FC3000D8F81030002B00F0EA8030238DF82A30FD
:10FC40002378814DDFF804A20021202209918DF84C
:10FC50002920002B00F08580252B264603D117E0B4
:10FC6000252B00F0868016F8013F002BF8D1B6EB6B
:10FC7000040B76D022465B4641464846FFF796FF86
:10FC800001306ED0099B32785B440993002A68D01A
:10FC900000234FF0FF31721C0493079306938DF8F5
:10FCA00053301A930591012604E0049906FA03F3F0
:10FCB0000B430493144664482178052200F0E8FCC5
:10FCC000621C431B0028F0D1049BD80644BF2022AD
:10FCD0008DF853201907217844BF2B228DF853202B
:10FCE0002A2968D0A1F13002092A0BD8079B14F801
:10FCF000011F03EB830302EB4303A1F13002092A46
:10FD0000F5D907932E293FD00322504800F0C0FCBC
:10FD100048B10499CAEB0000402202FA00F041EA1F
:10FD2000000301340493217849488DF828100622F5
:10FD3000013400F0ADFC00285FD0464BEBB103ABC3
:10FD400000934246444B04A94846AFF3008007465F
:10FD50007A1C06D0099B3B4409932378002B7FF43F
:10FD60007BAFB8F80C305B0658D409981DB0BDE8DD
:10FD7000F08FB6EB040B8BD07CE7039B073323F0AB
:10FD8000070308330393E5E761782A291DD0A1F121
:10FD900030020023092A04F101040593B4D814F8B1
:10FDA000011F03EB830302EB4303A1F13002092A95
:10FDB000F5D90593A8E7039A116804320029039244
:10FDC00015DB0791617801349CE7039B1A68059263
:10FDD000002A03F104030393B8BF4FF0FF3204F18C
:10FDE0000203AEBFA178A17805921C468CE7494278
:10FDF00043F0020307910493E4E703AB0093424608
:10FE0000154B04A9484600F0CDF80746A0E7414647
:10FE10004846FFF7C7FD00283FF40FAF4FF0FF3013
:10FE2000A4E7FEF72DFD054B98457FF4F3AED9F816
:10FE30000480F8E6D9F80880F5E600BF6C410108B7
:10FE40004C4101082C41010898420108A0420108D8
:10FE5000A442010800000000ADFB000810B4044CEF
:10FE600013460A460146206810BCFFF7C3BE00BF18
:10FE7000940200202DE9F0470C4691460969A268DA
:10FE8000DDF820808A42B8BF0A46C9F8002094F8FD
:10FE9000431006461F4611B10132C9F800202368FD
:10FEA00099065DD5D9F800200232C9F800202368F0
:10FEB00013F0060F19461DD1E1688A1A002AD8BF2F
:10FEC000194617DD04F1190A002505E0E368D9F8A1
:10FED00000209B1AAB420CDD0123524639463046C6
:10FEE000C047013005F10105F0D14FF0FF30BDE80A
:10FEF000F087216894F84330003318BF01238A0645
:10FF00000AD5E1185A1C302081F84300224494F8A5
:10FF1000451082F84310023304F14302394630465B
:10FF2000C0470130E1D0236803F00603042B29D039
:10FF3000A36822699342C8BF4FF000092FDD9B1AC6
:10FF400099441A34002501E04D4528D0012322466A
:10FF500039463046C047013005F10105F4D1C4E708
:10FF600013F0060F08D1E168D9F800208A1A002A98
:10FF7000D8BF1946A6DCBDE794F84330003318BF5C
:10FF80000123C9E7D9F80000E168A3682269091ACA
:10FF9000934221EAE179D2DCB9F1000FD1D10020FE
:10FFA000BDE8F0872DE9F0430C46097E85B06E2947
:10FFB000064617460C98984604F1430C5AD01AD8B6
:10FFC000632900F0128100F2D68000295CD0582904
:10FFD00040F0F58084F8451022680368DFF864E299
:10FFE000150603F104011ED4550653BF1B680160BA
:10FFF0001B88016019E0732900F0CF807ED86F293B
:020000040801F1
:1000000000F0E480702940F0DA80226842F020029B
:100010002260782384F845300368DFF82CE2150667
:1000200003F10401E0D51B680160D00744BF42F032
:1000300020022260002B40F09080226822F02002F3
:1000400022601021002284F843206068A06000280C
:10005000C0F28880226822F004022260002B62D164
:10006000002840F08180654608296AD0C5EB0C0362
:1000700023610CE023681A0640F1D58003686269A9
:10008000191D01601B681A60002365462361CDF8C5
:1000900000803B4603AA21463046FFF7EBFE0130C5
:1000A00021D02A46236939463046C04701301AD04C
:1000B0002368039813F0020FE36819D01A1A002A74
:1000C00016DD04F11909002504E0E36803981A1A03
:1000D000AA420DDD01234A4639463046C047013069
:1000E00005F10105F1D14FF0FF3005B0BDE8F08317
:1000F0009842B8BF184605B0BDE8F083752965D0B1
:1001000078295CD1226884E76168A1602D200029EC
:10011000C3F1000384F8430021DB22F00402DFF87E
:1001200024E122600A216546B3FBF1F201FB1230A3
:1001300013461EF8002005F8012D002BF4D10829E4
:1001400094D12368D90791D5626823699A428DDCDE
:10015000302305F8013C013D88E7102172E7DFF804
:10016000E4E00A21002BDED19EF8003084F8423012
:1001700004F1420578E7642901D069291FD122687A
:100180000368150603F104013AD51B680160002BD2
:10019000BADBDFF8B0E00A2157E703686268191D8F
:1001A00001601D680021284600F072FA002846D040
:1001B000401B60602061002384F8433067E701231F
:1001C00084F84210236104F14205F4E723681A061B
:1001D0001ED503681A1D1B680260227EDFF864E0EA
:1001E0006F2A14BF0A2108212CE703681A68191D19
:1001F0000123016004F1420584F842202361DAE71B
:10020000550653BF1B680160B3F900300160BEE7BB
:1002100013F0400F036803F1040215BF02601B686E
:100220001B880260D9E713F0400F0368626903F18D
:10023000040101601B6814BF1A801A6024E760681B
:10024000B8E700BFAC420108C0420108838903F04F
:100250000903092B01D000207047FEF709BA00BF3F
:10026000F8B50C46054610B18369002B45D0424BCA
:100270009C4247D0414B9C426FD0414B9C4208BFAF
:10028000EC68B4F90C2093B200219F06616031D470
:100290005E0722D5616B61B104F14403994202D03B
:1002A0002846FEF703FD236C636000206063002B8B
:1002B00043D12369002B52D0B4F90C70BEB2B307FE
:1002C00022D12269226028466369656A216AA847AB
:1002D0000028606009DD0020F8BDD80644D5190764
:1002E0002ED442F00402A281E3E7A3891DD143F09A
:1002F0002003A3814FF0FF30F8BDFEF7C1FA1E4B7B
:100300009C42B7D16C68BCE71E4B1F49186801239B
:10031000A38106F00906FEF7D3FA092EA781D0D1F2
:1003200021462846FEF7DAF8CBE7002243F04003E7
:10033000A38162604FF0FF30F8BDE36B2360F8BD2E
:1003400021462846FEF762F90028D3D1B4F90C20E3
:10035000A060A06122F00802C3E7AC6891E72146E3
:100360002846FFF7C7FBA7E742F0400209232B60AE
:100370004FF0FF30A281F8BD6C4101084C410108EB
:100380002C4101088C4101084D0201089368002BA3
:1003900076D02DE9F04F8B8985B00C461907019076
:1003A000164629D522693AB303F002081FFA88F0ED
:1003B000356800282FD04FF00009B44FC846B24628
:1003C000B84543464A4628BF3B460198B8F1000F5E
:1003D00050D0216AA66AB047002871DDDAF80830EB
:1003E0001B1A8144C0EB0808CAF80830002BE7D17B
:1003F000002005B0BDE8F08F21460198FFF7D2FA42
:10040000002840F03A81A389356803F002081FFAFA
:1004100088F00028CFD113F001095BD14F46029636
:100420001FB39A05D4F808802CD54745C246C0F0C2
:10043000A48013F4906F40F0B18020685246494682
:10044000FEF782FBA0682368C8EB00005344A0605D
:1004500023603846029A93681B1A81443F1A9360BE
:10046000002BC5D0A389002FDBD1D5F800906F6891
:100470000835D5E7D5F80090D5F8048008359FE712
:100480000020704720682369984203D861698F4231
:1004900080F0B780B84528BFB84642464946FEF7C7
:1004A00053FBA3682268C8EB03034244A3602260A5
:1004B000002B49D121460198FEF7A8F8002843D027
:1004C000B4F90C3043F040034FF0FF30A38105B086
:1004D000BDE8F08F8046029082468146B9F1000F58
:1004E0002AD0029B002B4CD0206823696269C84542
:1004F000C34628BFCB4698425F4604D9A36813443D
:100500009B4500F39080934520DB1346A76A216A40
:1005100001985246B847071ED2DDB8EB070823D032
:10052000B368DB1BBA44C7EB0909B360002B3FF487
:100530005FAFB9F1000FD4D10023D5F800A0D5F8F2
:10054000049002930835C9E7404683E75A4651466E
:10055000FEF7FAFAA2682368CBEB02025B44B8EB21
:100560000708A2602360DBD121460198FEF74EF810
:100570000028A5D1CDF80880D2E72068B846BA4651
:100580005CE74A460A21504600F082F800286FD006
:1005900001300123CAEB00080293A5E762692068D5
:1005A000216902EB4208C1EB000A08EBD8780AF196
:1005B00001004FEA680838444045424684BF8046FF
:1005C00042465B0542D511460198FEF7B5FB8346CE
:1005D000002855D052462169FEF71CFAA38923F45E
:1005E000906343F08003A381CAEB08030BEB0A007E
:1005F000C4F81480C4F810B02060A360B846BA46AE
:100600001CE76FF00043BB4228BF3B464A4693FBC2
:10061000F1F30198A66A01FB03F3216AB0470028B1
:100620003FF718AF4CE71A4651460393FEF78CFA92
:100630002268039B01981A4422602146FDF7E6FFD9
:10064000039B00287FF43CAF1F4666E7019800F04B
:100650006FF883460028C7D1019D21692846FEF71F
:1006600025FBB4F90C300C2223F080032A6029E723
:10067000012309F10108029336E74FF0FF30B8E695
:10068000019A0C231360B4F90C301BE700FCFF7FC8
:1006900001F0FF01102A2BDB10F0070F08D010F833
:1006A000013B013A8B422DD010F0070F42B3F6D137
:1006B000F0B441EA012141EA014122F007047FF050
:1006C00000070023F0E80256083C85EA010586EAA7
:1006D000010685FA47F5A3FA87F586FA47F6A5FAE3
:1006E00087F68EB9EED1F0BC01F0FF0102F00702EF
:1006F00032B110F8013B013A83EA010313B1F8D19A
:100700000020704701387047002D06BF354603387A
:10071000073815F0010F07D1013015F4807F02BFB3
:10072000013015F4C03F0130F0BC0138704700BF04
:10073000F9B1F8B506461546B2B10C4600F01CF802
:10074000854201D82046F8BD29463046FEF7F4FA26
:10075000074668B12A462146FEF75CF93046214635
:10076000FEF7A4FA3846F8BDFEF7A0FA2846F8BD11
:10077000F8BD1146FEF7E0BA51F8040C0028BEBFE0
:10078000091851F8043CC018043870474E4D4920F0
:1007900048414E444C4552004D454D204D414E413F
:1007A00047452048414E444C45520042555320464F
:1007B00041554C542048414E444C455200555341FC
:1007C0004745204641554C542048414E444C4552E3
:1007D000004445425547204D4F4E2048414E444C21
:1007E00045520044554D4D592048414E444C4552C8
:1007F000000A49535220737461636B206F766572EF
:10080000666C6F77656400537461636B20706F6909
:100810006E74657220636F727275707465642C20DB
:10082000726573657420746F20746F70206F66201A
:10083000737461636B000A436F6E74657874206231
:1008400065666F726520686172646661756C743A82
:100850000020202072303A2030782530386C780A19
:1008600020202072313A2030782530386C780A20E8
:10087000202072323A2030782530386C780A2020D7
:100880002072333A2030782530386C780A002020E6
:100890007231323A2030782530386C780A202020A6
:1008A0006C723A2030782530386C780A202020701D
:1008B000633A2030782530386C780A2020707372C3
:1008C0003A2030782530386C780A0A004653522F87
:1008D0004641523A0020434653523A203078253060
:1008E000386C780A0020484653523A203078253038
:1008F000386C780A0020444653523A20307825302C
:10090000386C780A0020414653523A20307825301E
:10091000386C780A0020424641523A20307825301F
:10092000386C780A004D4D4641523A2030782530D7
:10093000386C780A004D697363004558435F52452F
:10094000543A2030782530386C780A004174746548
:100950006D7074696E6720746F207265636F6E735B
:10096000747275637420737461746520666F72208D
:10097000646562756767696E672E2E2E00496E206A
:100980004744423A0A2020736574202470633D3046
:1009900078256C780A20206672616D6520300A2007
:1009A0002062740A000A49535220737461636B20F9
:1009B0006F766572666C6F7765642062792061740A
:1009C000206C656173742025642062797465732ED0
:1009D0000A0048415244204641554C542048414E5B
:1009E000444C4552004641494C45442041535345EF
:1009F0005254494F4E2E0025700A002A2A2A2052AE
:100A0000494F54206B65726E656C2070616E69632E
:100A10003A0A25730A0A002A2A2A2068616C74653A
:100A2000642E0A0A006D61696E28293A20546869AB
:100A3000732069732052494F5421202856657273E0
:100A4000696F6E3A20554E4B4E4F574E20286275B7
:100A5000696C646469723A202F686F6D652F656CEC
:100A60006F7065732F50464531352F52494F5429C9
:100A7000290A0069646C65006D61696E005F510050
:100A8000A90B0108B10B0108BA0B0108C30B01083F
:100A9000C90B0108D10B0108DA0B0108E30B0108AF
:100AA000EC0B0108F40B0108FC0B01087374617472
:100AB00065006E616D650009706964207C20252DDC
:100AC0003231737C20252D397351207C207072695E
:100AD000207C20737461636B20202820757365640B
:100AE00029207C2062617365206164647220207C0F
:100AF0002063757272656E7420202020200A000920
:100B000020202D207C206973725F737461636B20D9
:100B100020202020202020202020207C202D20206C
:100B20002020202020202D207C2020202D207C20F3
:100B3000253669202825356929207C20253130700B
:100B4000207C20253130700A000925336869207C1B
:100B500020252D323073207C20252D387320252E22
:100B60003173207C20253369207C2025366920289C
:100B700025356929207C2025313070207C202531C5
:100B80003070200A007C0053554D00092535732034
:100B9000252D3231737C253133732536732025366C
:100BA000692028253569290A0073746F707065649F
:100BB00000736C656570696E6700626C206D75749A
:100BC000657800626C20727800626C2073656E64D8
:100BD00000626C207265706C7900626C20616E79C5
:100BE000666C00626C20616C6C666C00626C206DDF
:100BF000626F780072756E6E696E670070656E6404
:100C0000696E6700004400400000020003000240DB
:100C100002000240070700260048004000000400D0
:100C2000090C0240080C02400707002707060402CF
:100C300001070705030200000030014007000240E1
:100C400006000240050002400400024005000000CA
:100C50000010000001000000003800400F040240B6
:100C60000E0402400D0402400C0402400500000086
:100C7000004000000000000000000040FFFFFFFFF8
:100C800001000000001C0000000C0040FFFFFFFFFF
:100C9000080000000032000002020000030D0108FD
:100CA000070D0108091A00080000000000000000FC
:100CB0000000000052494F54206E6574776F726BCC
:100CC00020737461636B206578616D706C65206161
:100CD00070706C69636174696F6E006E6577206E09
:100CE0006F64653F00416C6C2075702C2072756ECE
:100CF0006E696E6720746865207368656C6C206E21
:100D00006F77007564700073656E64206461746150
:100D1000206F7665722055445020616E64206C69A6
:100D20007374656E206F6E2055445020706F72741E
:100D3000730075736167653A202573205B73656E78
:100D4000647C7365727665725D0A007573616765B0
:100D50003A2025732073656E64203C616464723EA2
:100D6000203C706F72743E203C646174613E205B75
:100D70003C6E756D3E205B3C64656C617920696EEC
:100D80002075733E5D5D0A004572726F723A207580
:100D90006E61626C6520746F20706172736520648F
:100DA000657374696E6174696F6E206164647265E5
:100DB0007373004572726F723A20756E61626C6572
:100DC00020746F2070617273652064657374696E3E
:100DD0006174696F6E20706F7274004572726F7209
:100DE0003A20756E61626C6520746F20636F707954
:100DF000206461746120746F207061636B6574207E
:100E0000627566666572004572726F723A20756E21
:100E100061626C6520746F20616C6C6F63617465D6
:100E20002055445020686561646572004572726F98
:100E3000723A20756E61626C6520746F20616C6C13
:100E40006F6361746520495076362068656164651A
:100E500072004572726F723A20756E61626C652025
:100E6000746F206C6F636174652055445020746802
:100E70007265616400537563636573733A207365CB
:100E80006E74202575206279746528732920746F2B
:100E9000205B25735D3A25750A0075736167653AB5
:100EA00020257320736572766572205B737461729E
:100EB000747C73746F705D0A007374617274007572
:100EC0007361676520257320736572766572207380
:100ED00074617274203C706F72743E0A00457272C5
:100EE0006F723A2073657276657220616C7265610B
:100EF00064792072756E6E696E67206F6E20706FF8
:100F0000727420256C750A004572726F723A2069FE
:100F10006E76616C696420706F72742073706563A3
:100F2000696669656400537563636573733A20731A
:100F300074617274656420554450207365727665DF
:100F400072206F6E20706F7274202568750A0073AE
:100F5000746F70004572726F723A207365727665B5
:100F60007220776173206E6F742072756E6E696E79
:100F7000670A00537563636573733A2073746F7007
:100F80007065642055445020736572766572006503
:100F900072726F723A20696E76616C696420636F59
:100FA0006D6D616E64000000010000000300000030
:100FB000060C024002100240070C02400A0C0240DC
:100FC0005B6175746F5F696E69745F6E6574696685
:100FD0005D206572726F7220696E697469616C69F7
:100FE0007A696E672061743836726632787820725A
:100FF0006164696F202325750A0061743836726652
:1010000032787800252D3339730025303278005B33
:101010006669625F7072696E745F6E6F746966791B
:101020005F72705D207069645B25645D3A202564A1
:101030000A005B6669625F7072696E745F746162F8
:101040006C655D202564292069666163655F69645C
:101050003A2025642C20676C6F62616C3A20257001
:101060002C206E65787420686F703A2025702C20D3
:101070006C69666574696D653A20256C750A000AAD
:101080002D3D20536F7572636520726F75746520F6
:1010900028257029203D2D0A49666163653A20257F
:1010A000640A666C6167733A2025780A7061746817
:1010B0003A2025700A646573743A20004E6F7420DC
:1010C0007365742E002D3D20454E4420282570293F
:1010D000203D2D0A004E65787420486F7000252D44
:1010E00033397320252D31377320252D3339732063
:1010F000252D31307320252D31367320496E7465CE
:1011000072666163650A00457870697265730020D4
:1011100030782530386C7820004E202F252D336410
:1011200020004820202020202000455850495245CA
:101130004400252D3136732000256C752E25303561
:101140006C75004E4556455200535220466C6167FF
:101150007300535220466972737420486F700053B5
:10116000522044657374696E6174696F6E00252D39
:1011700033397320252D33397320252D36732025DF
:101180002D31367320496E746572666163650A009D
:101190002030782530346C7820006970763600294C
:1011A0003A11676E72635F6E65746465763A20709B
:1011B0006F737369626C79206C6F737420696E74DD
:1011C0006572727570742E007E7E20534E495020D9
:1011D000253269202D2073697A653A2025337520E0
:1011E000627974652C20747970653A20004E4554FC
:1011F000545950455F554E44454620282569290AD3
:10120000004E4554545950455F4E45544946202898
:101210002569290A004E4554545950455F53495891
:101220004C4F5750414E20282569290A004E4554FD
:10123000545950455F4950563620282569290A00DF
:101240004E4554545950455F49434D505636202819
:101250002569290A004E4554545950455F5544505C
:1012600020282569290A004E4554545950455F5598
:101270004E4B4E4F574E20282569290A007E7E206E
:10128000504B54202020202D2025326920736E6978
:1012900070732C20746F74616C2073697A653A20C6
:1012A00025336920627974650A00504B5444554DCA
:1012B000503A206461746120726563656976656483
:1012C0003A00504B5444554D503A206461746120AB
:1012D000746F2073656E643A00504B5444554D5002
:1012E0003A20726563656976656420736F6D657415
:1012F00068696E6720756E657870656374656400F3
:10130000706B7464756D7000FF02000000000000D7
:10131000000000000000001A52504C0001020000C2
:10132000366C6F00FF7F3F1F0F07030120202074E2
:101330007970653A2025336868752020636F64658D
:101340003A2025336868750A00202020636B737586
:101350006D3A20307825303468780A00FFFFFE802F
:101360000000000000000000000000000000FF017D
:101370000000000000000000000000000001FF026B
:101380000000000000000000000000000001FF025B
:101390000000000000000000000000000002FF024A
:1013A00000000000000000000001FF00000000003D
:1013B000000000000000000000000000000000002D
:1013C00000000000000000000000000000013031BB
:1013D00032333435363738396162636465660030DC
:1013E000313233343536373839414243444546008B
:1013F000696C6C6567616C2076657273696F6E20CD
:101400006669656C643A20256868750A00747261C3
:101410006666696320636C6173733A2030782530A7
:101420003278202845434E3A20307825782C2044C5
:101430005343503A20307825303278290A00666CC0
:101440006F77206C6162656C3A2030782530356C9E
:10145000780A006C656E6774683A202568752020EC
:101460006E657874206865616465723A2025752020
:1014700020686F70206C696D69743A2025750A00C8
:10148000736F7572636520616464726573733A206B
:1014900025730A0064657374696E6174696F6E20E8
:1014A000616464726573733A2025730A00303030CA
:1014B0003030303030007368656C6C3A20696E6390
:1014C0006F72726563742071756F74696E670068FE
:1014D000656C70004465736372697074696F6E0047
:1014E000436F6D6D616E6400252D3230732025735E
:1014F0000A007368656C6C3A20636F6D6D616E6491
:10150000206E6F7420666F756E643A2025730A0032
:101510007265626F6F74005265626F6F74207468D9
:1015200065206E6F6465007073005072696E74732D
:1015300020696E666F726D6174696F6E2061626F93
:1015400075742072756E6E696E672074687265615D
:1015500064732E0070696E67360050696E6720767E
:1015600069612049434D5076360072616E646F6D3B
:101570005F696E697400696E697469616C697A6526
:1015800073207468652050524E470072616E646F1C
:101590006D5F6765740072657475726E73203332A7
:1015A00020626974206F662070736575646F2072A5
:1015B000616E646F6D6E657373006966636F6E66EE
:1015C000696700436F6E666967757265206E657442
:1015D000776F726B20696E74657266616365730004
:1015E000666962726F757465004D616E6970756CC5
:1015F00061746520746865204649422028696E66DA
:101600006F3A2027666962726F757465205B61644A
:10161000647C64656C5D2729006E636163686500A6
:101620006D616E616765206E65696768626F7220C3
:1016300063616368652062792068616E6400726F1F
:1016400075746572730049507636206465666175FD
:101650006C7420726F75746572206C69737400729B
:10166000706C0072706C20636F6E66696775726172
:1016700074696F6E20746F6F6C20282772706C20F5
:1016800068656C702720666F72206D6F72652069C7
:101690006E666F726D6174696F6E290010150108B6
:1016A00017150108419B0008271501082A15010894
:1016B0004B9B0008541501085A150108B9B50008DC
:1016C0006A15010876150108559B00088B1501085D
:1016D000961501088D9B0008BA150108C31501086D
:1016E00079A40008E0150108E9150108E9AE000831
:1016F0001916010820160108D1B100083E1601088C
:1017000046160108CDB300085F16010863160108EC
:10171000A5BE00080000000000000000000000005E
:1017200050524E4720696E697469616C697A6564CC
:1017300020746F2063757272656E742074696D65B4
:101740003A2025640A0050524E4720696E69746938
:10175000616C697A656420676976656E2076616C74
:1017600075653A2025640A004F464600534C4545AE
:1017700050005354414E4442590049444C45005294
:1017800058005458005245534554002530387800CD
:101790002873686F727429206164647265737300C2
:1017A0006C6F6E67206164647265737300736F752C
:1017B0007263652061646472657373206C656E6723
:1017C0007468006368616E6E656C007061676500C7
:1017D0006E6574776F726B206964656E7469666993
:1017E000657200545820706F776572205B696E20B7
:1017F00064426D5D006D61782E2072657472616E59
:10180000736D697373696F6E730043534D4120723A
:10181000657472696573004343412074687265732F
:10182000686F6C64205B696E2064426D5D00656E5C
:101830006372797074696F6E00656E63727970742B
:10184000696F6E206B65790075736167653A202555
:1018500073203C69665F69643E20736574203C6B4D
:1018600065793E203C76616C75653E0A002020203B
:101870002020205365747320616E20686172647744
:101880006172652073706563696669632073706552
:1018900063696669632076616C75650A2020202083
:1018A00020203C6B65793E206D6179206265206F58
:1018B0006E65206F662074686520666F6C6C6F774C
:1018C000696E670A202020202020202A20226164BF
:1018D000647222202D2073657473202873686F72E0
:1018E000742920616464726573730A2020202020AB
:1018F00020202A2022616464725F6C6F6E67222050
:101900002D2073657473206C6F6E67206164647240
:101910006573730A202020202020202A2022616461
:1019200064725F73686F727422202D20616C69612C
:101930007320666F72202261646472220A20202064
:10194000202020202A20226368616E6E656C222090
:101950002D207365747320746865206672657175D7
:10196000656E6379206368616E6E656C0A20202065
:10197000202020202A20226368616E22202D2061F1
:101980006C69617320666F7220226368616E6E6598
:101990006C220A202020202020202A202263736D20
:1019A000615F7265747269657322202D207365749E
:1019B000206D61782E206E756D626572206F6620D5
:1019C0006368616E6E656C2061636365737320612B
:1019D0007474656D7074730A202020202020202AE2
:1019E00020226363615F7468726573686F6C642240
:1019F000202D2073657420454420746872657368D7
:101A00006F6C6420647572696E672043434120697E
:101A10006E2064426D0A202020202020202A2022CF
:101A20006E696422202D20736574732074686520AC
:101A30006E6574776F726B206964656E7469666930
:101A4000657220286F72207468652050414E2049CD
:101A500044290A202020202020202A20227061678B
:101A60006522202D20736574207468652063686189
:101A70006E6E656C2070616765202849454545207C
:101A80003830322E31352E34290A202020202020D3
:101A9000202A202270616E22202D20616C696173E2
:101AA00020666F7220226E6964220A202020202086
:101AB00020202A202270616E5F696422202D20611F
:101AC0006C69617320666F7220226E6964220A203D
:101AD0002020202020202A2022706F77657222206B
:101AE0002D20545820706F77657220696E206442F3
:101AF0006D0A202020202020202A20227265747266
:101B0000616E7322202D206D61782E206E756D62BE
:101B10006572206F662072657472616E736D697391
:101B200073696F6E730A202020202020202A202233
:101B30007372635F6C656E22202D20736574732051
:101B400074686520736F7572636520616464726583
:101B50007373206C656E67746820696E2062797497
:101B6000650A202020202020202A202273746174FE
:101B70006522202D20736574207468652064657665
:101B80006963652073746174650A20202020202019
:101B9000202A2022656E637279707422202D2073B2
:101BA00065742074686520656E6372797074696FFE
:101BB0006E206F6E2D6F66660A2020202020202068
:101BC0002A20226B657922202D2073657420746889
:101BD0006520656E6372797074696F6E206B6579CC
:101BE00020696E2068657861646563696D616C2049
:101BF000666F726D61740A00756E006572726F7245
